:100000000C9418140C9442140C9442140C94421442
:100010000C9442140C9442140C9442140C94421408
:100020000C9442140C9442140C9442140C944214F8
:100030000C9442140C940E740C9442140C944214BC
:100040000C9442140C94C8710C9443C20C94421446
:100050000C94323B0C94283B0C9442140C944214A4
:100060000C9442140C9442140C9442140C944214B8
:100070000C9442140C9442140C9442140C944214A8
:100080000C9442140C9442140C9442144E414E4968
:100090004E495459494E46CDCCCC3D0AD7233C1746
:1000A000B7D13877CC2B329595E6241FB14F0A0093
:1000B0000020410000C84200401C4620BCBE4CCA83
:1000C0001B0E5AAEC59D7400407A10F35A00A07200
:1000D0004E18090010A5D4E80000E8764817000083
:1000E000E40B54020000CA9A3B000000E1F5050051
:1000F0000080969800000040420F000000A086019A
:10010000000000102700000000E803000000006469
:1001100000000000000A00000000000100000000D4
:10012000002C76D888DC674F0823DFC1DFAE59E1A9
:10013000B1B796E5E3E453C63AE651997696E8E618
:10014000C28426EB898C9B62ED407C6FFCEFBC9CEB
:100150009F40F2BAA56FA5F490055A2AF75C936BFD
:100160006CF9676DC11BFCE0E40D47FEF520E6B5B8
:1001700000D0ED902E0300943577050080841E0892
:100180000000204E0A000000C80C333333330F98B0
:100190006E12831141EF8D2114893BE65516CFFE77
:1001A000E6DB18D1844B381BF77C1D901DA4BBE403
:1001B00024203284725E228100C9F124ECA1E53D45
:1001C00027434F4D4D554E49434154494F4E0044EE
:1001D000525952554E004552524F525300494E46C5
:1001E0004F004543484F00486F74656E6420496472
:1001F0006C652054696D656F757400486F74656E29
:10020000642049646C652054696D656F75740A00DB
:100210002121204B494C4C20636175736564206239
:100220007920746F6F206D75636820696E616374E7
:100230006976652074696D65202D2063757272651D
:100240006E7420636F6D6D616E643A200053544F7D
:10025000505045442E20005072696E7465722073B0
:10026000746F707065642064756520746F206572AA
:10027000726F72732E2046697820746865206572EB
:10028000726F7220616E6420757365204D39393943
:1002900020746F20726573746172742E2028546507
:1002A0006D70657261747572652069732072657313
:1002B00065742E20536574206974206166746572BC
:1002C0002072657374617274696E67290A004E6FDB
:1002D00020436865636B73756D2077697468206C63
:1002E000696E65206E756D6265722C204C61737449
:1002F000204C696E653A20004E6F20436865636B41
:1003000073756D2077697468206C696E65206E75F1
:100310006D6265722C204C617374204C696E653A75
:100320002000636865636B73756D206D69736D6123
:100330007463682C204C617374204C696E653A209C
:10034000004C696E65204E756D6265722069732080
:100350006E6F74204C617374204C696E65204E750D
:100360006D6265722B312C204C617374204C696E68
:10037000653A20004D3131300053657269616C205F
:10038000737461747573206D69736D617463680A49
:100390000053442072656164206572726F720A00B6
:1003A0004D6564696120496E7365727465640050BF
:1003B0006C65617365205265736574005052494ED7
:1003C0005445522048414C5445440025533A202579
:1003D0005300706F7765726F6666004B494C4C45F1
:1003E000442E20005072696E7465722068616C74CE
:1003F00065642E206B696C6C28292063616C6C65C8
:1004000064210A006563686F3A004572726F723A40
:10041000000A4D6561737572656420706F696E7452
:10042000733A0A00357835206D6573682E205A209E
:100430006F66667365743A2000206E6F7420656E77
:1004400074657265642E0A0050726F62696E67206F
:10045000506F696E740025532025692F256900208F
:100460006F6620004D424C2047323920706F696E14
:10047000742000290A004A206F7574206F6620726C
:10048000616E67652028302D00290A0049206F75AC
:1004900074206F662072616E67652028302D0047DA
:1004A00032384C30004D6573682070726F62696E2F
:1004B0006720646F6E65004D6573682070726F62AF
:1004C000696E6720646F6E652E0A005374617274E2
:1004D000206D6573682070726F62696E672077693E
:1004E00074682022473239205331222066697273A2
:1004F000742E0A004732395332004732384C300AE2
:10050000473239533200686173206E6F2064617422
:10051000612E0A004D65736820426564204C657643
:10052000656C696E67200053206F7574206F6620BC
:1005300072616E67652028302D35292E0A0020490A
:100540006E76616C6964206578747275646572207A
:1005500000536C6565702E2E2E004D6573682070FB
:100560006F696E74206F7574206F662072616E679C
:10057000650A00436C69636B20746F205265737564
:100580006D652E2E2E004E6F204D6F76652E004528
:100590006E642066696C65206C6973740A0042653C
:1005A00067696E2066696C65206C6973740A004E19
:1005B0006F206D656469610A00706175736500285C
:1005C0006E6F2066696C65290043757272656E7482
:1005D0002066696C653A20005344207072696E741D
:1005E000696E67206279746520004E6F74205344F1
:1005F000207072696E74696E670A002E0A00446585
:100600006C6574696F6E206661696C65642C204648
:10061000696C653A200046696C652064656C657498
:1006200065643A002569730025696D2025697300AA
:100630002569682025696D20256973002569642076
:100640002569682025696D20256973002569792051
:10065000256964202569682025696D202569730056
:100660005072696E742074696D653A20006F6B007A
:100670006F666600E201DD01D601CF01C10144458C
:100680004255473A0020573A0042656420436F6F55
:100690006C696E672E2E2E00426564204865617479
:1006A000696E672E2E2E00544D334420456E6465CE
:1006B0007233204F46462E004649524D574152450F
:1006C0005F4E414D453A4D61726C696E20322E305D
:1006D0002E375F4457372E332E3120544D3344206C
:1006E0004533534D444E4E202841707220323920FC
:1006F000323032312031343A31343A3039292053D2
:100700004F555243455F434F44455F55524C3A68FD
:10071000747470733A2F2F6769746875622E636FF3
:100720006D2F496E73616E6974794175746F6D6177
:1007300074696F6E2F4D61726C696E2F747265658E
:100740002F437265616C6974794477696E5F322EEC
:10075000302050524F544F434F4C5F5645525349EF
:100760004F4E3A312E30204D414348494E455F545B
:100770005950453A544D334420456E6465723320D8
:1007800045585452554445525F434F554E543A31A3
:1007900020555549443A63656465326132662D34AB
:1007A0003161322D343734382D396231322D633591
:1007B000356336326633363766660A002F2F004DB2
:1007C00031343520533C696E6465783E206F757412
:1007D000206F662072616E67652028302D31290AEE
:1007E00000205200416363656C65726174696F6ECD
:1007F0003A2050005741524E494E4721204C6F77C6
:10080000205A204A65726B206D6179206C656164A5
:1008100020746F20756E77616E74656420706175E9
:100820007365732E0A004D32303620580020204D5B
:1008300061783A2000200020204D696E3A20005354
:100840006F667420656E6473746F70733A2000462F
:10085000523A0020466C6F773A20004D424C2041BE
:10086000646A757374205A0020643A0020693A0063
:1008700020703A00496E76616C6964206578747204
:10088000756465720A0064697300656E0043290A25
:100890000061626C656420286D696E2074656D70FE
:1008A0002000436F6C6420657874727564657320F2
:1008B00061726520004F4646004F4E00426564203D
:1008C0004C6576656C696E6720004661696C65648D
:1008D00020746F20656E61626C6520426564204CF7
:1008E0006576656C696E670A004D657368204265C0
:1008F00064204C6576656C20646174613A0A004935
:100900006E76616C6964206D6573682E0A004D65B2
:10091000736820706F696E74206F7574206F662025
:1009200072616E67650A004D34323120696E636F03
:10093000727265637420706172616D657465722096
:1009400075736167650A004F66667365747320414D
:1009500070706C696564004572723A20546F6F2044
:100960006661722100546F6F206661722066726F3B
:100970006D207265666572656E636520706F696E65
:10098000740A00454550524F4D204F4B0A004D38D8
:100990003400446F6E65207072696E74696E6720F2
:1009A00066696C650A004D3737004D333100496E7A
:1009B00076616C69642065787472756465720A008A
:1009C00020573A00436F6F6C696E672E2E2E0048D9
:1009D000656174696E672E2E2E0045202553002315
:1009E000646566696E652044454641554C545F0018
:1009F0004B6420004B6920004B702000504944207C
:100A00004175746F74756E652066696E697368658B
:100A100064212050757420746865206C61737420A3
:100A20004B702C204B6920616E64204B6420636FF7
:100A30006E7374616E74732066726F6D2062656C84
:100A40006F7720696E746F20436F6E666967757289
:100A50006174696F6E2E680A0050494420417574B4
:100A60006F74756E65206661696C656421207469B8
:100A70006D656F75740A00504944204175746F7438
:100A8000756E65206661696C6564212054656D70C2
:100A90006572617475726520746F6F20686967682C
:100AA0000A00204B643A2000204B693A2000204B7A
:100AB000703A200020436C6173736963205049448D
:100AC000200A002054753A2000204B753A2000205F
:100AD0006D61783A2000206D696E3A200020643AFA
:100AE000200020626961733A20005049442041751A
:100AF000746F74756E652073746172740A00504966
:100B000044204175746F74756E65206661696C650B
:100B100064212054656D706572617475726520740E
:100B20006F6F20686967680A0050494420417574F6
:100B30006F74756E65206661696C65642120426121
:100B400064206865617465722069640A00504944D4
:100B5000204175746F74756E65004572723A207528
:100B600074663820666F6E74206E6F7420696E69CB
:100B70007469616C697A65642E004572723A2075F9
:100B800074663820666F6E74206E6F7420696E69AB
:100B90007469616C697A65642E004572723A2075D9
:100BA00074663820666F6E74206E6F7420696E698B
:100BB0007469616C697A65642E0042656400456EF3
:100BC000636C6F73757265002568753A25303268FD
:100BD000750025303268753A25303268750020205E
:100BE00020202020200020202020003FFFF038007F
:100BF0007030FC3020FC102078102030102C00D0F9
:100C00002E31D02F7BD02F7BD02E31D02C00D02076
:100C1000301020781020FC1030FC303800703FFF7E
:100C2000F03FFFF03800703186302387102787901F
:100C30002F87D02F03D0203010207810207810205C
:100C400030102F03D02F87D027879023871031862D
:100C5000303800703FFFF0041040020820020820E6
:100C6000041040082080104100104100082080043A
:100C700010400000001FFFF81FFFF863616E6365FE
:100C80006C005072696E742041626F72746564000A
:100C90004D32350050617573696E672E2E2E0072CD
:100CA0006573756D65004D32340046696C2E2044C5
:100CB00069612E004F6666004F6E004520696E2008
:100CC0006D6D5E33005654726176204D696E00562C
:100CD0006D696E00566D6178204500566D61782013
:100CE0005A00566D6178205900566D617820580081
:100CF000416D6178204500416D6178205A00416D59
:100D00006178205900416D6178205800412D54725E
:100D10006176656C00412D526574726163740041A7
:100D20006363656C0056652D4A65726B00565A2DDB
:100D30004A65726B0056592D4A65726B0056582DE4
:100D40004A65726B00452073746570732F6D6D007A
:100D50005A2053746570732F6D6D0059205374655C
:100D600070732F6D6D00582053746570732F6D6D07
:100D700000416476616E6365642053657474696EC6
:100D80006773003F0043616E63656C00496E697470
:100D9000004D34323800496E697469616C697A6556
:100DA00020454550524F4D0046696C616D656E742B
:100DB0000053746570732F6D6D004A65726B00414E
:100DC0006363656C65726174696F6E0056656C6F04
:100DD000636974790053657420486F6D65204F66B0
:100DE000667365747300436F6E66696775726174CC
:100DF000696F6E004C6576656C696E6720446F6E36
:100E00006521004D6F7665205A0047323953320014
:100E1000000C0F00FE07022503BB017FFE08FE0841
:100E2000FE05080806000040F0C88888987810057C
:100E30000808060000C0F88888888888F805050535
:100E40000600012030F83020050808060000207058
:100E5000F820202020E00509090600FF2070A8A83E
:100E6000B888887020070505070001D86C366CD853
:100E70000509090600FFF8A88888888888A8F80569
:100E80000A0A0600FE205050505088A8A888700317
:100E9000030306000340A040FFFFFFFFFFFFFFFF2B
:100EA000FFFFFFFFFFFFFFFFFFFFFFFFFFFF000050
:100EB000000605FF01070706020080808080800091
:100EC00080030303060105A0A0A005060606000096
:100ED00050F85050F8500509090600FF2070A8A0EE
:100EE0007028A87020050707060000C8C810204019
:100EF000989805070706000040A0A040A890680148
:100F000003030602058080800309090601FF2040D3
:100F1000408080804040200309090601FF80404056
:100F200020202040408005070706000020A87020F0
:100F300070A8200505050600012020F820200203E6
:100F4000030601FFC04080050101060003F802020C
:100F500002060100C0C005070706000008101020A7
:100F6000404080050707060000708898A8C8887070
:100F700003070706010040C040404040E005070766
:100F8000060000708808102040F8050707060000DA
:100F9000F808103008887005070706000010305068
:100FA00090F81010050707060000F880F008088880
:100FB00070050707060000304080F088887005073C
:100FC00007060000F808101020202005070706007B
:100FD0000070888870888870050707060000708890
:100FE0008878081060020505060100C0C000C0C076
:100FF0000206060601FFC0C000C0408003050506CA
:1010000001012040804020050303060002F800F89B
:101010000305050601018040204080050707060002
:101020000070881020200020050707060000708847
:10103000B8A8B88070050707060000708888F8888F
:101040008888050707060000F04848704848F00502
:1010500007070600007088808080887005070706F3
:101060000000F04848484848F0050707060000F827
:101070008080F08080F8050707060000F88080F087
:10108000808080050707060000708880809888703F
:10109000050707060000888888F8888888030707FE
:1010A000060100E04040404040E005070706000020
:1010B000381010101090600507070600008890A0F7
:1010C000C0A090880507070600008080808080808F
:1010D000F805070706000088D8A8888888880507CB
:1010E000070600008888C8A89888880507070600B2
:1010F0000070888888888870050707060000F088D7
:1011000088F080808005070706000070888888A81E
:101110009068050707060000F08888F0A090880511
:1011200007070600007088807008887005070706AA
:101130000000F82020202020200507070600008856
:10114000888888888870050707060000888888884E
:1011500050502005070706000088888888A8A850F6
:101160000507070600008888502050888805070773
:101170000600008888502020202005070706000070
:10118000F80810204080F80309090601FFE080807C
:101190008080808080E005070706000080404020B6
:1011A0001010080309090601FFE02020202020205C
:1011B00020E0050303060005205088050101060014
:1011C000FEF803030306010580402005050506001F
:1011D0000070087888780507070600008080F0888E
:1011E0008888F00505050600007080808870050776
:1011F0000706000008087888888878050505060035
:10120000007088F08070050707060000304840E055
:101210004040400507070600FE70888888780870FF
:101220000507070600008080F08888888803070784
:101230000601004000C0404040E00409090601FEEC
:101240001000301010101090600507070600008095
:10125000808890E09088030707060100C040404066
:101260004040E0050505060000D0A8A8A8A805058F
:1012700005060000B0C888888805050506000070CE
:10128000888888700507070600FEF0888888F08047
:10129000800507070600FE78888888780808050515
:1012A00005060000B0C880808005050506000078AE
:1012B000807008F00507070600002020F820202095
:1012C0001805050506000088888898680505050644
:1012D000000088888850200505050600008888A839
:1012E000A85005050506000088502050880507070E
:1012F0000600FE888888502040800505050600000D
:10130000F8102040F80309090601FF204040408002
:10131000404040200109090602FF808080808080D3
:101320008080800309090601FF8040404020404042
:10133000408005030306000248A890FF4142530085
:10134000504C41004E65787420506F696E740025D2
:1013500069202F2025750047323953310047323933
:10136000533200436C69636B20746F204265676978
:101370006E00486F6D696E672058595A0053746F3C
:1013800072652053657474696E6773004C6F616495
:101390002053657474696E677300426564205A0057
:1013A0004F6666004F6E00426564204C6576656C42
:1013B000696E67004C6576656C20426564004D6F10
:1013C00074696F6E00426564004E6F7A7A6C6500D6
:1013D00046616E20537065656400436F6E66696791
:1013E00075726174696F6E00526573746F726520F7
:1013F00044656661756C7473004C6F61642053655D
:101400007474696E67730053746F726520536574EA
:1014100074696E677300507265686561742024207A
:10142000436F6E6600416476616E63656420536548
:101430007474696E6773004D61696E003F004261AC
:10144000636B0053746F70004D3231005072696EDF
:10145000742066726F6D204D656469610052656C21
:1014600065617365204D65646961004D32320043EA
:101470006F6E66696775726174696F6E0054656D31
:101480007065726174757265004D6F74696F6E007E
:10149000526573756D65205072696E740041747485
:1014A000616368204D656469610054756E65005321
:1014B000746F70205072696E74005061757365208E
:1014C0005072696E7400496E666F20536372656571
:1014D0006E0043616E6E6F7420656E74657220736A
:1014E00075626469723A2000022E2E000152656610
:1014F00072657368004D61696E002100486F746504
:101500006E6420746F6F20636F6C64004261636B64
:101510000050726F63656564004D6F74696F6E0093
:1015200044697361626C6520537465707065727391
:10153000004D383400426564204C6576656C696EF8
:1015400067004175746F20486F6D65004732380041
:101550004D61696E00507265686561742024204594
:101560006E64005072656865617420242042656471
:101570000054656D70657261747572650040133C4E
:1015800013436F6F6C646F776E00507265686561AE
:101590007420240046616E205370656564004265C6
:1015A00064004E6F7A7A6C65004D61696E0042612D
:1015B000627973746570205A00466C6F77004661DB
:1015C0006E20537065656400426564004E6F7A7AE0
:1015D0006C6500426564205A005370656564004D77
:1015E00061696E00486F6D696E67204661696C6560
:1015F00064006F70656E0054524947474552454438
:10160000003A20007A5F6D696E00795F6D696E0047
:10161000785F6D696E005265706F7274696E6720D5
:10162000656E6473746F70207374617475730A00EF
:1016300020746F6F206C6F6E67206578747275739D
:10164000696F6E2070726576656E7465640A00203D
:10165000636F6C6420657874727573696F6E207047
:10166000726576656E7465640A0000000000000013
:101670000000000000005761726E696E673A2048F2
:101680006F6D696E672042756D702044697669736D
:101690006F72203C20310A0002020400007A4300ED
:1016A000007A4300007A430000004100000041003E
:1016B00000004000007A4300007A4300007A4300B3
:1016C0000000000000000000000000536574746911
:1016D0006E67732053746F72656400454550524FB6
:1016E0004D20496E697469616C697A65640A003BD2
:1016F000200020440020490020204D33303120506C
:10170000005049442073657474696E67733A002011
:10171000460020420020480020204D31343520531F
:10172000004D6174657269616C20686561747570E3
:1017300020706172616D65746572733A0020204794
:101740003239205334205A00204A002020473239B1
:1017500020533320490020204D3432302053004D97
:1017600065736820426564204C6576656C696E67B8
:101770003A0020204D323036205800486F6D6520E9
:101780006F66667365743A0020580020530020206D
:101790004D323035204200416476616E6365643AB3
:1017A00020423C6D696E5F7365676D656E745F7432
:1017B000696D655F75733E20533C6D696E5F66654C
:1017C0006564726174653E20543C6D696E5F74722D
:1017D0006176656C5F66656564726174653E20580C
:1017E0003C6D61785F785F6A65726B3E20593C6D35
:1017F00061785F795F6A65726B3E205A3C6D6178F3
:101800005F7A5F6A65726B3E20453C6D61785F650B
:101810005F6A65726B3E0020540020520020204D0C
:10182000323034205000416363656C6572617469C5
:101830006F6E2028756E6974732F7332293A2050A9
:101840003C7072696E745F616363656C3E20523CEC
:10185000726574726163745F616363656C3E20548A
:101860003C74726176656C5F616363656C3E0020F9
:10187000204D3230312058004D6178696D756D20F2
:10188000416363656C65726174696F6E2028756E63
:101890006974732F7332293A0020204D323033207F
:1018A00058004D6178696D756D206665656472617B
:1018B0007465732028756E6974732F73293A005309
:1018C000746570732070657220756E69743A0020BB
:1018D000440020204D323030205300204469736191
:1018E000626C65640A0046696C616D656E74207394
:1018F000657474696E67733A0020204D3134392065
:1019000043203B20556E69747320696E2043656CDB
:10191000736975730A0020286D6D290020204732F5
:1019200031202020203B20556E69747320696E2081
:101930006D6D0000803B4400803B4400002041006E
:101940000096420000A0420000A0420000C84300F0
:1019500000BE42D0070000D0070000640000004B2A
:1019600000000024F4D43050C38E20C2A24017825D
:101970008B7011127A910D816CD90AA861E108C7A8
:10198000586607615143061E4B5D05C145A7041A01
:10199000411104093D9803713931034036DB02657A
:1019A000339102D4305402802E1D02632CEE017557
:1019B0002AC501B028A001102781018F2564012BC1
:1019C000244B01E0223401AC211F018D200D018048
:1019D0001FFC00841EED00971DDF00B81CD200E63E
:1019E0001BC600201BBC00641AB200B219A8000A72
:1019F00019A0006A189900D117910040178B00B503
:101A000016840031167E00B31579003A157300C7AD
:101A1000146F0058146A00EE1366008813630025E3
:101A2000135E00C7125B006C12570015125400C100
:101A300011510070114F0021114B00D61049008D3B
:101A40001047004610440002104200C00F400080C2
:101A50000F3E00420F3C00060F3B00CB0E380093B8
:101A60000E37005C0E3500270E3400F30D3200C136
:101A70000D3100900D3000600D2E00320D2D00054F
:101A80000D2C00D90C2B00AE0C2900850C29005C14
:101A90000C2700350C27000E0C2600E80B2400C490
:101AA0000B2400A00B23007D0B23005A0B210039CF
:101AB0000B2100180B2000F80A1F00D90A1E00BBDA
:101AC0000A1E009D0A1D00800A1D00630A1C0047B3
:101AD0000A1B002C0A1B00110A1A00F7091A00DD64
:101AE000091900C4091900AB091900920917007BF4
:101AF000091800630917004C091600360916002062
:101B00000916000A091500F5081500E0081400CCB4
:101B1000081400B8081400A4081400900813007DED
:101B20000812006B0813005808120046081200340F
:101B3000081100230811001208110001081100F01B
:101B4000071000E0071000D0071000C0071000B019
:101B5000070F00A107100091070E0083070F007404
:101B6000070F0065070E0057070E0049070E003BE0
:101B7000070D002E070E0020070D0013070D0006AD
:101B8000070D00F9060C00ED060D00E0060C00D470
:101B9000060C00C8060C00BC060C00B0060C00A425
:101BA000060B0099060C008D060B0082060B0077D1
:101BB000060B006C060B0061060A0057060B004C72
:101BC000060A0042060A0038060A002E060A002409
:101BD000060A001A060A001006090007060A00FD98
:101BE000050900F4050900EB050900E2050900D923
:101BF000050900D0050900C7050900BE050900B5A3
:101C0000050800AD050800A50509009C050800941D
:101C10000508008C050800840508007C0508007490
:101C20000508006C050700650508005D05070056FE
:101C30000508004E05070047050700400508003865
:101C4000050700310507002A050700230507001CCA
:101C5000050600160507000F050700080506000227
:101C6000050700FB040600F5040700EE040600E883
:101C7000040600E2040700DB040600D5040600CFDA
:101C8000040600C9040600C3040600BD040600B72C
:101C9000040600B1040500AC040600A6040600A07A
:101CA0000405009B04060095040500900406008AC4
:101CB00004050085040500800406007A040500750B
:101CC000040500700405006B04050066040500614E
:101CD0000405005C04050057040500520405004D8E
:101CE00004050048040500430405003E0404003ACE
:101CF00004050035040500300404002C0405002709
:101D0000040400230405001E0404001A0404001641
:101D1000040500110404000D040400090405000476
:101D200004040000040400FC030400F8030400F4AD
:101D3000030400F0030400EC030400E8030400E4DF
:101D4000030400E0030400DC030400D8030400D40F
:101D5000030400D0030400CC030400C8030300C53F
:101D600003030024F404D9201BC40C5C0E9804C4A3
:101D7000095F0265077101F405F900FB04B300482F
:101D8000048700C10369005803550003034500BEE2
:101D9000023A008402310053022A0029022500047D
:101DA000022000E4011C00C8011900AF01170098CF
:101DB0000114008401130071011000610110005131
:101DC000010E0043010D0036010B002B010B00201A
:101DD000010B00150109000C01090003010800FBBB
:101DE000000800F3000800EB000700E4000600DE36
:101DF000000600D8000600D2000600CC000500C78F
:101E0000000500C2000500BD000400B9000400B5D3
:101E1000000400B1000400AD000400A9000400A506
:101E2000000300A20003009F0004009B0003009831
:101E30000003009500020093000300900003008D52
:101E40000002008B0003008800020086000200846C
:101E5000000300810002007F0002007D0002007B81
:101E60000002007900020077000100760002007491
:101E700000020072000100710002006F0002006D9C
:101E80000001006C0002006A0001006900020067A6
:101E900000010066000100650001006400020062AC
:101EA00000010061000100600001005F0002005DB0
:101EB0000001005C0001005B0001005A00010059B4
:101EC00000010058000100570001005600010055B4
:101ED00000010054000100530000005300010052B3
:101EE00000010051000100500001004F0001004EB0
:101EF0000000004E0001004D0001004C0001004BAD
:101F00000000004B0001004A0001004900010048A8
:101F100000000048000100470001004600000046A4
:101F2000000100450000004500010044000100439D
:101F30000000004300010042000000420001004197
:101F400000000041000100400001003F0000003F90
:101F50000001003E0000003E0001003D0000003D89
:101F60000001003C0000003C0000003C0001003B80
:101F70000000003B0001003A0000003A0001003977
:101F8000000000390001003800000038000000386F
:101F90000001003700000037000100360000003665
:101FA000000000360001003500000035000000355B
:101FB0000001003400000034000000340001003350
:101FC0000000003300000033000100320000003246
:101FD000000000320001003100000031000000313B
:101FE0000001003000000030000000300001002F30
:101FF0000000002F0000002F0000002F0001002E25
:102000000000002E0000002E0001002D0000002D19
:102010000000002D0000002D0001002C0000002C0D
:102020000000002C0000002C0001002B0000002B01
:102030000000002B0000002B0001002A0000002AF5
:102040000000002A0000002A0001002900000029E9
:1020500000000029000000290000002900010028DC
:1020600000000028000000280000002800000028D0
:1020700000010027000000270000002700000027C3
:1020800000000027000100260000002600000026B6
:1020900000000026000000260001002500000025A9
:1020A000000000250000002500000025000000259C
:1020B000000100240000002400000024000000248F
:1020C0000000002400010023000000230000002382
:1020D0000000002300000023000000230000002374
:1020E0000001002200000022000000220000002267
:1020F0000000002200000022000100210000002159
:10210000000000210000002100000021000000214B
:10211000000000210001002000000020000000203D
:10212000000000200000002000000020000000202F
:10213000000000200001001F0000001F0000001F21
:102140000000001F0000001F0000001F0000001F13
:102150000001001E0000001E0000001E0000001E06
:10216000000000043700001E290000511B00005829
:1021700010000010090000CC0400007802000041AB
:1021800001000020436F756E7420583A0042656468
:1021900000453100626564002C2073797374656DAD
:1021A0002073746F70706564212048656174657276
:1021B0005F49443A200048656174696E6720466152
:1021C000696C65640048656174696E672066616961
:1021D0006C6564004D3131322053687574646F77DB
:1021E0006E001000C90210012C0140012201700193
:1021F0001801B0010E01F00104015002FA00B00212
:10220000F0003003E600D003DC009004D20070053B
:10221000C800A006BE000008B400B009AA00D00B98
:10222000A000600E960060118C000015820020193D
:102230007800C01D6E00A0226400B0275A00902CC8
:10224000500000314600E0343C0010383200903A33
:102250002800603C1E00A03D1400803E0A00203F84
:102260000000544845524D414C2052554E41574173
:102270005900546865726D616C2052756E617761AA
:1022800079004572723A204D415854454D50004DE9
:10229000415854454D502074726967676572656492
:1022A000004572723A204D494E54454D50004D49FB
:1022B0004E54454D502074726967676572656400BD
:1022C000202F002042403A0020403A007C3C3E5EF5
:1022D0002B3D3F2F5B5D3B2C2A225C0043616E6EE1
:1022E0006F74206F70656E20737562646972200070
:1022F00053442063617264206F6B0A006F70656ED7
:10230000526F6F74206661696C65640A00766F6C49
:10231000756D652E696E6974206661696C65640A05
:10232000004E6F20534420636172640A000A4D32EC
:1023300034004D3233202573002E0A006F70656E15
:10234000206661696C65642C2046696C653A2000E2
:1023500046696C652073656C65637465640A00206A
:1023600053697A653A200046696C65206F70656E26
:1023700065643A2000454E4420535542524F55540F
:10238000494E450A002220706F730022207061724E
:10239000656E743A2200535542524F5554494E458A
:1023A0002043414C4C207461726765743A2200539B
:1023B000756263616C6C204F766572666C6F770036
:1023C0004578636565646564206D61782053554286
:1023D000524F5554494E452064657074683A005711
:1023E000726974696E6720746F2066696C653A2043
:1023F00000667265736800646F696E6700206669C5
:102400006C653A20004E6F7720002F6175746F2540
:10241000632E670070012C0190012701B001220199
:10242000C0011D01F00118011002130130020E015C
:102430006002090190020401C002FF000003FA00DB
:102440004003F5008003F000D003EB002004E60019
:102450007004E100E004DC004005D700C005D200B4
:102460004006CD00D006C8008007C3003008BE007B
:10247000F008B900C009B400B00AAF00B00BAA0060
:10248000D00CA500000EA000500F9B00C0109600BD
:102490005012910000148C00C0158700B017820004
:1024A000B0197D00D01B7800001E730040206E0024
:1024B00090226900F024640040275F0090295A00B0
:1024C000E02B5500102E500020304B0010324600FB
:1024D000E033410090353C0010373700703832004F
:1024E000A0392D00B03A2800A03B2300603C1E001C
:1024F000103D1900903D1400103E0F00703E0A0080
:10250000C03E0500003F0000403FFBFF803FF6FF5C
:10251000C03FF1FF2020506C616E6E65724275669F
:1025200066657242797465733A200020467265656B
:10253000204D656D6F72793A2000436F6D70696C44
:1025400065643A2041707220323920323032310ACB
:1025500000204C61737420557064617465643A2086
:10256000323032312D30342D3138207C2041757499
:10257000686F723A2054696E794D616368696E655F
:102580007333440A00322E302E375F4457372E33D0
:102590002E310A004D61726C696E0020536F6674B3
:1025A000776172652052657365740A002057617403
:1025B0006368646F672052657365740A0020427215
:1025C0006F776E206F75742052657365740A0020F2
:1025D00045787465726E616C2052657365740A008B
:1025E000506F77657255700A0073746172740A00D7
:1025F0004739310A47315A350A4739300A4D38349C
:102600000A4D31303453300A4D3134305330004D9F
:1026100031303031006F6B006572726F72207772EB
:102620006974696E6720746F2066696C650A00447E
:102630006F6E6520736176696E672066696C652EC2
:102640000A004D323900456E6473746F7073002553
:102650005320256320256320256320256300205A0D
:102660003A0020593A0020583A00656E6473746F3E
:102670007073206869743A200000000001020009AC
:102680000A0000000004030807000000000000002A
:10269000000000000000000000004D6F766520255E
:1026A000736D6D004D6F766520302E316D6D004D70
:1026B0006F766520316D6D004D6F76652031306D20
:1026C0006D004D6F766520417869730045787472AE
:1026D00075646572004D6F7665205A004D6F7665A2
:1026E0002059004D6F76652058005072696E742035
:1026F00066726F6D204D6564696100FFFFFF486F72
:102700006D652025732573257320466972737400E7
:10271000220A00556E6B6E6F776E20636F6D6D6170
:102720006E643A202200544D334420456E64657235
:10273000332052656164792E005072696E74696E3F
:10274000672E2E2E005072696E742050617573656D
:102750006400204500205A00205900204D393220C5
:10276000580020453A00205A3A0020593A00583A79
:10277000004572726F722077726974696E67207497
:102780006F20454550524F4D210A0020746F6F2035
:102790006C6F6E6720657874727573696F6E2070E8
:1027A000726576656E7465640A0020636F6C6420E0
:1027B000657874727573696F6E2070726576656E78
:1027C0007465640A00526573656E643A2000000007
:1027D0002200250028002B000000210024002700F3
:1027E0002A00020202020202020204040404040497
:1027F00004040303030303030303010101010101B3
:102800000101010204081020408001020408102088
:1028100040800102040810204080804020100804FD
:1028200002012F2F616374696F6E3A00A7D67ADDBB
:1028300011241FBECFEFD0E4DEBFCDBF12E0A0E079
:10284000B1E0E4E5F7ED01E00BBF02C007900D92A7
:10285000AE31B107D9F727E1AEE1B2E001C01D9278
:10286000A93BB207E1F714E1C7E1D4E104C0219725
:10287000FE010E9401E9C631D107C9F70E94CBD7FA
:102880000C949DEB0C9400008F929F92AF92BF929C
:10289000CF92DF92EF92FF92CF936B017C0120E009
:1028A00030E0A9010E941CE287FD9FC06DEB77E339
:1028B00086E095E3A70196010E9413E96B017C0174
:1028C00020E030E040E251E40E9482E220E030E08B
:1028D00048EC52E40E9482E24B015C0120E030E0CF
:1028E000A901C701B6010E941CE220E030E040EAE5
:1028F00050E487FF04C020E030E040EA50ECC5011E
:10290000B4010E9413E920E030E040E251E40E946B
:1029100096E90E9408EA6B017C018BE2F7FE09C090
:10292000F094E094D094C094C11CD11CE11CF11C23
:102930008DE28093D503C701B60120E137E240E084
:1029400050E00E94E2E88AE0882E912CA12CB12C64
:10295000CA01B901A50194010E94E2E8605D60939B
:10296000D603C701B60128EE33E040E050E00E94F4
:10297000E2E8CA01B901A50194010E94E2E8605DA4
:102980006093D703C701B60124E630E040E050E091
:102990000E94E2E8CA01B901A50194010E94E2E89F
:1029A000605D6093D8038EE28093D903C701B601BE
:1029B000A50194010E94E2E8C62FCA01B901A50150
:1029C00094010E94E2E8605D6093DA03C05DC09309
:1029D000DB0385ED93E0CF91FF90EF90DF90CF90F8
:1029E000BF90AF909F908F9008956DEB77E386E056
:1029F00095EB60CF8F929F92AF92BF92CF92DF9272
:102A0000EF92FF92CF936B017C0120E030E0A901AF
:102A10000E941CE287FDAAC06DEB77E386E095E398
:102A2000A70196010E9413E96B017C0120E030E0D0
:102A3000A9010E941CE287FF9EC0C701B601905801
:102A400020E030E040E251E40E9482E220E030E009
:102A500040E251E40E9482E220E030E040EA50E4AB
:102A60000E9413E920E030E040E251E40E9496E940
:102A70000E9408EA6B017C0180E28093D50360E24A
:102A800080E1C81687E2D806E104F1048CF0C701A2
:102A9000B60120E137E240E050E00E94E2E8CA01DE
:102AA000B9012AE030E040E050E00E94E2E8605DD9
:102AB0006093D60360E288EEC81683E0D806E1048E
:102AC000F1048CF0C701B60128EE33E040E050E09D
:102AD0000E94E2E8CA01B9012AE030E040E050E09B
:102AE0000E94E2E8605D6093D70360E284E6C81666
:102AF000D104E104F1048CF0C701B60124E630E012
:102B000040E050E00E94E2E8CA01B9012AE030E06A
:102B100040E050E00E94E2E8605D6093D8038AE004
:102B2000882E912CA12CB12CC701B601A5019401CE
:102B30000E94E2E8C62FCA01B901A50194010E94D2
:102B4000E2E8605D6093D9038EE28093DA03C05DB2
:102B5000C093DB0385ED93E0CF91FF90EF90DF9082
:102B6000CF90BF90AF909F908F9008956DEB77E3DB
:102B700086E095EB55CF20E030E040E251E4C7011C
:102B8000B60162CFCF93DF93EC01CB01BA010E9473
:102B900023E220E030E040E251E40E9496E920E0A8
:102BA00030E0A9010E9413E9688379838A839B83BB
:102BB000DF91CF9108950E9423E220E030E040E2CF
:102BC00051E40E9496E920E030E0A9010E9413E957
:102BD0000C94FA14CF93DF93EC01CB01BA010E945D
:102BE00023E220E030E048EC52E40E9496E920E045
:102BF00030E0A9010E9413E9688379838A839B836B
:102C0000DF91CF9108950E9423E220E030E048EC6C
:102C100052E40E9496E920E030E0A9010E9413E905
:102C20000C944414CF93DF93EC01CB01BA010E94C2
:102C300023E220E030E0A9010E9413E96883798350
:102C40008A839B83DF91CF910895CF93DF93EC012B
:102C5000CB01BA010E9423E220E030E0A9010E94EA
:102C600013E9688379838A839B83DF91CF910895E9
:102C7000CF93DF93EC01CB01BA010E9423E22AE05B
:102C800037ED43E25DE30E9496E920E030E0A901E0
:102C90000E9413E90E940FEA688379838A839B83E9
:102CA000DF91CF910895CF93DF93EC01CB01BA016F
:102CB0000E9423E22AE037ED43E25DE30E9496E9B9
:102CC00020E030E0A9010E9413E9688379838A83B8
:102CD0009B83DF91CF910895CF93DF93EC01CB01DC
:102CE000BA010E9423E220E030E04AE754E40E9467
:102CF00096E920E030E0A9010E9413E96883798316
:102D00008A839B83DF91CF910895FC01849108957C
:102D1000FC0180810895FC0180E09191992329F0C4
:102D2000907C9038D1F38F5FF8CF08951198000010
:102D3000000087FD52C0419800000000119A000079
:102D4000000011980000000086FD53C0419800006B
:102D50000000119A0000000011980000000085FD9D
:102D600046C0419800000000119A00000000119830
:102D70000000000084FD39C0419800000000119A55
:102D80000000000011980000000083FD2CC0419855
:102D900000000000119A00000000119800000000DF
:102DA00082FD1FC0419800000000119A0000000041
:102DB00011980000000081FD12C041980000000041
:102DC000119A0000000011980000000041980000D6
:102DD0000000119A000000000895419AADCF419A79
:102DE000EDCF419AE0CF419AD3CF419AC6CF419AD5
:102DF000B9CF419AACCF90E080E00895CF93DF93B4
:102E0000DB01F9019C919130C1F0943080F0945035
:102E10009C938830D1F480819181009771F0019763
:102E200091838083480F591FEA01188206C08C35B0
:102E300039F49C5F9C93943041F4DF91CF910895D5
:102E40008B3339F781E08C93F8CF20813181B90140
:102E50006F5F7F4F71836083420F531FEA01888346
:102E6000808191818F3591056CF7E7CF0F931F9388
:102E700081E00091C2161091C3162091C4163091C2
:102E8000C5164091BE165091BF166091C016709144
:102E9000C116041715072607370708F480E01F91AD
:102EA0000F910895282F90914003833021F495FDD0
:102EB0000FC094FD0FC0892F90E0B0E0A0E004C0E7
:102EC000B695A795979587952A95D2F7817008951D
:102ED00081E0089580E0089580915301882341F0B6
:102EE0006091D0037091D10341E081E00C942CBC3F
:102EF000089563E972E084E690E00E94BA946AEB78
:102F000072E084E690E00C94BA9481110C947917E5
:102F100068EB71E084E190E00C94BA94CF93DF9376
:102F200000D000D0CDB7DEB70E940FEA0E9421E2A8
:102F300069837A838B839C83CE0101960E94E09003
:102F40000F900F900F900F90DF91CF9108950E94F6
:102F500023E22AE037ED43E25DE30E9496E920E0B8
:102F600030E0A9010E9413E90C948E17CF92DF92F2
:102F7000EF92FF92CF93DF9300D000D0CDB7DEB7B2
:102F80006B017C0120E030E0A9010E941CE287FD7A
:102F90001BC06DEB77E386E095E3A70196010E94E5
:102FA00013E969837A838B839C83CE0101960E9407
:102FB000E0900F900F900F900F90DF91CF91FF90C6
:102FC000EF90DF90CF9008956DEB77E386E095EB7F
:102FD000E4CF0E9423E22AE037ED43E25DE30E9462
:102FE00096E920E030E0A9010E9413E90C94B6179D
:102FF0000E9423E220E030E0A9010E9413E90C9432
:10300000B617CF92DF92EF92FF926B017C0120E026
:1030100030E0A9010E941CE287FD26C06DEB77E33A
:1030200086E095E3A70196010E9413E96B017C01FC
:1030300020E030E0A9010E941CE220E030E040E006
:103040005FE387FF04C020E030E040E05FEBC701B2
:10305000B6010E9413E90E9408EACB01FF90EF90AD
:10306000DF90CF900C947E926DEB77E386E095EB4A
:10307000D9CF0E9423E220E030E0A9010E9413E9A9
:103080000C9401180E9423E220E030E04AE754E467
:103090000E9496E920E030E0A9010E9413E90C9417
:1030A000E794EF92FF920F931F9383E8E82E8DE051
:1030B000F82E06E91DE030E020E045E95DE165E835
:1030C0007DE08CE89DE00E94C0C41F910F91FF90AD
:1030D000EF9008950E9489740C9485170E943C8F8C
:1030E0000C9479170C949A770C949A770C949A779D
:1030F0000C949A770C944C770C944C770C944C77F6
:103100000C944C770E9478A60C948517AF92BF92CE
:10311000CF92DF92EF92FF920F931F93CF93DF93A3
:103120006B01E9014A3009F4B8C0453109F06AC0C1
:10313000DB011296ED91FC91F280C681D781139A42
:1031400088E28A950000E9F7BF2CB29420EFB22202
:1031500030E1A32EAF0C48E2E42E88EF0E949616D1
:103160008E2D8A950000E9F7BFE1BF1508F481C0F4
:103170008F2D807780680E9496168B2D0E94961660
:103180008E2D8A950000E9F780E80E94961680E06F
:103190000E9496168E2D8A950000E9F78AEF0E940C
:1031A00096168E2D8A950000E9F78E01005F1F4F5D
:1031B0008881807F0E94961689918295807F0E94E7
:1031C0009616C017D107A1F78E2D8A950000E9F752
:1031D000F394E0E1BE0EFA10C0CF1398D601129618
:1031E000CD91DC91CE010E948DC28111EEC1DF91A3
:1031F000CF911F910F91FF90EF90DF90CF90BF90F4
:10320000AF900895FB0102811381423309F498C104
:1032100008F49CC1463409F489C1473409F48CC1CF
:103220004B3329F589812B81D80112966C91129725
:1032300013964C91213009F4DFC1233009F0A9C164
:1032400038EF380F582F91E0431708F490E041E031
:10325000531708F040E031E0561708F430E0592FDA
:10326000542B352309F0BDC1942309F0BAC181E084
:10327000BECF80EE8F0D8068807F0E9496168F2DC6
:103280008295807F0E9496168E2D8A950000E9F720
:1032900080E80E94961680E87BCF0B9A1398399AA3
:1032A0004198099A119A139A88E28A950000E9F7E1
:1032B00088E790E0CEE9DFE0FE013197F1F7019772
:1032C000D9F788EF0E94961618E2812F8A950000A0
:1032D000E9F780E20E94961680E00E949616812F00
:1032E0008A950000E9F780E00E94961680E80E9427
:1032F0009616812F8A950000E9F780E00E949616C5
:1033000080E10E949616812F8A950000E9F7CE0190
:103310000197F1F7CE010197F1F7CE010197F1F78F
:10332000CE010197F1F7CE010197F1F7CE01019798
:10333000F1F7CE010197F1F7CE010197F1F7CE0138
:103340000197F1F7CE010197F1F7CE010197F1F75F
:10335000CE010197F1F7CE010197F1F7CE01019768
:10336000F1F72197F1F780E20E94961680E40E941F
:103370009616812F8A950000E9F780E20E94961642
:1033800080E60E9496161A950000E9F710E0D0E05A
:10339000C8E28D2F807780680E949616812F0E9448
:1033A00096168C2F8A950000E9F780E80E94961601
:1033B00080E00E9496168C2F8A950000E9F78AEF2C
:1033C0000E9496168C2F8A950000E9F780E21198EA
:1033D00000000000419800000000119A0000000069
:1033E000119800000000419800000000119A0000B0
:1033F0000000119800000000419800000000119AA0
:10340000000000001198000000004198000000003A
:10341000119A00000000119800000000419800007F
:103420000000119A0000000011980000000041986F
:1034300000000000119A0000000011980000000038
:10344000419800000000119A00000000119800004F
:103450000000419800000000119A0000000011983F
:1034600000000000419800000000119A00000000D8
:10347000119800000000419800000000119A00001F
:103480000000119800000000419800000000119A0F
:1034900000000000119800000000419800000000AA
:1034A000119A0000000011980000000041980000EF
:1034B0000000119A000000001198000000004198DF
:1034C00000000000119A00000000119800000000A8
:1034D000419800000000119A0000000011980000BF
:1034E0000000419800000000119A000000009C2F8D
:1034F0009A950000E9F7815009F069CF88EF0E94A2
:1035000096168C2F8A950000E9F7DF5F105FD032A6
:1035100009F03FCF80E00E94961680EC0E9496163C
:10352000CA950000E9F7139881E061CED80115969D
:103530008C91888381E05BCEF80181818883FACF0A
:10354000B901C8010E94AAC281E051CE443171F094
:10355000473109F08CCE1882F801828189838581F8
:1035600081508A8383818B8381E041CED801159677
:103570004C91159750E0440F551F70E060E016968F
:103580008D919C910E943EEBC8010E94A3C281E0F4
:103590002ECE481708F46BCE861708F468CEFA8052
:1035A000E12CD12C243070F41DC0BE01C8010E9452
:1035B000AAC2898198819D0D98838E0D8983FF0C05
:1035C00009F455CEF7FEF6CFF0CF4D8150E0440F11
:1035D000551F70E060E08E819F810E943EEB81E08C
:1035E00006CEFA8030E0F901EE58FE4FD080225925
:1035F0003E4FF901E080E6CF58E0580F382F23CE38
:1036000020914803022E000C330B8217130641F061
:103610008093480360E17EE08AE495E10C9462C601
:103620000895EF92FF920F931F93CF93DF93EC01D6
:103630008B017A018A859B858617970731F08881EF
:1036400099810E9462C61B870A87B7018881998188
:103650000E9402BD2E813F81820F932F911D9F8377
:103660008E8390E080E0DF91CF911F910F91FF90CA
:10367000EF9008959F92AF92BF92CF92DF92EF9218
:10368000FF920F931F93CF93DF93EC018B01942E46
:10369000A52E8A859B858617970731F088819981A9
:1036A0000E9462C61B870A8788859985019649F51D
:1036B000BC800A818E81080FC880D980D6015596BA
:1036C000ED91FC91C6010995B80EE92CFA2C10E099
:1036D000F70121917F01211127C08E819F81810FE8
:1036E000911D9F838E8390E080E0DF91CF911F91A9
:1036F0000F91FF90EF90DF90CF90BF90AF909F9091
:1037000008950E811F81692D7A2D888199810E94EB
:1037100002BD800F912F911D288539852817390703
:1037200038F681E090E0E1CF4B2D602FC6010E947A
:10373000BAC6080F180FCCCFDF92EF92FF920F930B
:103740001F93CF93DF93EC01D62E1CAD0BAD7C0104
:1037500084E0E80EF11CE98DFA8DC7010995412F2F
:10376000480F2D2D602FC7010E94BAC69BAD890F4F
:103770008BAF81E090E0DF91CF911F910F91FF908F
:10378000EF90DF900895CF92DF92EF92FF920F9328
:103790001F93CF93DF93CDB7DEB72C970FB6F89476
:1037A000DEBF0FBECDBFF0908115E0908215209155
:1037B0004A0321111DC04AE75BE06E2D8F2D0E9448
:1037C00026C790E080E0F80EF0928115E092821515
:1037D00099272C960FB6F894DEBF0FBECDBFDF91B0
:1037E000CF911F910F91FF90EF90DF90CF900895B0
:1037F000C0904E15D0904F152AE435E13A832983C5
:103800002F2D30E03C832B832E2D30E03E832D8303
:1038100018861F827A8769871C861B860AE31BE14C
:103820009E012F5F3F4F45E856E1BC01C6010E9453
:1038300073B6B6018AE495E10E9462C68F819885CD
:10384000C2CFEF92FF920F931F93CF937C01009111
:10385000430310914403C0E0F701EC0FF11D6081B8
:10386000662351F0062E000C770BC8010E9463EB13
:10387000892B49F4CF5FF0CF80E0CF911F910F915A
:10388000FF90EF90089581E0F8CF682F880F770BB5
:1038900080914303909144030E9463EBFC0181E01B
:1038A000309709F480E0309781F0918120ED290F65
:1038B0002A3030F09E3251F4928190539A3098F42D
:1038C0003196F0933503E093340308959D3211F05F
:1038D0009B3249F4928120ED290F2A3088F39E32E1
:1038E00011F49381EACFF0E0E0E0EBCF8091340374
:1038F00090913503009731F04AE050E070E060E0CD
:103900000C943EE060E070E0CB01089580913403B8
:1039100090913503009731F04AE050E070E060E0AC
:103920000C9410DF60E070E0CB0108950E94861CCB
:10393000CB0108950F931F93CF93809134039091FF
:1039400035030097E9F0FC018F01C1912C2F2F7DE9
:1039500081F0C53411F0C536B9F7F801108270E076
:1039600060E00E94B2DDF801C083CF911F910F91FA
:10397000089570E060E0CF911F910F910C94B2DD3B
:1039800060E070E0CB01F1CFCF93DF93CDB7DEB72E
:1039900020E24F8158856E818D810E9489BCDF9124
:1039A000CF9108958F929F92AF92BF92EF92FF9224
:1039B0000F931F93CF93DF93EC018B01E42EF22E34
:1039C00080914415909145158C179D0709F43EC0D0
:1039D0002091CA0327FD1092CA032AE9C23BD207ED
:1039E00009F03FC08452944371F40E94A2C16E5109
:1039F0007B4F8F4F9F4F6093CC037093CD03809389
:103A0000CE039093CF03D0934515C093441530E077
:103A100020E00093CE051093CF052093D00530937E
:103A2000D105E092C705F092C805C452D44321F4F1
:103A30001092C6051092CB0382E08093530181E07F
:103A40008093DE051092D4031092C505DF91CF91CB
:103A50001F910F91FF90EF90BF90AF909F908F902C
:103A6000089524E3C432D20771F6825B9A4919F0B3
:103A7000C4E2D4E3C8CF0E94A2C18090CC0390904E
:103A8000CD03A090CE03B090CF03681979098A09BD
:103A90009B0997FFEDCF809194058770873041F7A0
:103AA000C0E9D6E6B0CF80911E1590911F15891BF5
:103AB0008F7051F480910006813031F08091C616EC
:103AC00082FB882780F9089581E00895E091CB0377
:103AD000E63010F581E08E0F8093CB034091CE0548
:103AE0005091CF056091D0057091D1059091C70597
:103AF0008091C80528E0E29FF0011124E656FC4FB2
:103B0000209144153091451531832083428353839E
:103B10006483758396838783089520E040E070E096
:103B200060E084E294E30C94D21CCF930E943C8F1B
:103B30000E948974C82F882319F080E00E94A4A0F5
:103B40008C2F0E948517CF910C948D1DE091CB0393
:103B5000EE2389F0E150E093CB0388E0E89FF00189
:103B60001124E656FC4F6281738127814681808152
:103B700091810C94D21C0C948D1D8091D2038111E3
:103B800006C01092C6050E94A61D0E94791780915A
:103B90005301882331F041E064EF7DE081E00E9431
:103BA0002CBC82E08093530108954F925F926F92F4
:103BB0007F928F929F92AF92BF92CF92DF92EF92BD
:103BC000FF920F931F93CF93DF930E94531D782E84
:103BD0000E94B5BDC091C70515E0711001C016E087
:103BE0006C2E85E0582E5C0E05E00C1B84E0F82E50
:103BF000FC1A83E0E82EEC1A82E0982E9C1A91E9D8
:103C0000A92E9DE0B92E25EDC22E2DE0D22E81E009
:103C1000882E8C1A4C2E4194C11132C08091C90556
:103C2000882389F080915301882309F447C081E0FB
:103C30009091C905911180E024E046EE5DE0642D8D
:103C40000E9489BC3BC08091C4051092C4058823A2
:103C500049F30E94A61D8091DE05882319F3DF91A8
:103C6000CF911F910F91FF90EF90DF90CF90BF9079
:103C7000AF909F908F907F906F905F904F9008953E
:103C8000C13009F05BC08091C905813009F443C09F
:103C900080915301882391F01F92DF92CF928F92EF
:103CA00081E09091C905913009F080E08F930E94E6
:103CB000C41C0F900F900F900F900F90711079C04F
:103CC000C53009F076C08091C905853009F49EC0E1
:103CD000809153018111ABC0D6E081E08D0F8C1330
:103CE00013C09091C9059C1709F4CCC08091530171
:103CF000882351F06C2F661981E09C1380E023E04B
:103D000046E95DE00E9489BCCF5FC51185CFDE5FCB
:103D1000D093C805A4CF8091C4051092C405882310
:103D200009F4B6CFB092A205A092A1050E948D1D04
:103D30008091DE05882309F4ABCF91CFC23009F022
:103D4000C2C08091C905823081F0809153018823DF
:103D500009F4B4CF81E09091C905923009F080E078
:103D600023E04CEC5DE0692D6BCF8091C40510928F
:103D7000C405882351F38EE696E20E941B9580913C
:103D8000DE05882311F36BCF8091C9058330F1F0F4
:103D900080915301882309F491CF81E09091C90566
:103DA000933009F080E023E04FEB5DE06E2D0E9440
:103DB00089BC1C1309C08091C905811709F444C04E
:103DC00080915301811151C0D12F87CF8091C405BB
:103DD0001092C4058823E1F28EE398E20E941B95BD
:103DE0008091DE058823A1F23ACF8091C40510921C
:103DF000C405882309F472C087E39BE20E941B95E7
:103E00008091DE05882309F469C029CF8091C4051B
:103E10001092C405882309F45BCF85E19DE20E94DE
:103E20001B958091DE05882309F452CF18CF81E0DD
:103E30009091C905953009F080E023E041EB5DE009
:103E4000602F0E9489BC48CF8091C4051092C405A0
:103E5000882309F4B5CF84E49EE20E941B958091EB
:103E6000DE05882309F4ACCFFACE6C2F661981E009
:103E70009091C9059C1380E023E048EA5DE00E9430
:103E800089BCA2CF8091C4051092C405882309F48F
:103E90002DCF0E94661D20E040E070E060E081E5EB
:103EA00098E1DF91CF911F910F91FF90EF90DF90FC
:103EB000CF90BF90AF909F908F907F906F905F90CA
:103EC0004F900C94D21CC33009F45ECFC43009F07B
:103ED000F5CE8091C905843009F487CF80915301D4
:103EE000882309F4EBCE81E09091C905943009F064
:103EF00080E023E04AEB5DE06F2D59CFCF93DF9355
:103F0000CDB7DEB78D8190919612891768F08093B6
:103F100096129E01285F3F4F4E815F816AE270E0FA
:103F20008BE692E10E94E3E1DF91CF9108950F9338
:103F30001F93CF93DF938C016F3F19F41092961269
:103F400060E020919612862F062E000C990B281700
:103F5000190609F0F4F460939612C8010E9469E111
:103F6000800F911FEC01C01BD10BCB32D1053CF06F
:103F70000197FC012491207C2038D1F3F3CFDD2779
:103F8000AE01B8018BE692E10E948AE1C559DD4E8F
:103F90001882DF91CF911F910F910895CF93809157
:103FA0009203811109C084E99CE09093D10380932E
:103FB000D00381E0809392030E94661D20E040E0E0
:103FC00070E060E08CE697E10E94D21CC1E0C093F3
:103FD000C6050E94BE771092C6050E94A61DC0931A
:103FE000C60560E085E497E20E94971F80E99CE0A7
:103FF0009093A2058093A105CF910895109291030B
:10400000109252018091C61680648093C6168BE789
:104010009CE00E94A0B560E082E89CE00E94971FAF
:104020000C948D1D0F931F930E94A2C100918D03CC
:1040300010918E0320918F0330919003601B710BC0
:10404000820B930B97FD0CC089B183FB882780F905
:1040500091E089274A9B8260309B846080938C0327
:1040600080918C03817090918C0391FD826090917E
:104070008B03981749F0813009F148F0823079F0CC
:10408000833091F080938B031F910F9108959130AD
:1040900079F09230B9F790918A0391500CC099232E
:1040A00039F09330C1F3EECF9130A9F3923051F74C
:1040B00090918A039F5F90938A03E4CF992359F3E9
:1040C000933001F7F5CFCF92DF92EF92FF92CF932B
:1040D000C82F0E94A2C16B017C0124EA30E74DE7A2
:1040E0005FE360911B0170911C0180911D01909113
:1040F0001E010E941CE287FD18C08AEF90E0A0E03C
:10410000B0E08C0D9D1DAE1DBF1D80937A03909372
:104110007B03A0937C03B0937D03C0931901CF91DF
:10412000FF90EF90DF90CF90089580E090E0DC0169
:10413000E8CFCF9380914B03811154C01092811529
:10414000109282151092831510924F1510924E15F1
:1041500010925115109250151092531581E08093D2
:10416000521582E2809354151092591510925815E9
:10417000EDE6F5E12BE735E18FEF81932E173F0751
:10418000E1F7C1E0C0936A152EE237EA309360157B
:1041900020935F15C09361151092621510926315FC
:1041A00090E490936415109265152CEF36EA3093E5
:1041B0007C1520937B1521E131E030934D15209340
:1041C0004C159EE19093711591E1909372159CE1CD
:1041D00090936F1580936E1580936D150E94EBC2BE
:1041E000C0934B0381E080934A0388EC9BE090935B
:1041F00098148093971410929A14109299145398CB
:104200005B9A52985A9A3898409A0E9412201092BB
:104210008A03CF910895FC01A081B1811C92A281F3
:10422000B3818C918F5F8C930280F381E02D90811C
:104230008CE0989F800D1124E6E4F5E113AE84AF85
:104240000895FC0180E09491992331F0907C90389E
:1042500009F08F5F3196F7CF0895AF92BF92CF925A
:10426000DF92EF92FF920F931F93CF93DF93EC01B6
:104270005B018A01FB01099587FD16C0C82ED12C70
:10428000F12CE12C2196F801C082D182E282F382E6
:10429000CE01DF91CF911F910F91FF90EF90DF90B2
:1042A000CF90BF90AF900895982F907E903CA9F446
:1042B0008F7190E0B0E0A0E06C017D0156E0CC0C85
:1042C000DD1CEE1CFF1C5A95D1F7CE010196F501BD
:1042D00009958F73C82A2296D6CF982F907F903E4B
:1042E00011F58F7090E0B0E0A0E06C017D0136E048
:1042F000CC0CDD1CEE1CFF1C3A95D1F7CE010196CB
:10430000F50109958F73C82A46E0CC0CDD1CEE1C24
:10431000FF1C4A95D1F7CE010296F50109958F73DE
:10432000C82A2396B0CF982F987F903F79F5877051
:1043300090E0B0E0A0E06C017D0186E0CC0CDD1CDB
:10434000EE1CFF1C8A95D1F7CE010196F501099567
:104350008F73C82A96E0CC0CDD1CEE1CFF1C9A95CE
:10436000D1F7CE010296F50109958F73C82A26E090
:10437000CC0CDD1CEE1CFF1C2A95D1F7CE01039658
:10438000F50109958F73C82A24967DCF982F907CCC
:10439000903841F4807C803869F42196CE01F50193
:1043A0000995F8CF8E7F8D3F28F02196CE01F5013B
:1043B0000995F8CFC12CD12C760165CF9CE0899F5F
:1043C000802D112491E0980F909349032CE0280F41
:1043D0002093E40530E02E5F3F4F40917E15421759
:1043E000130619F014F080E00895209180159217BB
:1043F000D0F7662341F08E5F0E940CC48091E405E3
:104400008E5F0E940CC48091E40590917E158917FF
:1044100050F32091801590914903291720F31092B1
:1044200081158093821581E00895CF92DF92EF92FB
:10443000FF920F931F93CF93DF93CDB7DEB72C97E7
:104440000FB6F894DEBF0FBECDBF6F3F710581057B
:10445000910509F0D0F486E495E10E949C1BE0915F
:104460004E15F0914F153196849190E02C960FB631
:10447000F894DEBF0FBECDBFDF91CF911F910F919A
:10448000FF90EF90DF90CF900895F0908115E0902D
:10449000821520914A0321110FC04AE95BE06E2D7D
:1044A0008F2D0E9426C790E080E0F80EF0928115D3
:1044B000E09282159927DACFC0904E15D0904F1513
:1044C0002AE435E13A8329832F2D30E03C832B8386
:1044D0002E2D30E03E832D8318861F822FEF3FEF75
:1044E0003A8729871C861B860AE31BE19E012F5F02
:1044F0003F4FAB01BC01C6010E94AFB5B6018AE4D3
:1045000095E10E9462C68F819885CFCFAF92BF920E
:10451000CF92DF92EF92FF920F931F93CF93DF938F
:1045200000D000D0CDB7DEB77C01062F6A01122F74
:1045300086E0A82EB12C11160CF040C0AE014F5FE2
:104540005F4F65E876E1C7010E942D217C016981FA
:104550007A818B819C81611571058105910571F1CD
:104560006D3371058105910509F450C06E377105F1
:104570008105910509F44AC06A32710581059105EA
:1045800069F507FF12C08EEB9BE00E3F11F08AEB3E
:104590009BE026E01202B00111240E94C31B66E0DA
:1045A00070E00E94CEE8161B61C065E470E080E018
:1045B00090E00E941522115059F510E0812F0F90C4
:1045C0000F900F900F90DF91CF911F910F91FF905F
:1045D000EF90DF90CF90BF90AF9008956432710557
:1045E0008105910579F4C114D10461F026E012022D
:1045F000B0011124C6010E94C31BB5010E94CEE880
:10460000161B99CF0E941522115095CF07FDBBCFE5
:1046100061E089819A81AB81BC81CD97A105B1050B
:1046200009F460E0600F6A30ACF01150862F6AE048
:104630000E94ACE8092F682F880F770B605D7F4FD1
:10464000072E000C880B990B0E941522112309F4E8
:10465000B4CF602F062E000C770B605D7F4F072EC6
:10466000000C880B990B0E9415221150112309F49C
:10467000A4CF86E01802B0011124C7010E94C31B19
:1046800066E070E00E94CEE8161B98CF6FEF7FEFD8
:104690000C94C31BCF92DF92EF92FF920F931F9364
:1046A000CF93DF93CDB7DEB72C970FB6F894DEBF6C
:1046B0000FBECDBFF0908115E090821520914A0386
:1046C00021111DC04AE55BE06E2D8F2D0E9426C78B
:1046D00090E080E0F80EF0928115E0928215992723
:1046E0002C960FB6F894DEBF0FBECDBFDF91CF91F1
:1046F0001F910F91FF90EF90DF90CF900895C090A1
:104700004E15D0904F152AE435E13A8329832F2D99
:1047100030E03C832B832E2D30E03E832D831886A2
:104720001F827A8769871C861B860AE31BE19E012C
:104730002F5F3F4F48E856E1BC01C6010E9473B6A7
:10474000B6018AE495E10E9462C68F819885C2CF46
:104750006FEF7FEF0C944A23AF92BF92CF92DF921C
:10476000EF92FF920F931F93CF93DF935C016B0146
:104770000E942121E82EC6010E948B16F12C03E134
:1047800010E0081B1109C5E20E151F050CF4CFE15E
:104790008C2F90E09C012E5F3F4F40917E15421779
:1047A000130609F0CCF509972091801528171906F2
:1047B0009CF14091E6055091E7056091E505109266
:1047C0008115C093821525E1C5010E948622D1E0A2
:1047D000C114D104B1F06AE370E080E090E00E947F
:1047E00015220E151F05D4F4C45F80917E15C817DD
:1047F00040F0209180154C2F4950550B2417150679
:104800007CF4DF91CF911F910F91FF90EF90DF909B
:10481000CF90BF90AF900895D0E0DACFDD2389F339
:10482000802F880F080F000F00938115C093821509
:1048300060E270E080E090E00E941522C601DF9106
:10484000CF911F910F91FF90EF90DF90CF90BF908D
:10485000AF900C94A823CF92DF92EF92FF92CF9368
:10486000DF9300D000D0CDB7DEB78091C4051092A1
:10487000C405882331F18091D3038F5F8093D303E4
:104880008931E0F081E08093D20320E040E070E0E5
:1048900060E08DEB9DE10E94D21C8AE09EE0909347
:1048A000A2058093A1050F900F900F900F90DF91BC
:1048B000CF91FF90EF90DF90CF9008950E9476A067
:1048C000F2CF6091CE057091CF058091D005909187
:1048D000D105611571058105910509F43EC00E945D
:1048E00023E22DEC3CEC4CEC5CE30E9482E2209154
:1048F0004C0B30914D0B40914E0B50914F0B0E9441
:1049000013E96B017C0120E030E040E850EC0E94AC
:104910001CE287FD53C020E030E040E850E4C701CE
:10492000B6010E9496EA18160CF44FC0C0924C0BC8
:10493000D0924D0BE0924E0BF0924F0B8EE891E02F
:104940000E94818582E0809353011092CE051092DF
:10495000CF051092D0051092D10580915301882384
:1049600009F4A1CFC0904C0BD0904D0BE0904E0BB2
:10497000F0904F0B20E030E0A901C701B6010E9482
:104980001CE227E137EB41ED58E387FF04C027E144
:1049900037EB41ED58EBC701B6010E9413E969837B
:1049A0007A838B839C836BE2CE0101960E94639194
:1049B000BC0183E09EE00E94AC2375CFC12CD12CBA
:1049C00090E8E92E90ECF92EB1CFC12CD12C80E8E3
:1049D000E82E80E4F82EAACF0F931F93CF93DF9396
:1049E000FC01EB018091CE059091CF05A091D005FF
:1049F000B091D105B7FF08C01092CE051092CF0537
:104A00001092D0051092D1058091D2059091D305D6
:104A1000A091D405B091D5054091CE055091CF0518
:104A20006091D0057091D10584179507A607B70747
:104A300044F48093CE059093CF05A093D005B09316
:104A4000D105809153018823E1F06091CE057091EA
:104A5000CF058091D0059091D1050091D605109198
:104A6000D7052091D8053091D905600F711F821F9D
:104A7000931F0995BC018091DC059091DD050E9492
:104A8000AC238091C405811108C08091CB05882397
:104A9000D1F1809153018823B1F18091DA05909191
:104AA000DB050097B1F04091CE055091CF056091A4
:104AB000D0057091D1050091D6051091D7052091B0
:104AC000D8053091D905400F511F621F731FFE0199
:104AD0000995E091CC05F091CD05309741F080919A
:104AE000CB05811103C08091C40581110995809186
:104AF000C4051092C405882331F0DF91CF911F9136
:104B00000F910C94A61DDF91CF911F910F910895E5
:104B100062EC75E18BED95E10C94EC246AEE75E1A5
:104B200083E096E10C94EC2465E276E189E398E178
:104B30000C94EC2468E376E187EA97E10C94EC248A
:104B400063E576E189EE97E10C94EC2462E176E18D
:104B500088EF97E10C94EC246CE676E182E498E12E
:104B60000C94EC248F929F92AF92BF92CF92DF92DF
:104B7000EF92FF920F931F93CF93DF93CDB7DEB7E2
:104B80002C970FB6F894DEBF0FBECDBF982F862F9F
:104B90005A017901D02E692F0E94DE21882309F461
:104BA00087C010914A03C701002381F10E9421218F
:104BB000C82E80904E1590904F15111143C01FEFD5
:104BC00023E12C194091E6055091E7056091E50538
:104BD000C5010E948622CC2009F46AC0B6E08B9FF2
:104BE000500111246AE370E080E090E00E941522F9
:104BF00057E0A516B10408F442C060E270E080E01E
:104C000090E00E941522A81AB90AF2CF0E948B16D2
:104C1000C82E80904E1590904F15112381F2FE0101
:104C200033968AE0DF011D928A95E9F78AE495E1DF
:104C30009A83898301E11BE19E012F5F3F4F48E882
:104C400056E112C0FE0133968AE0DF011D928A957B
:104C5000E9F78AE495E19A83898301E11BE19E01EA
:104C60002F5F3F4F45E856E1B701C4010E9473B67C
:104C7000B4018AE495E10E9462C61F81A1CF4091F0
:104C8000E405212F30E0A6E0CA9EC00111242E5F6A
:104C90003F4F281739070CF49C0180E8821B809352
:104CA000811540938215C701DD20A9F00E9446239B
:104CB0002C960FB6F894DEBF0FBECDBFDF91CF911B
:104CC0001F910F91FF90EF90DF90CF90BF90AF902A
:104CD0009F908F9008950E94A823EACF7F928F9291
:104CE0009F92AF92BF92CF92DF92EF92FF920F937B
:104CF0001F93CF93DF930E94B5BDC091C70565E0B8
:104D0000862E8C0ED6E0DC1B85E0D82EDC1A84E0E3
:104D1000C82ECC1A83E0B82EBC1A82E0A82EAC1A9A
:104D200081E0982E9C1A7C2E7194C11134C0809120
:104D3000C9058823B1F080915301882359F081E09F
:104D40009091C905911180E024E041E75DE0672D75
:104D50000E9489BCCF5FC811E8CF87E08093C80567
:104D60000CC08091C4051092C405882321F30E94D1
:104D7000A61D8091DE058823F1F2DF91CF911F916E
:104D80000F91FF90EF90DF90CF90BF90AF909F90EA
:104D90008F907F900895C130E9F58091C9058130E9
:104DA000E9F0809153018823A9F211E08091C905AF
:104DB000813009F010E06091200B7091210B8091FF
:104DC000220B9091230B0E94B61700E09C0149EE44
:104DD0005CE0692D812F0E94B225BCCF8091C40573
:104DE0001092C4058823E9F20E9436BDE12C1CE331
:104DF000F12E0CE116E420E030E040E85FE360E2F1
:104E00007BE089EE9CE00E940BBE8091DE0588234A
:104E100041F2B3CFC23009F006C18091C90582309A
:104E2000D9F080915301882309F494CF11E0809147
:104E3000C905823009F010E06091240B7091250BB8
:104E40008091260B9091270B0E94B61700E09C01E1
:104E500042EE5CE06A2DBECF8091C4051092C4057D
:104E60008823F9F20E9436BDE12C1CE3F12E0CE1FF
:104E700016E420E030E040E85FE364E27BE082EEAD
:104E80009CE00E940BBE8091DE05882351F275CF15
:104E90008091C9058330D9F080915301882309F4AA
:104EA00059CF11E08091C905833009F010E060917D
:104EB000280B7091290B80912A0B90912B0B0E944B
:104EC000B61700E09C014BED5CE06B2D83CF809129
:104ED000C4051092C4058823F9F20E9436BDE12C66
:104EE0001CE3F12E0CE116E420E030E040E85FE343
:104EF00068E27BE08BED9CE00E940BBE8091DE05BA
:104F0000882351F23ACF8091C9058430D9F080913D
:104F10005301882309F41ECF11E08091C905843024
:104F200009F010E060912C0B70912D0B80912E0BED
:104F300090912F0B0E94B61700E09C0144ED5CE0BD
:104F40006C2D48CF8091C4051092C4058823F9F2D6
:104F50000E9436BDE12C1CE3F12E0CE116E420E0AA
:104F600030E040E85FE36CE27BE084ED9CE00E948F
:104F70000BBE8091DE05882351F2FFCE8091C905DA
:104F80008530D9F080915301882309F4E3CE11E0F4
:104F90008091C905853009F010E060913C0B70915B
:104FA0003D0B80913E0B90913F0B0E94B61700E0A5
:104FB0009C014FEC5CE06D2D0DCF8091C4051092EB
:104FC000C4058823F9F20E9436BDE12C1CE3F12EC2
:104FD0000CE116E420E030E0A9016CE37BE08FEC0B
:104FE0009CE00E940BBE8091DE05882359F2C5CE5D
:104FF0008091C4051092C405882329F10E9436BD12
:10500000E12C1CE3F12E0CE116E420E030E0A901D4
:1050100060E47BE085EC9CE00E940BBE8091DE05A5
:10502000882389F0AACEC33009F432CFC43009F402
:105030006ACFC53009F4A2CFC63009F08BCE80917B
:10504000C9058630A9F280915301882309F482CEE4
:1050500011E08091C905863009F010E06091400BA5
:105060007091410B8091420B9091430B0E94B617B7
:1050700000E09C0145EC5CE06D2FACCE2F923F929E
:105080004F925F926F927F928F929F92AF92BF9258
:10509000CF92DF92EF92FF920F931F93CF93DF9304
:1050A000CDB7DEB72C970FB6F894DEBF0FBECDBFDD
:1050B000C090000BD090010BE090020BF090030B1E
:1050C0008091040B9091050BA091060BB091070BFA
:1050D0008C159D05AE05BF0510F4D701C601C09023
:1050E000FC0AD090FD0AE090FE0AF090FF0ABC0195
:1050F000CD016C157D058E059F0510F4C701B60125
:105100000E9421E22B013C010E94B5BD2091C70500
:105110002B872E83822F8B5F8D8387E0922F821BBC
:105120008F8386E0821B888785E0821B898784E0E5
:10513000821B8A8783E0282E221A82E0382E321AB8
:1051400091959C872B85211142C08091C9058823A8
:10515000C9F080915301882359F081E09091C905ED
:10516000911180E024E041E75DE06C850E9489BCFC
:105170008B858F5F8B879D819813E4CF88E0809328
:10518000C8050CC08091C4051092C405882309F39A
:105190000E94A61D8091DE058823D9F22C960FB6B9
:1051A000F894DEBF0FBECDBFDF91CF911F910F915D
:1051B000FF90EF90DF90CF90BF90AF909F908F9037
:1051C0007F906F905F904F903F902F9008958B85C8
:1051D000813009F089C08091C9058130F9F0809152
:1051E0005301882329F211E08091C905813009F02B
:1051F00010E06091300B7091310B8091320B9091E7
:10520000330B0E94B61761E02E81621B00E09C0107
:105210004FE15DE0812F0E94B225AACF8091C405A5
:105220001092C4058823D9F20E9436BD2AE037EDDA
:1052300043E25DE3C301B2010E9482E220E030E07C
:10524000A9010E9413E94B015C0120E030E040E03D
:105250005FE40E941CE287FD05C0812C912CA12CEB
:105260003FE4B32E2AE037ED43E25DE36091300B7B
:105270007091310B8091320B9091330B0E9482E23E
:1052800020E030E0A9010E9413E920E030E040E88E
:105290005FE30E9412E90E940FEA69837A838B839D
:1052A0009C83C501B4010E9408EA7B018C0121E0C6
:1052B000E21AF10801091109912C812C20EAA22E91
:1052C00025E2B22EC980DA8021E030E040E050E0F3
:1052D00060E37BE08FE19DE00E9442BD8091DE05AE
:1052E000882309F47CCF5ACF8B85823009F08EC198
:1052F0008091C9058230D9F080915301882309F447
:1053000037CF11E08091C905823009F010E060913B
:10531000340B7091350B8091360B9091370B0E94B6
:10532000B61700E09C0145E15DE0632D73CF8091ED
:10533000C4051092C4058823F9F20E9436BD60911D
:10534000080B7091090B80910A0B90910B0B0E9436
:1053500021E27B018C0120E030E048EC52E464E380
:105360007BE085E19DE00E940BBE8091DE058823F5
:1053700019F214CF8091C9058330D9F0809153017F
:10538000882309F4F5CE11E08091C905833009F036
:1053900010E06091380B7091390B80913A0B90912D
:1053A0003B0B0E94B61700E09C014CE05DE0622DD3
:1053B00031CF8091C4051092C4058823F9F20E9470
:1053C00036BD2AE037ED43E25DE3C301B2010E943E
:1053D00082E220E030E0A9010E9413E94B015C0168
:1053E00020E030E040E05FE40E941CE287FD05C061
:1053F000812C912CA12C9FE4B92E2AE037ED43E2B9
:105400005DE36091380B7091390B80913A0B90916C
:105410003B0B0E9482E220E030E0A9010E9413E9E8
:1054200020E030E040E85FE30E9412E90E940FEACA
:1054300069837A838B839C83C501B4010E9408EA47
:105440007B018C0121E0E21AF10801091109912C7C
:10545000812C80EAA82E85E2B82EC980DA8021E06E
:1054600030E040E050E068E37BE08CE09DE00E94AB
:1054700042BD8091DE05882309F480CF8FCE8091D4
:10548000C9058430E9F080915301882309F470CE76
:1054900011E08091C905843009F010E06091FC0AA8
:1054A0007091FD0A8091FE0A9091FF0A0E9421E20C
:1054B0000E948E1700E09C0145E05DE06A85AACE5F
:1054C0008091C4051092C4058823E9F20E9436BD7C
:1054D00000E818E124E630E040E050E06CEF7AE0CC
:1054E00085E09DE00E94A8BE8091DE05882359F2E8
:1054F00055CE8091C9058530E9F08091530188230C
:1055000009F436CE11E08091C905853009F010E02C
:105510006091000B7091010B8091020B9091030B35
:105520000E9421E20E948E1700E09C014EEF5CE099
:10553000698570CE8091C4051092C4058823E9F274
:105540000E9436BD0EE718E124E630E040E050E06E
:1055500060E07BE08EEF9CE00E94A8BE8091DE05BB
:10556000882359F21BCE8091C9058630E9F08091DD
:105570005301882309F4FCCD11E08091C9058630E0
:1055800009F010E06091040B7091050B8091060BFF
:105590009091070B0E9421E20E948E1700E09C016F
:1055A00047EF5CE0688536CE8091C4051092C40553
:1055B0008823E9F20E9436BD0CE718E12AE030E0CA
:1055C00040E050E064E07BE087EF9CE00E94A8BEF2
:1055D0008091DE05882359F2E1CD8091C4051092B7
:1055E000C405882339F10E9436BD0AE718E124E694
:1055F00030E040E050E068E07BE080EF9CE00E941B
:10560000A8BE8091DE058823A9F0C8CD2B85233064
:1056100009F4B0CE243009F432CF253009F469CF33
:10562000263009F4A0CF273009F0A2CD8091C9051A
:10563000873099F280915301882309F499CD11E0C4
:105640008091C905873009F010E06091080B7091D6
:10565000090B80910A0B90910B0B0E9421E20E9492
:105660008E1700E09C0140EF5CE06F81D3CD3F924C
:105670004F925F926F927F928F929F92AF92BF9262
:10568000CF92DF92EF92FF920F931F93CF93DF930E
:105690000E94B5BDC091C705A5E04A2E4C0ED4E0CE
:1056A000DC1B83E0782E7C1A82E0682E6C1A81E085
:1056B000582E5C1A3C2E3194C11138C08091C90516
:1056C0008823B1F080915301882359F081E09091B3
:1056D000C905911180E024E041E75DE0632D0E945F
:1056E00089BCCF5FC411E8CF85E08093C8050CC0AA
:1056F0008091C4051092C405882321F30E94A61D41
:105700008091DE058823F1F2DF91CF911F910F91F7
:10571000FF90EF90DF90CF90BF90AF909F908F90D1
:105720007F906F905F904F903F900895C13009F047
:105730005BC08091C9058130E9F0809153018823D5
:1057400081F211E08091C905813009F010E060918B
:105750000F067091100680911106909112060E941A
:10576000011800E09C014DE35DE0652D812F0E9452
:10577000B225B7CF8091C4051092C4058823E9F201
:105780000E9436BD20E030E0A90160910F067091C3
:10579000100680911106909112060E9413E920E0F4
:1057A00030E040E85FE30E9412E90E940FEA912C8A
:1057B000812CE4E9AE2EE5E2BE2E6B011DEDE12E5B
:1057C00013E0F12E00E010E021E030E040E050E096
:1057D0006FE076E08DE39DE00E9442BD8091DE05A2
:1057E000882309F4AACF90CFC23009F0F8C0809185
:1057F000C9058230D9F080915301882309F471CF13
:1058000011E08091C905823009F010E06091130623
:105810007091140680911506909116060E94011849
:1058200000E09C0145E35DE0662DA0CF8091C405BA
:105830001092C4058823F9F20E9436BD20E030E0C2
:10584000A90160911306709114068091150690913C
:1058500016060E9413E920E030E040E85FE30E9472
:1058600012E90E940FEA912C812C44E9A42E45E212
:10587000B42E6B011DEDE12E13E0F12E00E010E0DF
:1058800021E030E040E050E063E176E085E39DE038
:105890000E9442BD8091DE05882309F4ACCF34CF4D
:1058A0008091C9058330D9F080915301882309F490
:1058B00018CF11E08091C905833009F010E06091A4
:1058C0001706709118068091190690911A060E9489
:1058D000441400E09C014DE25DE0672D47CF8091CC
:1058E000C4051092C4058823F9F20E9436BD20E059
:1058F00030E048EC52E460911706709118068091F0
:10590000190690911A060E9482E220E030E0A90177
:105910000E9413E920E030E040E251E40E9412E9E5
:105920000E940FEA912C812C2EE8A22E25E2B22EA5
:105930006B011EEAE12E12E8F12E01E010E02AE0F0
:1059400030E040E050E067E176E08DE29DE00E94CB
:1059500042BD8091DE05882309F4A6CFD5CE809183
:10596000C4051092C405882309F444C00E9436BDC2
:1059700020E030E048EC52E460911B0670911C0678
:1059800080911D0690911E060E9482E220E030E088
:10599000A9010E9413E920E030E040E251E40E94B6
:1059A00012E90E940FEA912C812C8EE8A82E85E244
:1059B000B82E6B011EEAE12E12E8F12E01E010E094
:1059C0002AE030E040E050E06BE176E085E29DE0E7
:1059D0000E9442BD8091DE05882361F095CEC330E0
:1059E00009F45ECFC43009F07CCE8091C9058430C3
:1059F00009F4B5CF80915301882309F472CE11E0E8
:105A00008091C905843009F010E060911B06709107
:105A10001C0680911D0690911E060E94441400E011
:105A20009C0145E25DE06D2FA1CEBF92CF92DF9247
:105A3000EF92FF920F931F93CF93DF930E94B5BD18
:105A4000C091C70585E0C82ECC0ED4E0DC1B13E066
:105A50001C1B82E0F82EFC1A81E0E82EEC1ABC2E0A
:105A6000B194C11130C08091C9058823B1F08091F3
:105A70005301882359F081E09091C905911180E08C
:105A800024E041E75DE06B2D0E9489BCCF5FCC1123
:105A9000E8CF85E08093C8050CC08091C4051092C2
:105AA000C405882321F30E94A61D8091DE0588236A
:105AB000F1F2DF91CF911F910F91FF90EF90DF9066
:105AC000CF90BF900895C130B9F58091C90581305C
:105AD000F1F0809153018823C9F2DD24D3948091A1
:105AE000C905813009F0D12C6091100B7091110B18
:105AF0008091120B9091130B0E94FA1400E09C010C
:105B000046E65DE06E2D8D2D0E94B225BFCF8091BF
:105B1000C4051092C4058823E1F20E9436BD48E70F
:105B200058E160E17BE086E69DE00E9428BF80911D
:105B3000DE05882371F2BDCFC23009F07FC08091AD
:105B4000C9058230E1F080915301882309F49ECF8A
:105B5000DD24D3948091C905823009F0D12C609165
:105B6000140B7091150B8091160B9091170B0E94DE
:105B7000FA1400E09C014BE55DE06F2DC4CF8091ED
:105B8000C4051092C4058823F1F20E9436BD46E791
:105B900058E164E17BE08BE59DE00E9428BF8091A5
:105BA000DE05882381F285CF8091C9058330E1F03D
:105BB00080915301882309F469CFDD24D394809127
:105BC000C905833009F0D12C6091180B7091190B25
:105BD00080911A0B90911B0B0E94FA1400E09C011B
:105BE00040E55DE0612F8FCF8091C4051092C40520
:105BF0008823F1F20E9436BD44E758E168E17BE07A
:105C000080E59DE00E9428BF8091DE05882381F217
:105C100050CF8091C4051092C4058823C9F00E941A
:105C200036BD42E758E16CE17BE085E49DE00E94EF
:105C300028BF8091DE05882359F03BCFC33009F49B
:105C4000B3CFC43009F022CF8091C905843009F365
:105C500080915301882309F419CFDD24D3948091D6
:105C6000C905843009F0D12C60911C0B70911D0B7B
:105C700080911E0B90911F0B0E94FA1400E09C0172
:105C800045E45DE06D2F3FCF2F923F924F925F92A0
:105C90006F927F928F929F92AF92BF92CF92DF923C
:105CA000EF92FF920F931F93CF93DF930E94B5BDA6
:105CB000C091C70535E0432E4C0E43E0342E57E526
:105CC000652E5FE5752ED1E0DC1B2C2E219482E041
:105CD000582E5C1AC11141C08091C9058823F1F08A
:105CE00080915301882359F081E09091C905911169
:105CF00080E024E041E75DE0622D0E9489BC809154
:105D00000604882309F4C3C0C23009F45CC083E0F0
:105D1000CF5FC411DFCF8093C8050CC08091C4054C
:105D20001092C4058823E1F20E94A61D8091DE0531
:105D30008823B1F2DF91CF911F910F91FF90EF90E7
:105D4000DF90CF90BF90AF909F908F907F906F909B
:105D50005F904F903F902F900895C13081F68091D1
:105D6000C9058130C9F080915301882341F281E057
:105D70009091C905913009F080E09091060428EBDC
:105D80003CE0911102C024EB3CE001E04BEB5CE015
:105D90006D2F0E94B225B3CF809106049091C40567
:105DA0001092C4059923F9F28C278093060430924F
:105DB00053016114710411F00E94575F8091DE0558
:105DC000882389F2B7CF8091C9058230F1F08091A4
:105DD0005301882309F49BCF11E08091C9058230DB
:105DE00009F010E0609102047091030480910404B2
:105DF000909105040E94E79400E09C014AEA5CE06F
:105E0000652D812F0E94B22582CF8091C40510920A
:105E1000C4058823E1F20E9436BD20E030E04AE765
:105E200054E4609102047091030480910404909101
:105E300005040E9482E220E030E0A9010E9413E9FB
:105E400020E030E84BEB54E40E9412E90E940FEA94
:105E500087E5882E8FE5982E9CEAA92E95E2B92E2B
:105E60006B0116EDE12E16E0F12E00E010E02CEDB6
:105E700035E040E050E062E074E08AEA9CE00E9495
:105E800042BD8091DE05882309F4A1CF53CF82E083
:105E90003FCFE6E4F5E183AF64AFCA010C94A823D9
:105EA0000F931F93CF9310924203109241032FE35D
:105EB0002093470310924603109245039C01F90179
:105EC00090812F5F3F4F9032D1F39E34C9F481818E
:105ED00090ED980F9A3020F08D3211F08B3281F4D2
:105EE00032969F012F5F3F4F808180538A3008F4A4
:105EF00068C09F012F5F3F4F8081803209F463C0EB
:105F0000F093F205E093F1058F010F5F1F4FC08101
:105F10006AE270E0C8010E9463EB009731F0FC0177
:105F2000319780818032E1F31182CD3429F0C4357C
:105F300019F0C73409F041C0F80180810F5F1F4F8D
:105F40008032D1F380538A30C0F5C093470330E0EC
:105F500020E06AE0AF014F5F5F4F629FC001639F27
:105F6000900D11249C01205331098081280F311D8F
:105F700087FD3A95FA01808180538A3058F3309337
:105F8000460320934503CA01FC010196408140323B
:105F9000D9F3F0934403E0934303CD3401F52E315C
:105FA000310539F090F42731310519F02C313105E4
:105FB000B1F4F0934203E0934103CF911F910F910D
:105FC0000895F9018ECFF90194CF2537310538F0C6
:105FD0002737310570F3203A83E0380751F350E05A
:105FE00040E0CF0101966081662309F45AC0613216
:105FF00091F4CD3481F42032310569F49093420359
:106000008093410363E270E00E9463EB0097A9F282
:10601000FC011082D2CFFC01DF018D91803271F042
:1060200090ED980F9A3008F18E3251F4918190538F
:106030009A30D8F041155105E1F414C0FD01ECCFC0
:106040008D3211F08B3259F4918160ED690F6A3015
:1060500060F09E3221F4928190539A3030F04115D5
:10606000510519F4AF014150510981548A3108F4A6
:10607000B8CFDF01FD018D91882309F4B2CF90EDF7
:10608000980F9A30B8F393ED980F923098F38B32C3
:1060900089F3CF0101966081603209F0A2CFFC0143
:1060A000F8CF509342034093410387CF0E94861C50
:1060B00097FD0CC00E94861C6F3F710581059105FC
:1060C00009F034F40E94861C862F089580E008951C
:1060D0008FEF08958091340390913503892B41F01F
:1060E0000E94563091E0811101C090E0892F0895FF
:1060F00091E0FCCF0E94451C882341F081E0209173
:10610000340330913503232B09F480E00895CF93B5
:10611000DF93EB010E947A30882319F00E94861CDD
:10612000EB01CE01DF91CF910895CF93DF93C82F7C
:10613000D62F0E947A30882321F0DF91CF910C94E2
:106140006A308C2F0E94451C811101C08D2FDF9178
:10615000CF91089510926B0410926C0410926D040C
:1061600010926E04E7E0F4E084E6DF011D928A9568
:10617000E9F70895909101049817B1F00E94BE7755
:1061800080910104882341F084E49BE00E94F7772A
:10619000109201040C94738681E08093010484E4DE
:1061A0009BE00E94DF77F6CF08959091010481E093
:1061B00089270C94BA30EF92FF920F931F93CF93DD
:1061C000DF9307E014E0C5E07801D5E0F7016191C5
:1061D0007191819191917F0120E030E0A9010E94AD
:1061E0001CE281110EC0D15089F7C1500C5E1F4FC7
:1061F000C111EACFDF91CF911F910F91FF90EF90E6
:10620000089581E0F7CFEFE6F0E08081826080833F
:1062100008954F925F926F927F928F929F92AF926A
:10622000BF92CF92DF92EF92FF920F931F93CF9383
:10623000DF9300D000D0CDB7DEB70E94A2C14B01E2
:106240005C01809119018F3F09F441C00E94A2C1F5
:10625000C0907A03D0907B03E0907C03F0907D03A4
:106260006C197D098E099F0997FD31C080911E151B
:1062700090911F158F5F8F70891749F1E091190177
:1062800080E090E0A8E4B3E4E43050F424E0E29F3E
:10629000F0011124EA58FE4F80819181A281B381DF
:1062A00089839A83AB83BC83C12CD12C76018E0168
:1062B0000F5F1F4F20E53BE04CE45BE068E47BE0D0
:1062C00084E49BE00E9459B98FEF809319010E94EA
:1062D000122080918C0382FF33C080918903811149
:1062E00031C091E090938903809191038927809335
:1062F000C4051092910383E08093530110928C03A4
:106300000E94A2C16C507E4F8F4F9F4F60938D03B0
:1063100070938E0380938F039093900368E873E1EA
:1063200082E090E00E94BA9416E0115059F00E9469
:106330005E9462E070E080E090E00E9407C1F5CFDB
:10634000109289038091850390918603A091870321
:10635000B0918803A5019401281B390B4A0B5B0BF4
:10636000DA01C901B7FF05C08091D403882309F47D
:10637000C6C1D501C4018C599F4FAF4FBF4F809309
:10638000850390938603A0938703B093880360915D
:106390008A03062E000C770B77FF03C07195619579
:1063A000710990918A0380918403981365C06330CA
:1063B00008F062C010928A0380918A03809384035C
:1063C000643008F069C08091C4058111E7C08091F4
:1063D0004415909145158452944341F480911A01DB
:1063E000882309F4EDC0815080931A010E94E57959
:1063F000C0903306D0903406E0903506F090360613
:1064000081110E940331D701C6013AE0B695A795E4
:10641000979587953A95D1F7009741E0A407B10584
:1064200020F08FEF9FEFA0E0B0E096958795209148
:1064300053012111D7C03091D40331118EC1809105
:106440004415909145158452944309F46DC180918F
:10645000C605811169C18091800390918103A0914B
:106460008203B0918303881A990AAA0ABB0AB7FC6F
:1064700069C10E948D1D66C1633009F09DCF809176
:106480008A0387FD07C081E0880F880F80938A0305
:1064900064E092CF8FEFF8CF8091E30521E030E008
:1064A00040E050E0882309F456C0C090DF05D0904A
:1064B000E005E090E105F090E205C114D104E104AB
:1064C000F104E9F170E090E080E00E9421E220E038
:1064D00030E040E85EE30E9482E22B013C01C5010E
:1064E000B4016C197D098E099F090E9421E29B016C
:1064F000AC01C301B2010E9496E920E030E04AE716
:1065000054E40E9482E26B017C0120E030E042E032
:1065100053E40E9496EA24E630E040E050E087FF32
:1065200012C020E030E040EA52E4C701B6010E9408
:1065300096EA2AE030E040E050E087FF04C021E026
:1065400030E040E050E08092DF059092E005A092BC
:10655000E105B092E205A0918A030A2E000CBB0B64
:106560000E940AE924E030E040E050E00E94E2E8C6
:106570008091CE059091CF05A091D005B091D10525
:10658000820F931FA41FB51F8093CE059093CF0554
:10659000A093D005B093D10510928A03D501C40110
:1065A0008856954CAF4FBF4F8093800390938103E3
:1065B000A0938203B093830381E08093530107CFBC
:1065C0008CE080931A0180917E0390917F03009765
:1065D00029F0019790937F0380937E0381E080935D
:1065E000530104CF009741F040917E0350917F0307
:1065F0004817590708F023CF8091D40381111DC09B
:10660000223038F0243008F44CC0243011F41092B9
:10661000530180918315811105C081E0809383151A
:106620000E94EBC280914C1590914D150E94C4C2FE
:1066300081E08093CA058093D40383E00E94001B0D
:1066400081E080936A15E0914415F0914515099514
:106650001092CA058091D403811127C01092C405FD
:1066600080914415909145158452944309F0EFCEE2
:106670000E94A2C1DC01CB0188199909AA09BB09B2
:10668000C0907E03D0907F03F12CE12CC816D90670
:10669000EA06FB0608F0D3CE90937F0380937E0337
:1066A000CECE81E080935301B4CF8AE495E10E947D
:1066B00030C691E0811101C090E09093D40388230B
:1066C00069F2809144159091451584529443B9F430
:1066D0000E94A2C1DC01CB0188199909AA09BB0952
:1066E000C0907E03D0907F03F12CE12CC816D90610
:1066F000EA06FB0620F490937F0380937E030F90BD
:106700000F900F900F90DF91CF911F910F91FF90FD
:10671000EF90DF90CF90BF90AF909F908F907F9041
:106720006F905F904F90089548E9840E4AE3941E5D
:10673000A11CB11C8092800390928103A0928203DD
:10674000B09283038091D4038111D9CF80915301FA
:106750008130A9F610925301D2CF009709F46DCF82
:1067600043CF8091EC059091ED05892B79F48091D0
:10677000EC059091ED05892B49F42091EC053091C1
:10678000ED0581E0232B19F480E0089581E0089560
:10679000CF92DF92EF92FF926B017C0183E3C816E8
:1067A000D104E104F10470F082E3C81AD108E108D1
:1067B000F10862E370E080E090E00E9407C10E946F
:1067C0007586ECCFC701B6010E9407C1FF90EF901C
:1067D000DF90CF900C9475865E9A809194058E7FA1
:1067E000809394055E9A809194058D7F80939405A3
:1067F000159A809194058B7F809394055E9A0895F5
:106800009091C61693FB882780F993FF06C081E01C
:106810009091BB14911101C080E008950E94D7BAF5
:106820000E940034882351F08091C61682FD06C074
:1068300086EA9CE09093A2058093A1058FE99CE0F5
:106840000E94A0B50C94A7904F925F926F927F9296
:106850008F929F92AF92BF92CF92DF92EF92FF9270
:106860000F931F93CF93DF9300D000D01F92CDB72B
:10687000DEB71092E3058091C4051092C405882309
:10688000E9F020E040E070E060E082EB9AE90F90F0
:106890000F900F900F900F90DF91CF911F910F915C
:1068A000FF90EF90DF90CF90BF90AF909F908F9030
:1068B0007F906F905F904F900C94D21C20911F019D
:1068C000309120014091CE055091CF05CA01820F31
:1068D000931F2436310509F015C44730510544F0A3
:1068E00006978A3091050CF01CC48AE090E023C41E
:1068F00006964A3F5F4FACF38091CA05882309F49E
:10690000C0C12091010630910206409103065091CA
:1069100004066091440B7091450B8091460B909159
:10692000470B0E9413E94B015C0120910506309151
:10693000060640910706509108066091480B709139
:10694000490B80914A0B90914B0B0E9413E969838C
:106950007A838B839C832091090630910A064091AB
:106960000B0650910C0660914C0B70914D0B809171
:106970004E0B90914F0B0E9413E92B013C0120E03C
:1069800030E040E251E40E9482E220E030E048EC56
:1069900052E40E9482E26B017C0120E030E0A90118
:1069A000C301B2010E941CE220E030E040EA50EC5A
:1069B00087FD04C020E030E040EA50E4C701B601A2
:1069C0000E9413E920E030E040E251E40E9496E9A1
:1069D0000E9408EA2B013C0180E277FE09C0709416
:1069E000609450944094411C511C611C711C8DE2B8
:1069F0008093D50360E2F0E14F16F7E25F06610491
:106A000071048CF0C301B20120E137E240E050E0B4
:106A10000E94E2E8CA01B9012AE030E040E050E01B
:106A20000E94E2E8605D6093D60360E228EE4216C1
:106A300023E05206610471048CF0C301B20128EE18
:106A400033E040E050E00E94E2E8CA01B9012AE0E8
:106A500030E040E050E00E94E2E8605D6093D703E0
:106A6000C301B20124E630E040E050E00E94E2E8D9
:106A70006AE0C62ED12CE12CF12CCA01B901A70184
:106A800096010E94E2E8605D6093D803C301B20101
:106A9000A70196010E94E2E86D83CA01B901A7012E
:106AA00096010E94E2E8CD80CC2009F454C38EE226
:106AB0008093D903605D6093DA032C2D205D2093D1
:106AC000DB0365ED73E082E793E00E946EEB20E06C
:106AD00030E0A901C501B4010E941CE220E030E0D1
:106AE00040E05FEB87FD04C020E030E040E05FE382
:106AF000C501B4010E9413E90E9408EACB010E947B
:106B0000FF91BC018DE693E00E946EEB20E030E047
:106B1000A90169817A818B819C810E941CE220E01D
:106B200030E040E05FEB87FD04C020E030E040E073
:106B30005FE369817A818B819C810E9413E90E94C5
:106B400008EACB010E94FF91BC0188E693E00E9415
:106B50006EEB4091CA034F774983411127C00E94D1
:106B60000034882319F18091BE169091BF16A09130
:106B7000C016B091C1160097A105B105B9F0BC01CE
:106B8000CD016D597F4F8F4F9F4F24E630E040E09D
:106B900050E00E9464E86091C2167091C316809123
:106BA000C4169091C5160E9464E829830E945A90E9
:106BB000B62E872E982EA92E6D8380911801C9803C
:106BC0008C15C1F0C092180128E4C29EB0011124B6
:106BD00090E080E00E9421E22AE037ED43E25CE3AE
:106BE0000E9482E20E940FEA60936703C110C5C24F
:106BF0001092620380911701CD80C81609F441C03C
:106C0000B09217016B2D782D892D9A2D20E13EE051
:106C100040E050E00E9464E869012CE3422E512CD0
:106C2000612C712C6B2D782D892D9A2DA301920149
:106C30000E9464E8CA01B901A30192010E9464E8BC
:106C400024E6C216D10408F0BFC27F936F93DF928F
:106C5000CF9282ED9BE09F938F9382E593E09F9389
:106C60008F930E94B3E10FB6F894DEBF0FBECDBF85
:106C700085E0982F990F990F891B880F8058809372
:106C800051030E94A2C100914D0310914E03209127
:106C90004F03309150036B017C01C01AD10AE20A04
:106CA000F30A9701860137FD11C020914C0320950E
:106CB00020934C036A547C4F8F4F9F4F60934D033A
:106CC00070934E0380934F0390935003D0904C03E6
:106CD000D98281E00E94001B80917E15843158F496
:106CE00080918015883038F027E53CE04CE068E082
:106CF00080E50E9463C380917E158431A0F4809169
:106D00008015823080F0E980EE2031F080913706E6
:106D100021E23CE0811102C02BEE3BE042E162E067
:106D200088E60E9463C380917E158C3108F0D0C044
:106D3000E090A514F090A614883028F58091A7144F
:106D40009091A8140E947E92FC01808193E0803291
:106D500029F4818192E0803209F491E043E050E02F
:106D6000491B51094E0F5F1F892F880F880F981BF1
:106D7000892F67E0815F0E94492F69E070E080E021
:106D800090E00E94152280917E158C3130F5809123
:106D90008015843110F1C7010E947E92FC01808130
:106DA00093E0803229F4818192E0803209F491E00D
:106DB00043E050E0491B51094E0F5F1F892F880F98
:106DC000880F981B892F6CE1815F0E94492F69E031
:106DD00070E080E090E00E941522E090A905F0901C
:106DE000AA0580917E15883028F58091AB05909199
:106DF000AC050E947E92FC01808193E0803229F4F0
:106E0000818192E0803209F491E043E050E0491B37
:106E100051094E0F5F1F892F880F880F981B892FEC
:106E200067E0865A0E94492F69E070E080E090E0B8
:106E30000E94152280917E158C3130F5809180154D
:106E4000843110F1C7010E947E92FC01808193E0A1
:106E5000803229F4818192E0803209F491E043E0AC
:106E600050E0491B51094E0F5F1F892F880F880F73
:106E7000981B892F6CE1865A0E94492F69E070E0C7
:106E800080E090E00E94152280917E158C3100F503
:106E9000809180158431E0F0809137068823C1F01D
:106EA00024E6829FC001112481589F4F6FEF70E04C
:106EB0000E94CEE8CB010E947E92AC016CE187E695
:106EC0000E94492F65E270E080E090E00E94152268
:106ED0000E940034882369F180917E15843348F53F
:106EE000809180158A3228F107E028E04AE26AE2C0
:106EF0008AE495E10E946CC405E022E04CE262E382
:106F00008AE495E10E946CC46AE08AE20E9425C48A
:106F100060914C1570914D1582E3809366158BE25C
:106F20008093671526E635E142E38AE495E10E9405
:106F3000C0C280917E15853340F4809180158133E5
:106F400020F06AE486E30E9425C480917E15843394
:106F500068F480918015823348F002E02091670345
:106F600042E367E38AE495E10E946CC480917E1558
:106F70008033D8F4809180158832B8F08091620314
:106F8000882361F042E653E060E387E30E94492FE3
:106F900065E270E080E090E00E94152242E553E057
:106FA00060E3809151030E94492F80917E158732C2
:106FB00008F055C0809180158F3108F450C083E0EF
:106FC0008093811546E24093821568E570E080E089
:106FD00090E00E9415228BE08093811566E2609319
:106FE0008215C980CC2009F404C18DE693E00E948B
:106FF000A82388E280938115F6E2F093821569E573
:1070000070E080E090E00E94152280E3809381157B
:1070100096E2C92EC0928215D980DD2009F40AC1FA
:1070200088E693E00E94A8238DE480938115F6E220
:10703000F09382156AE570E080E090E00E941522EE
:1070400085E58093811586E2C82EC0928215D9808D
:10705000DD2009F412C182E793E00E94A823809109
:107060007E15833338F5809180158B3218F183E0DB
:107070000E94001B83E08093811583E38093821537
:1070800066E070E080E090E00E94152281E00E94BE
:10709000001B80911F01909120010E947E92AC0103
:1070A00063E38CE00E94492F65E270E080E090E0AD
:1070B0000E94152280917E15813408F007C18091CD
:1070C0008015863308F402C1109281158EE38093F7
:1070D00082158BE692E10E948B16898360E870E04E
:1070E0008BE692E10E944A23F981F53108F0EEC067
:1070F00060E270E080E090E00E94152229812F5F1D
:107100002983F2CF243631054CF48536910504F5F8
:107110008A30910534F48AE090E009C08436910504
:10712000BCF0883EE3E09E0714F087EE93E028175A
:10713000390709F4E1CB9093200180931F0110924D
:10714000CE051092CF051092D0051092D105D4CB68
:1071500084E690E0F0CF662351F08EE28093D9036D
:10716000605D6093DA0380E28093DB03AACC80E267
:107170008093DA038093D903F6CF498180E24436C5
:1071800028F0842F64E60E94A0E8805D8093D903F4
:10719000698190E26A3040F02AE0862F622F0E94D7
:1071A000A0E80E94A0E8905D9093DA0389816AE0EC
:1071B0000E94A0E8905D9093DB0369ED73E082E6A6
:1071C00093E00E946EEB16CD7F936F93DF92CF9288
:1071D00088EC9BE09F938F9382E593E09F938F933E
:1071E0000E94B3E10FB6F894DEBF0FBECDBF86E0BC
:1071F00040CD87E00E946B8580FF13C00DE613E051
:10720000F80161918F01662309F4F3CE6F320CF01F
:107210006FE3062E000C770B880B990B0E9415224A
:10722000EFCF8091940580FDE0CE86EE9BE00E943A
:107230004623DFCE87E00E946B85869580FF13C0D2
:1072400008E613E0F80161918F01662309F4ECCEA2
:107250006F320CF06FE3062E000C770B880B990B46
:107260000E941522EFCF80919405869580FDD8CE9F
:1072700086EE9BE00E944623D7CE87E00E946B8576
:107280008695869580FF17C082E793E09A8389836D
:10729000E981FA816191FA83E983662309F4DFCEFB
:1072A0006F320CF06FE3062E000C770B880B990BF6
:1072B0000E941522EDCF809194058695869580FDDC
:1072C000CACE8EED9BE00E944623C9CE0F900F9050
:1072D0000F900F900F90DF91CF911F910F91FF9022
:1072E000EF90DF90CF90BF90AF909F908F907F9066
:1072F0006F905F904F9008950E940034882339F07A
:107300008091C61682FB882780F991E0892708952D
:1073100081E008959091C00095FFFCCF8093C60056
:107320000895CF93DF93EC018991882319F00E948F
:107330008A39FACF8DE00E948A398AE0DF91CF91B5
:107340000C948A39CF93DF93EC01FE01849121964E
:10735000882319F00E948A39F8CFDF91CF910895E0
:10736000E0913E0C81E6E89FF0011124E056F34FD6
:107370008081811107C085E196E20E94A2398AE0EE
:107380000C948A3908950E948A3989E394E00C9418
:10739000A239AF92BF92CF92DF92EF92FF920F93FA
:1073A0001F93CF93DF9384E294E00E94A23960910F
:1073B0006B0470916C0480916D0490916E0445E0B3
:1073C0000E94AF7081E194E00E94A239C0E0D9E050
:1073D000D15021F080E20E948A39FACF8C2F0E948E
:1073E000B4C7CF5FC53099F78AE00E948A3907E0B9
:1073F00014E0C0E080E20E948A398C2F0E94B4C75A
:107400005801D5E080E20E948A39F501C080D18020
:10741000E280F380A7019601C701B6010E9414EB38
:1074200081112CC020E030E0A901C701B6010E9403
:1074300096EA87FD03C08BE20E948A3945E0C701C6
:10744000B6010E94AF70D15084E1A80EB11CD111D9
:10745000D9CF8AE00E948A39CF5F0C5F1F4FC530B9
:1074600049F68AE0DF91CF911F910F91FF90EF9045
:10747000DF90CF90BF90AF900C948A39F12C80E2CE
:107480000E948A39F3948DE3F8E0FF12F9CFDBCF45
:10749000CF92DF92EF92FF926A017B010E94A239A4
:1074A00042E0C701B601FF90EF90DF90CF900C94BF
:1074B000AF70CF93DF93EB010E94A239CE01DF9131
:1074C000CF910C9450B78AE094E00C94A23984E0F8
:1074D00094E00C94A239CF9384E50E947A30C0E006
:1074E0008823D9F00E945630C82F1816B4F40E9491
:1074F000673A8DE40E948A39809145039091460352
:107500000E94BBC76C2FCC0F770B8EE395E00E94D7
:10751000593A8AE00E948A39CFEF8C2FCF91089593
:10752000EC018B01F42E0E9400720E94633A84EEFB
:1075300093E00E94A2390115110511F409E916E240
:10754000209711F4CBEDD3E00E9499201F930F9365
:10755000DF93CF938BEC93E09F938F93D1E0DF93F6
:107560000E947E1F0E948D1DC0914B15C695C69529
:107570008DB79EB707960FB6F8949EBF0FBE8DBF0E
:1075800080918315811104C0D09383150E94EBC2B2
:1075900080914C1590914D150E94C4C2DC2FDD0FD7
:1075A0001D2F1C0F83E00E94001B4BE652E16C2F45
:1075B00080E00E94492F10928115D09382158CEBA8
:1075C00093E00E94462310928115109382158FEA52
:1075D00093E00E9446238AE495E10E9430C681111F
:1075E000E1CF82ED93E00E94A0B589EE93E030E612
:1075F000019729F0232F2A950000E9F7F9CFF89495
:1076000089EE93E038EE019729F0232F2A950000A8
:10761000E9F7F9CF0E940072FF2021F00E94EC33BD
:10762000A895FECF5E9AFCCF8091540B9091550B9C
:107630002FEF3FEF981751F0E92FF0E0EC5AF44F9D
:10764000228130E09F5F9F779093550BC901089589
:107650001F920F920FB60F9211240F900FBE0F9032
:107660001F9018951F920F920FB60F9211240BB610
:107670000F922F933F934F935F938F939F93EF932B
:10768000FF938091C6004091550B9091540B31E0CF
:10769000390F3F77209121032C3008F072C0E22F80
:1076A000F0E0EB5AF44C0C9401E9613B883B973BCA
:1076B000A23BA93BC13BAD3BC13BB13BB53BC13B51
:1076C000B93B803229F0E8F48A3011F08D30F1F4C2
:1076D000431731F0E92FF0E0EC5AF44F8283932FF7
:1076E0009093540BFF91EF919F918F915F914F91E8
:1076F0003F912F910F900BBE0F900FBE0F901F90D8
:1077000018958D3481F021E08E3471F02BE00CC09F
:107710008A3338F48033E0F68032D1F28D32B1F71B
:10772000D7CF8D3499F722E020932103D1CF813335
:1077300029F0843329F0803249F7CACF23E0F4CF0F
:1077400028E0F2CF24E0803379F326E0813361F33F
:10775000DDCF25E08833D1F6E7CF27E08233B1F6DD
:10776000E3CF29E0813391F6DFCF2AE0803371F651
:10777000DBCF8A3019F08D3009F0AACF10922103A7
:10778000A7CF8A3019F08D3009F0A2CF509184151F
:107790005523A1F3273049F02A3059F0253071F7ED
:1077A0001092520110929103E9CF21E020937104CD
:1077B000E5CF21E020937004E1CF8EBD0DB407FE2C
:1077C000FDCF08958FEF8EBD0DB407FEFDCF8EB5B2
:1077D0000895909164009B7F90936400982F906A25
:1077E00096959CBD80FD03C091E0863009F490E041
:1077F0009DBD0895CF92DF92EF92FF92CF936B01E0
:107800007C01C42F4A3069F4F7FE0BC0F094E09479
:10781000D094C094C11CD11CE11CF11C8DE20E94CB
:107820008A394C2FC701B601CF91FF90EF90DF90BE
:10783000CF900C944DC7CF92DF92EF92FF926A01E6
:107840007B010E94A2394AE0C701B601FF90EF9088
:10785000DF90CF900C94FA3B2F923F924F925F9221
:107860006F927F928F929F92AF92BF92CF92DF9250
:10787000EF92FF920F931F93CF93DF93CDB7DEB7B5
:10788000EB970FB6F894DEBF0FBECDBF85E40E9424
:107890007A30882321F00E94961C811183C283E5EF
:1078A0000E947A30882309F45EC00E94961C9A8355
:1078B000898383E40E947A30A5E07A2E882319F028
:1078C0000E94961C782E60E085E50E9495308FAB73
:1078D00060E08DE49BE00E94971F49815A81BA01C4
:1078E000550F880B990B0E9423E2162F7D838E8300
:1078F000292E0E94A2C16B877C878D879E8760910D
:107900005001709151016F507109072E000C880BC6
:10791000990B0E9423E29B01AC01612F7D818E8136
:10792000922D0E9496EA18161CF58EEF9AE00E949E
:10793000A239EB960FB6F894DEBF0FBECDBFDF9134
:10794000CF911F910F91FF90EF90DF90CF90BF905C
:10795000AF909F908F907F906F905F904F903F90EF
:107960002F900C94D7BA24EB30E03A832983A1CF2F
:107970008B859C85AD85BE85805B9C43AF4FBF4F9B
:107980008BAB9CABADABBEAB8AEE9AE00E94A2394A
:107990000E9400728FE78093A91481E080935201C6
:1079A0008B849C84AD84BE848AA69BA6ACA6BDA60F
:1079B0001C8E1D8E1E8E1F8E18A219A21AA21BA22B
:1079C00019821A821B821C822FE730E040E050E0CF
:1079D0002F87388B498B5A8B1F8230E43D8B4CE1CB
:1079E0004E8B56E45F8B188E198E1A8E1B8EFFE716
:1079F000CF2ED12CE12CF12C1EA61FA618AA19AA55
:107A00001AAA1DA21EA21FA218A68CA31C8A1B8A3A
:107A1000312C00E01AAE1BAEA72D770CBB0BB9AF13
:107A2000A8AF80915201882309F48BC00E94A2C1A3
:107A30002B013C01B0917204B9A7BB2309F46BC0C0
:107A40000E94B3726091A5147091A614072E000CC9
:107A5000880B990B0E9423E2362E072F8AAF9BAF2B
:107A6000288D398D4A8D5B8D0E9496EA181634F464
:107A7000388E098F2AAD2A8F3BAD3B8F2F813D89F0
:107A80004E895F89632D702F8AAD9BAD0E941CE2E9
:107A900087FF06C03F820D8B4AAD4E8B5BAD5F8B7F
:107AA0008CA1232D302F4AAD5BAD612F7D818823C2
:107AB00009F494C18E81922D0E941CE287FF2BC095
:107AC000B301A201481959096A097B09DB01CA01FE
:107AD00088589341A109B109B7FD1DC08F859889C8
:107AE000A989BA898C199D09AE09BF09B595A795D1
:107AF000979587958093A9144DA35EA36FA378A74C
:107B0000188F9D81998FAE81AA8F2B8E4B865C86B4
:107B10006D867E861CA220E030E040EF51E4612FAC
:107B20007D818E81922D0E9413E9232D302F4AAD45
:107B30005BAD0E941CE287FF22C087E79AE00E94AB
:107B4000A239109252010E940072F3CE4BEEC42E65
:107B5000D12CE12CF12C95C184E190E0A0E0B0E0C3
:107B60008F87988BA98BBA8B34E1C32ED12CE12C53
:107B7000F12C95C1CF86D88AE98AFA8A90C1D301BF
:107B8000C2012AA53BA54CA55DA5821B930BA40BA6
:107B9000B50BB7FD4CC080E00E9453718AE00E9493
:107BA0008A39D301C2018053984FAF4FBF4F8AA784
:107BB0009BA7ACA7BDA79EA5911167C02FA538A90B
:107BC00049A95AA9632D702F8AAD9BAD0E9496EAF0
:107BD00018160CF046C020E030E040E050E4632D81
:107BE000702F8AAD9BAD0E9413E96FA778AB89AB6C
:107BF0009AABA3019201205B3C434F4F5F4F2BABED
:107C00003CAB4DAB5EAB20E030E040EC50E4612F8C
:107C10007D818E81922D0E9412E9232D302F4AAD55
:107C20005BAD0E941CE2881F8827881F8EA78B856A
:107C30009C85AD85BE8588169906AA06BB0610F4FC
:107C4000D501C401481A590A6A0A7B0A31E8431669
:107C50003FE4530632E16306710480F189E59AE05E
:107C60006ECFD301C2012BA93CA94DA95EA9821BED
:107C7000930BA40BB50B46EB51E265EC71E2B7FD3B
:107C8000D6CF80E00E94CB72D2CF20E030E040EF30
:107C900051E4612F7D818E81922D0E9412E99B011A
:107CA000AC01632D702F8AAD9BAD0E941CE287FF53
:107CB000BECF42E652E262E772E2E3CF48AD59AD91
:107CC0008B899C89481759070CF069C003970CF4FD
:107CD00066C08CEF99E00E94A2398FED99E00E9476
:107CE000A23949815A816B817C8188EF99E00E9499
:107CF000483A8AE00E948A398FED99E00E94A239C1
:107D000048A159A16AA17BA184EF99E00E94483A59
:107D10008AE00E948A398FED99E00E94A2394C8D49
:107D20005D8D6E8D7F8D80EF99E00E94483A8AE0EC
:107D30000E948A399FA9992309F4FBCD29813A81B0
:107D40004B815C812093AA143093AB144093AC1404
:107D50005093AD142CEA35EC47E25EE368A179A1BB
:107D60008AA19BA10E9482E26093AE147093AF142B
:107D70008093B0149093B1142CEA35EC47E25EE3A3
:107D80006C8D7D8D8E8D9F8D0E9496E96093B214CF
:107D90007093B3148093B4149093B514CACD0E9419
:107DA00009313FCE89E29BE0EB960FB6F894DEBF37
:107DB0000FBECDBFDF91CF911F910F91FF90EF903C
:107DC000DF90CF90BF90AF909F908F907F906F90FB
:107DD0005F904F903F902F900C94A2398E81922DFE
:107DE0000E9496EA18160CF096CED301C2012B859C
:107DF0003C854D855E85821B930BA40BB50BAC01B6
:107E0000BD01485853416109710977FD84CE4B8902
:107E10005C89452B09F4FEC08DA09EA0AFA0B8A43C
:107E2000880E991EAA1EBB1E2DA13EA14FA158A5CA
:107E3000281B390B4A0B5B0BC701B6010E9454E8A3
:107E4000A50194010E94E2E8CF84D888E988FA88E5
:107E5000C20ED31EE41EF51E54E1C516D104E10482
:107E6000F1040CF479CE8CEEC816D104E104F104CF
:107E70000CF06CCE90E8C916D104E104F1040CF4C6
:107E800079CECF86D88AE98AFA8A2EEF30E040E0B0
:107E900050E02C193D094E095F0969017A014F85AF
:107EA000588969897A8982EE9AE00E941B3CB70161
:107EB000A6018DED9AE00E941B3C4F815D896E8981
:107EC0007F8986ED9AE00E94483A488D598D6A8DE7
:107ED0007B8D8FEC9AE00E94483AAB89BC8913975E
:107EE0000CF498C0C701B6010E9423E220E030E004
:107EF00040E850E40E9482E269837A838B839C830A
:107F00002F813D894E895F89688D798D8A8D9B8D02
:107F10000E9412E92BED3FE049E450E40E9482E226
:107F200020E030E040E05FE30E9482E29B01AC0190
:107F300069817A818B819C810E9496E96F83788721
:107F400089879A87C501B4010E9423E22FE632E1B6
:107F500043E85AE30E9482E24B015C012AE939E9D5
:107F600049E15FE36F81788589859A850E9482E285
:107F700069837A838B839C839B01AC010E9413E904
:107F8000A50194010E9496E968A379A38AA39BA303
:107F900029813A814B815C81C501B4010E9482E252
:107FA00020E030E040E05EE30E9482E26C8F7D8F53
:107FB0008E8F9F8F4F81588569857A8589EC9AE0ED
:107FC0000E94483AB501A40183EC9AE00E94483A25
:107FD0008AE00E948A3984EB9AE00E94A2394981A2
:107FE0005A816B817C818EEA9AE00E94483A48A1CE
:107FF00059A16AA17BA188EA9AE00E94483A4C8D77
:108000005D8D6E8D7F8D82EA9AE00E94483A8AE00B
:108010000E948A398F859889A989BA898C0D9D1DFE
:10802000AE1DBF1DB595A795979587958093A9140B
:108030002B893C892F5F3F4F3C8B2B8B1F833D81CE
:108040003D8B4E814E8B2F8A5301420159A55CA373
:1080500062CDCF93DF93EB010E94A239CE01DF9175
:10806000CF910C94D7CB4F925F926F927F928F9269
:108070009F92AF92BF92CF92DF92EF92FF920F93B7
:108080001F93CF93DF9300D01F92CDB7DEB78091BF
:108090003D0C803108F0C7C131E6E32E80913D0CE4
:1080A000803108F0F8C08091540B9091550B891BDA
:1080B0008F7709F4F0C00E94143B97FF0BC00E9419
:1080C000633A89E793E00E94A2398091540B809330
:1080D000550BE4CF8A3019F08D3009F0D3C01092DF
:1080E0003C0C8091DA0B9091DB0BFC01EA52F44FCF
:1080F0001682892B19F40E947586D0CF1092DB0B63
:108100001092DA0B0CED1BE0F8018191803209F43A
:1081100046C08E3409F0A1C064E773E0C8010E9434
:1081200099E16C01892B41F06EE470E0C80104967E
:108130000E9463EB009709F4C8014AE050E070E048
:1081400060E001960E9410DF4B015C018091D60B2C
:108150009091D70BA091D80BB091D90B0196A11D8E
:10816000B11D88169906AA06BB0629F060E081E4D5
:1081700093E0CD2851F16AE270E0C8010E9492EBD1
:108180009C01009729F1982F901BF12C992349F01D
:108190009150F801E90FF11D8081F826F7CF8F018A
:1081A000B3CF4AE050E070E060E0C90101960E9460
:1081B00010DF4F2C512C712C612C64157505860530
:1081C000970551F060E082E293E00E94D0B866CF5C
:1081D00060E088EF92E0F9CF8092D60B9092D70BB7
:1081E000A092D80BB092D90B8091A4058130E1F018
:1081F00067E470E0C8010E9463EB0097A9F04AE0D1
:1082000050E070E060E001960E9410DF623071057E
:108210008105910548F487E592E00E94A23960E06B
:108220008DE492E00E94971F8091DC0B8B3309F460
:1082300035CF80913D0C803108F030CF80913F0CDC
:108240008E9DC00111246CED7BE0805C934F0E94F9
:108250006EEB80E00E949CB821CF8091C61680FF13
:10826000C3CF62E476E2C8010E9499E1009731F041
:10827000FC01838180538A3008F0B6CF60E08EEC39
:1082800092E0A3CF2AED3BE04CED5BE06CE37CE0B9
:108290000E94FE1603CF8091C61682FFC4C01A82C8
:1082A000198281E6F82E90E1B92E29E6A22E80915E
:1082B0003D0C803108F0B7C00E9436178111B3C061
:1082C00041E050E0BE016D5F7F4F88EB94E10E947A
:1082D0005ACD0B8110E0019711F00FEF1FEF809145
:1082E000C0149091C114A091C214B091C314809392
:1082F000C2169093C316A093C416B093C5160E94DD
:1083000036170F3F100749F4811107C00E94633AE6
:1083100081E993E00E94A239CACF40913F0C242FFB
:1083200030E00A3061F00D3051F0882309F46DC05F
:1083300089819A81009719F001969A838983109216
:108340002E0389819A81F29EF001F39EF00D112493
:10835000E35CF34FDF01A80FB91F13961C92892B22
:10836000B9F50E9475860E943617882309F49FCFBD
:108370000E94BE7788EB94E10E94696C8091BD16E3
:108380008823F1F181508093BD168A9DC00111248C
:1083900062E0835E9A4F0E9491CFE091BD1624E087
:1083A000E29FF0011124E75EFA4F40815181628122
:1083B00073814093C2165093C3166093C416709392
:1083C000C51688EB94E10E9432CC0E94D0C76FCFD3
:1083D0001A82198283818D3479F48481823361F425
:1083E0008581853349F4868180538A3028F08091D5
:1083F000C6168B7F8093C61681E00E949CB8B3CFCF
:108400000E94C1C7B092A40552CF4F9DA001112474
:10841000405C534F9E012F5F3F4F6EE273E0802F11
:108420000E94FE1644CF0E94A2C14B015C018091C4
:108430003C0390913D03A0913E03B0913F03009710
:10844000A105B10551F14091E8055091E905609110
:10845000EA057091EB05840F951FA61FB71FA501B4
:108460009401281B390B4A0B5B0BDA01C901B7FDDC
:1084700014C00E94633A6091F1057091F20580E1A9
:1084800092E00E9429408AE00E948A3940E070E030
:1084900060E090E080E00E94903A80910B01909122
:1084A0000C01A0910D01B0910E01892B8A2B8B2B11
:1084B00079F090911E1580911F15981709F4FCC052
:1084C0008092E8059092E905A092EA05B092EB054A
:1084D0000E94A2C16B017C0180919103811108C0AF
:1084E00020911E1590911F1581E0291301C080E095
:1084F0002091A5143091A61491E089272A3A3105DC
:108500000CF480E091E040912A0350912B0360919C
:108510002C0370912D03452B462B472B09F490E03B
:10852000981789F0882309F401C1D701C601805644
:108530009444A24FBF4F80932A0390932B03A093A0
:108540002C03B0932D034090500B5090510B609032
:10855000520B7090530B20912603309127034091CA
:10856000280350912903C301B2010E941CE2882311
:1085700019F180912A0390912B03A0912C03B091C3
:108580002D03409226035092270360922803709295
:108590002903892B8A2B8B2B09F449C0D701C601EB
:1085A00080569444A24FBF4F80932A0390932B038D
:1085B000A0932C03B0932D0380912A0390912B0359
:1085C000A0912C03B0912D030097A105B10579F17D
:1085D000C81AD90AEA0AFB0AF7FC29C010922A0332
:1085E00010922B0310922C0310922D038BEF91E02D
:1085F0000E94A23960E087EE91E00E94971F80916F
:10860000A7149091A8141816190624F490E080E09D
:108610000E946AA08091AB059091AC0518161906CE
:1086200034F41092AC051092AB050E948A628091DE
:108630002F0390913003A0913103B0913203A50133
:108640009401281B390B4A0B5B0BDA01C901B7FDFA
:108650008FC090911E1580911F15F09037069817C6
:1086600049F0E0911F153BE4E39FF0011124EF5620
:10867000F94FF0800E94A2C1FF2009F4D1C00091FF
:108680002203109123032091240330912503011527
:1086900011052105310509F04DC06C597F4F8F4FF1
:1086A0009F4F60932203709323038093240390933E
:1086B0002503FF24FA9444C00E94A2C10091E8055A
:1086C0001091E9052091EA053091EB05C0900B016E
:1086D000D0900C01E0900D01F0900E010C0D1D1DCD
:1086E0002E1D3F1D601B710B820B930B97FF03C068
:1086F00010923303EDCE809133038111E9CE81E0F6
:10870000809333035E9A809194058E7F80939405C5
:108710005E9A809194058D7F80939405159A80913F
:1087200094058B7F809394055E9AD2CE80E090E092
:10873000DC0101CF601B710B820B930B97FDB9CF4E
:108740000F2D10E084E00E945AB8F11072C060E072
:1087500084E00E94ABC044E6840E911CA11CB11CB5
:1087600080922F0390923003A0923103B092320393
:108770000E9475868091A4058823F1F1109108016B
:108780001130B1F18091C61680628093C61681E0E7
:108790008093080164EF71E080E090E00E94C833AC
:1087A0000E94F2D18091C61683FFA5C0123028F432
:1087B00060E080EA93E00E94971F01E083E08093ED
:1087C00053010E94A2C16C597F4F8F4F9F4F6093FE
:1087D0008503709386038093870390938803002317
:1087E00039F0123029F481E08093BC160E944DD2FA
:1087F0000E945E940E9409310F900F900F90DF91BC
:10880000CF911F910F91FF90EF90DF90CF90BF908D
:10881000AF909F908F907F906F905F904F90089552
:108820001092220310922303109224031092250326
:1088300087CF0F3F110511F461E08ACFEDE7F6E233
:10884000E491E150EA3008F051C0F0E0E65DFB4B06
:108850000C9401E9344439443E4448447644764417
:1088600052445A4462446C4484B5806884BDF7BC69
:1088700072CF84B5806284BDF8BC6DCF80918000DA
:10888000806880938000109389000093880063CFF4
:108890008091800080628093800010938B00009311
:1088A0008A0059CF8091B00080688093B000F09228
:1088B000B30051CF8091B00080628093B000F092FD
:1088C000B40049CF8091900080688093900010930D
:1088D0009900009398003FCF809190008062809330
:1088E000900010939B0000939A0035CF003811053B
:1088F0000CF0A2CF2CCF00E0112309F479CF5ECF8A
:108900002F923F924F925F926F927F928F929F929F
:10891000AF92BF92CF92DF92EF92FF920F931F938D
:10892000CF93DF93CDB7DEB764970FB6F894DEBF71
:108930000FBECDBF8091FB0A83FDB0C10E946B3A90
:10894000898787FDABC189E40E947A30882309F4C6
:1089500097C10E94563090E01816190614F481E071
:1089600090E026E0289FF001299FF00D1124E255A8
:10897000FA4F808191811B8A0E946AA02091A714DE
:108980003091A8148091A5149091A6148217930792
:108990008CF48FEC99E09F938F938AED99E09F93ED
:1089A0008F931F920E947E1F0F900F900F900F9039
:1089B0000F9005C02B8984EC99E0222361F381E0BC
:1089C000809352011C821D821E821F821A861B8682
:1089D0001C861D861F862CE3288B3CE1398B46E4E0
:1089E0004A8B212C312C50E85A838FEB8B831982D0
:1089F00091E09E87812C912C540101C01E8600912C
:108A0000A7141091A814B801012E000C880B990B23
:108A10000E9423E2D62EE72EF82E988791014A81F4
:108A20005B810E941CE2882391F08091A5149091B3
:108A3000A6143B893111E7C041E0498308171907A3
:108A40000CF019822D2C3E2CFA8258855B830E94F3
:108A5000A2C16B017C01DC01CB012A853B854C85E1
:108A60005D85821B930BA40BB50BB7FD2FC0D701FF
:108A7000C60188519C4FAF4FBF4F8A879B87AC87F9
:108A8000BD8789850E94537180EC99E00E94A239CC
:108A900081149104A104B10409F4E0C0C501B4013A
:108AA0006053784F8F4F9F4F6C197D098E099F0936
:108AB00028EE33E040E050E00E9464E8CA01B901CA
:108AC0004AE00E94FA3B8AE00E948A390E943340C1
:108AD0000E94A2C16093E8057093E9058093EA05BE
:108AE0009093EB056091A5147091A614072E000CCD
:108AF000880B990B0E9423E26887072F182F9C8B05
:108B0000262F372F482F592FB1018A819B810E9430
:108B100012E92B013C0120E030E0A9010E9496EA15
:108B200087FF04C077FA709477F8709481149104E9
:108B3000A104B10409F096C020E030E040E85FE312
:108B4000C301B2010E941CE287FF10C09E85812CE8
:108B5000912C5401992331F08AE9882E82E0982ED5
:108B6000A12CB12C8C0C9D1CAE1CBF1CA981AA236E
:108B700099F12C813D814E815F812115310541059F
:108B8000510541F0D701C601821B930BA40BB50B15
:108B9000B7FD22C02885302F412F5C896F857889E9
:108BA00089899A890E9412E920E030E040EC5FE375
:108BB0000E941CE287FD2AC0D701C601805A954158
:108BC000AF4FBF4F8C839D83AE83BF8398859F87B4
:108BD000088B198BAC89AA8B809152018823B1F044
:108BE00081149104A104B10409F408CFB0EDCB1AAB
:108BF000B7E0DB0AE108F108C818D908EA08FB0861
:108C0000F7FCFCCE03C0081719070CF58091520140
:108C1000882309F443C01092520164960FB6F89469
:108C2000DEBF0FBECDBFDF91CF911F910F91FF909F
:108C3000EF90DF90CF90BF90AF909F908F907F90FC
:108C40006F905F904F903F902F900C94D7BA2D2C3F
:108C50003E2CFA8288858B831982F9CE8FE30E949D
:108C60008A3931CF20E030E040E450E4C301B20162
:108C70000E9496EA18160CF079CF4601570176CF7C
:108C800083E50E947A308B8B811105C082E50E94BA
:108C90007A30882319F00E94961C6ECE64960FB627
:108CA000F894DEBF0FBECDBFDF91CF911F910F9122
:108CB000FF90EF90DF90CF90BF90AF909F908F90FC
:108CC0007F906F905F904F903F902F9008952F92DC
:108CD0003F924F925F926F927F928F929F92AF924C
:108CE000BF92CF92DF92EF92FF920F931F93CF9399
:108CF000DF93CDB7DEB7CB54D1090FB6F894DEBF02
:108D00000FBECDBF2C968FAF2C97809147038D342B
:108D100009F481C4843511F40C94EA5B873491F42E
:108D200080914503909146038C31910509F434C23A
:108D300008F06AC08430910509F4AEC130F402979E
:108D400008F4F7C00E94FDBA77C18531910509F496
:108D500073C14B97B9F70E940BBB81116DC18CE0B9
:108D6000EEE5F1E0DE01119601900D928A95E1F7B2
:108D700070E060E080E50E94873040E050E068E409
:108D800072E44CA35DA36EA37FA340E050E060EAD1
:108D900070E448A359A36AA37BA3813009F4B5C149
:108DA000823009F4D1C120E030E040E050E460912D
:108DB0004C0B70914D0B80914E0B90914F0B0E947C
:108DC00013E97B018C0120E030E04AE753E40E9484
:108DD00096EA181624F4E12CF12C0AE713E4A9848E
:108DE000BA84CB84DC849701A801B501C6010E9436
:108DF00096EA181614F475018601C701D8018C8F04
:108E00009D8FAE8FBF8FC2C18A35910509F4E6C32D
:108E100060F58D31910509F43DC38A9709F092CF31
:108E20008091A405813009F007C189E40E947A305D
:108E3000082F10E0882319F00E94961C182F8AE44E
:108E40000E947A30F82E882311F40C944C5C0E9416
:108E5000961C002309F421C3153010F40C943E5CD9
:108E60008AE595E00E94A239E7C08B35910509F4A7
:108E7000B8C38C35910509F065CF9AE6C92E91E00B
:108E8000D92EF12CE12C00E010E0D6018D916D017E
:108E90000E947A30382E8823E1F10E949A1C4B01FF
:108EA0005C01133059F0F701EF5FF94F20813181F8
:108EB000428153810E9412E94B015C01F701EC5B96
:108EC000F44F2081318142815381C501B4010E9458
:108ED00012E92B013C012DEB37E346E855EB0E94EC
:108EE00096EA87FD0AC02DEB37E346E855E3C30158
:108EF000B2010E941CE2181664F4133009F075C325
:108F00008092500B9092510BA092520BB092530B47
:108F1000032D1F5FB4E0EB0EF11C143009F0B5CF48
:108F2000002321F080E59BE00E94A3830E94348E01
:108F300083C08091A405813009F07EC06DEEC62EFD
:108F400063E0D62E74E4E72E7BE0F72EE1E0AE2E50
:108F5000E6E0BE2E10E088E5810F0E947A3088237B
:108F600009F47EC00E949A1C2B013C01812F0E94B3
:108F70005217882309F46AC0D7012D913D914D9174
:108F80005C91C301B2010E9413E9D6016D937D93F8
:108F90008D939C9313971F5FF4E0CF0ED11C24E0B8
:108FA000E20EF11C34E0A30EB11C1330A1F685E4EF
:108FB0000E947A30882309F45EC00E949A1C6B01DB
:108FC0007C0183E00E945217882371F02091500B9E
:108FD0003091510B4091520B5091530BC701B60188
:108FE0000E9413E96B017C01C092F903D092FA034D
:108FF000E092FB03F092FC0386E40E947A3088231F
:10900000C9F00E949A1C20E030E0A9010E9496EA73
:10901000181684F40E949A1C20E030E040E752E4E5
:109020000E9496E9609321017093220180932301AD
:10903000909324010E947E892C96FFAD2C97F1110C
:109040000C949B510E94B0390C949B51F5012081E6
:10905000318142815381C301B2010E9412E995CF4F
:10906000F70180819181A281B381F6018083918390
:10907000A283B38390CF8091500B9091510BA0911C
:10908000520BB091530B8093F9039093FA03A09382
:10909000FB03B093FC03B0CF80E50E947A30C12C73
:1090A000D12C7601882321F00E94761C6B017C0173
:1090B00083E50E947A30882361F00E949A1C20E0A8
:1090C00030E04AE754E40E9482E20E940FEA6B011A
:1090D0007C010E94BE7780916B12811105C060E017
:1090E00081E595E00E94971F0E94A2C1C60ED71E7F
:1090F000E81EF91E0E94A2C16C197D098E099F0904
:1091000097FF9ACF0E943340F5CFBE01605E7F4F3C
:10911000CE0109960E945486E0904C0BF0904D0BC6
:1091200000914E0B10914F0B2D813E814F81588540
:1091300069817A818B819C81DE0194966D010E9408
:109140009C850E94348E78CF29853A854B855C8535
:1091500060914C0B70914D0B80914E0B90914F0B89
:109160000E9413E96B017C0120E030E04AE753E400
:109170000E941CE287FD06C0C12CD12C5AE7E52EC7
:1091800053E4F52ECC8EDD8EEE8EFF8EBE01605E3A
:109190007F4FCE014C96BECF87E00E946B8588231F
:1091A00009F464C10E94BE77109228016091010405
:1091B0008CE40E949530982E80E00E94BA300E9484
:1091C000A2C16093E8057093E9058093EA05909346
:1091D000EB058091210190912201A0912301B09192
:1091E00024018093380390933903A0933A03B093FA
:1091F0003B0380911F01909120019093370380934E
:10920000360384E690E09093200180931F0181E073
:10921000809392050E94318F8AE50E94451CA82EFA
:1092200088E50E94451C182F89E50E94451CB82E30
:10923000181308C0B12EA11205C011E0BB24B394CD
:10924000AA24A39482E50E947A30882309F416C1E7
:109250000E949A1C3B01882EC92E20E030E0A90113
:109260000E941CE2882309F444C0111103C0BB20F2
:1092700009F4D0C0D0904C0BE0904D0BF0904E0B09
:1092800000914F0B9301482D5C2D6D2D7E2D8F2D60
:10929000902F0E9496EA181624F0D62CE72CF82C72
:1092A0000C2D80E090E0A0E8B0E48C8F9D8FAE8F15
:1092B000BF8F20E030E04AE753E46D2D7E2D8F2DE7
:1092C000902F0E941CE287FD05C0D12CE12C2AE7DB
:1092D000F22E03E48D2D9E2DAF2DB02F89839A831E
:1092E000AB83BC83BE01645E7F4FCE0101960E94BA
:1092F0005486112309F489C0BB2009F483C010925D
:10930000440B1092450B1092460B1092470B109293
:10931000480B1092490B10924A0B10924B0B0E9473
:109320007386EBE9F6E1C590D590E590F490EFE90E
:10933000F6E14590559065907490A7019601C301A0
:10934000B2010E941CE287FFA0C0A7019601C301E1
:10935000B2010E9496E99B01AC010E9482E220E0EA
:1093600030E040E85FE30E9413E90E94D4EA20E085
:1093700030E048E452E40E9482E269837A838B837E
:109380009C8320914C0B30914D0B40914E0B509192
:109390004F0B28A739A74AA75BA720E030E040EC95
:1093A0005FE3C301B2010E9482E22B013C0177FA24
:1093B000709477F8709420E030E040EC5FE3C701F0
:1093C000B6010E9482E29058AE014F5F5F4F6A0182
:1093D000E8A4F9A40AA51BA5A30192010E949C85FB
:1093E0000E944C901092440B1092450B1092460B29
:1093F0001092470B1092480B1092490B10924A0B97
:1094000010924B0B80E00E94E38CBB2019F081E0AE
:109410000E94E38CAA2019F082E00E94E38C0E9453
:1094200073868091910580939205892D0E94BA30B0
:109430008091380390913903A0913A03B0913B0396
:109440008093210190932201A0932301B0932401E2
:1094500080913603909137039093200180931F01F0
:1094600083E0809353010E94348EE6CD60E08FE468
:109470000E949530882309F495CEDECD612C712CA5
:1094800030E8832E40E4C42EF0CEA3019201C70140
:10949000B6015FCF0E94CD5CCFCD853008F0E0CC27
:1094A00090E1E4E4FBE0ADEEB3E001900D929A951B
:1094B000E1F70023A1F054E01502F0011124E75672
:1094C000FA4E40815181628173814093ED03509344
:1094D000EE036093EF037093F003FF2091F094E0AC
:1094E0008902F0011124EB57FA4E80819181A2810B
:1094F000B3818093F1039093F203A093F303B093AD
:10950000F40386E40E947A30811151C0C12CD12C21
:1095100076018090210190902201A0902301B090CB
:10952000240120E030E0A901C701B6010E941CE23D
:10953000882341F0C0922101D0922201E0922301C0
:10954000F092240100911F011091200184E690E027
:109550009093200180931F01C0905801D090590131
:10956000E0905A01F0905B0180E090E0A0E8BFE35A
:109570008093580190935901A0935A01B0935B01D5
:109580000E947E898092210190922201A092230163
:10959000B09224011093200100931F01C092580142
:1095A000D0925901E0925A01F0925B0145CD0E94A0
:1095B0009A1C6B017C0120E030E0A9010E9496EA30
:1095C00018160CF0A3CF20E030E040E752E4C701CA
:1095D000B6010E9496E96B017C019BCF109240037B
:1095E0002BCD8FE08093400327CDF701EF51FC4F47
:1095F0005F01A301920160817181828193810E9448
:1096000013E9D5016D937D938D939C931397812FCF
:109610000E944B857ECC8091450390914603823712
:10962000910511F40C941B5508F080C18934910503
:1096300009F445C608F0D9C08831910509F498C4E9
:1096400008F06CC08231910511F40C942A5400F595
:109650008230910508F411C4419709F073CB8BE077
:1096600092E00E94211C882309F45BC488E50E94D3
:10967000451C81115E9889E50E94451C81115E9808
:109680008AE50E94451C882309F4D6CC1598D4CCD1
:109690008531910509F456C458F5449709F052CB29
:1096A0008091C61683FF47C48EE995E00E94A239D7
:1096B0008091C61683FF17C08EEE94E10E94C16DA3
:1096C0008BE1EEEEF4E1DE01119601900D928A95A8
:1096D000E1F770E060E0CE0101960E94BBD0CE01C0
:1096E00001960E94C66D8FE895E00E94A239A4CC35
:1096F0008631910509F429C4479709F023CB80915D
:10970000410390914203FC012191222309F42AC4D0
:109710002032D1F7DF0111971C92F6CF8C319105E1
:1097200009F4A5C420F58A31910509F44FC408F461
:109730002EC483E40E94451C882309F467C489EC85
:1097400095E00E94A2398091BB14882309F459C482
:10975000BE016F5F7F4F88EB94E10E948C6CCE015D
:1097600001960E94D7CB8AE00E948A3965CC8E315F
:10977000910509F48BC408F482C48F31910509F472
:10978000F4C4809709F0DECA8091C61682FD0E945B
:10979000BE778091C61683FF4FCC60E080E50E94C3
:1097A0009530182F682F80914103909142030E94B9
:1097B00091CF83E50E947A30882381F00E94861C35
:1097C000AB01BC014093C2165093C3166093C416FC
:1097D0007093C51688EB94E10E9432CC0E94D0C7EA
:1097E00011112ACC0E94A79027CC8C35910511F439
:1097F0000C947E5408F049C08135910511F40C9405
:10980000055478F48C34910509F469C58D349105BB
:1098100009F47AC58B34910509F094CA0E94A79087
:109820000BCC8335910511F40C94225410F40C9454
:109830001A548435910511F40C942A5485359105F8
:1098400009F080CA83E50E94451C882309F4F4CB03
:109850000E94A2C16093E8057093E9058093EA0530
:109860009093EB050E949A1C20E030E04AE754E414
:109870000E9482E20E940FEA60933C0370933D03D2
:1098800080933E0390933F03D7CB8C36910509F428
:10989000D3CBE8F58936910509F43EC540F5883605
:1098A000910509F04FCA8091FB0A83FDC5CB0E9448
:1098B0006B3A87FDC1CB89E40E947A30882311F48A
:1098C0000C940B5C0E94563090E01816190614F4A4
:1098D00081E090E026E0289FF001299FF00D1124FF
:1098E000E255FA4F808191810E946AA0A5CB8A3609
:1098F000910509F43AC58B36910509F023CA80E534
:109900000E9460BB811198CB1092370695CB8E36A2
:10991000910509F45EC508F4FBC48F36910509F47E
:109920006BC58037910509F487CB0CCA8232E1E020
:109930009E0711F40C94E25708F0AAC18E3B9105E2
:1099400009F4C7C508F094C08737910511F40C9449
:10995000705588F48537910511F40C94235510F057
:109960000C9435558337910509F0ECC988EB96E0E6
:109970000E94A23961CB8937910511F40C947D5571
:1099800010F40C9474558C38910509F476C581391E
:10999000910509F0D7C983E50E947A30882311F434
:1099A0000C9485550E94961C823010F00C948955B9
:1099B0008C01112788E40E947A308823D1F00E941C
:1099C000961C8A3A910514F40C9491550E94961CA9
:1099D0008D32914014F00C9495550E94961C26E00F
:1099E000209FF001219FF00D1124E255FA4F918341
:1099F000808382E40E947A308823C9F00E94961CFA
:109A0000059714F40C9499550E94961C8D38910575
:109A100014F00C949D550E94961C26E0209FF001A6
:109A2000219FF00D1124E255FA4F9383828386E43F
:109A30000E947A30882309F4FFCA0E94961C97FF7F
:109A400002C00C94A1550E94961C8F3F910519F0FD
:109A500014F00C94A5550E94961C26E0209FF0015E
:109A6000219FF00D1124E255FA4F95838483E4CAB7
:109A70008D3C910511F40C94415608F070C0893C5E
:109A8000910511F40C94AC5590F5883C910509F0C2
:109A900059C90E946B3A182F87FDCECA009106045F
:109AA00084E40E947A30F82E8823C1F00E949A1C28
:109AB0004B015C0120E030E0A9010E941CE28823F8
:109AC00011F40C94A95524E01202F0011124EE5F68
:109AD000FB4F80829182A282B3820F2D602F83E59B
:109AE0000E949530809306040E94575FA5CA8B3C64
:109AF000910511F40C94D6558C3C910509F022C9BE
:109B000083E092E00E94211C81110C94F955409150
:109B1000300B5091310B6091320B7091330B84EE0E
:109B200097E00E94483A4091340B5091350B609178
:109B3000360B7091370B81EE97E00E94483A4091C6
:109B4000380B5091390B60913A0B70913B0B87E1C8
:109B500098E10E94483A8AE00E948A396DCA833DA2
:109B6000910511F40C94C25608F04DC045E9E42E5D
:109B700045E0F42E10E08E3C910509F0E3C888E53D
:109B8000810F0E94451C882351F00E949A1CF70106
:109B90006083718382839383812F0E944B851F5F33
:109BA000F4E0EF0EF11C133051F780E192E00E94D7
:109BB000211C8111BBC9409195055091960560917A
:109BC00097057091980586E298E00E94483A409186
:109BD000990550919A0560919B0570919C0588E5C7
:109BE00097E20E94483A40919D0550919E056091F0
:109BF0009F057091A00585E597E20E94483A8AE0AA
:109C00000E948A3919CA8C3D910511F40C948A5727
:109C10008D3D910509F096C80E946B3A082F87FD8B
:109C20000BCA83E50E947A30002E000C110B7801DC
:109C3000EE0CFF1C882311F40C94C8570E94961C4C
:109C4000F701EB5DFE4F91838083000F111F000F22
:109C5000111F9801285A3E4F7901BC01990F880BBA
:109C6000990B0E9423E22AE037ED43E25CE30E9475
:109C700082E203501C4FD8012D913D914D915C9192
:109C80000E9482E2F7016083718382839383D4C947
:109C90008C3A21E0920711F40C94FE5A08F083C02C
:109CA0008F3241E0940711F40C94035910F58D3272
:109CB000A1E09A0711F40C943C5810F00C94BD5894
:109CC0008C32914009F03EC864E071E083E50E9467
:109CD00087308C0168EE73E080E50E948730893818
:109CE000F3E19F0710F088E893E1B8010E94BA946D
:109CF000A3C98A39F1E09F0709F49EC938F4803975
:109D0000914009F01FC80E94BE7796C9843A41E08D
:109D1000940711F40C940759853A914011F00C9472
:109D2000A24688E50E94451CC82E89E40E94451C75
:109D3000A82E882311F40C94655A0E94961C082FB3
:109D400089E50E94451CF82E8AE40E94451CE82EF5
:109D5000882311F40C94905A0E94961C182F8AE5BF
:109D60000E94451CD82EB12C811104C081E50E94AF
:109D7000451CB82EA11001C0E12C8E2D90E0C11021
:109D800001C0F12C8F0D911D019731F4D1100C946D
:109D9000BB5AB1100C94BB5A0E94633A87E299E017
:109DA0000E94A23949C9883FA1E09A0711F40C9496
:109DB000B85B18F5853FE1E09E0711F40C94B05BA9
:109DC00040F4843F914011F00C94A2460E948974A3
:109DD00033C9863F31E0930711F40C94B45B873F9D
:109DE000914011F00C94A24661E083E50E94953009
:109DF00091E089270E94A4A01FC9803A53E09507EB
:109E000009F4A5C178F48C30924011F00C94A2466C
:109E10008091C61682FD02C00C94CB5B8064809357
:109E2000C6160AC9873EE3E09E0711F40C94D35B83
:109E3000893E934011F00C94A2468091BC1681118A
:109E40000C94E35B0E945A906D3371058105910576
:109E500020F08AEA99E00E945B5C86EA99E00E9421
:109E60005B5C84EE8093CA0382E999E00E94A23988
:109E70008EE899E00E945B5CDFC880E50E947A3042
:109E8000C12CD12C7601882321F00E94761C6B0115
:109E90007C0183E50E947A30882361F00E949A1C3D
:109EA00020E030E04AE754E40E9482E20E940FEA98
:109EB0006B017C010E94BE77809141039091420327
:109EC0000097E1F00E9479B881E080939103C1147A
:109ED000D104E104F10431F00E94A2C1C60ED71EE4
:109EE000E81EF91E809191038823B1F0C114D104BA
:109EF000E104F10449F40E943340F4CF60E083E7C9
:109F000095E00E94971FE0CF0E94A2C16C197D09C5
:109F10008E099F0997FDEFCF109291030E94D7BA47
:109F20008BC860E086E895E00E94971F5E985E9877
:109F300015985E9881C80E94673A8FEA95E00E9462
:109F4000A2397AC80E94F2D177C88091C61682FDE4
:109F500073C80E94C1C78091C616877F80628093B4
:109F6000C6166AC860E00E9491CF1092CA0364C806
:109F70000E940034882321F00E94D0C70E94A7903D
:109F80008FE99CE00E94A0B50E94D7BA55C8809185
:109F9000C61682FF03C08B7F8093C6168091000691
:109FA000813069F482E0809300060E94A2C1609330
:109FB000DD037093DE038093DF039093E0030E9440
:109FC000D7BA89EB95E00E94A0B536C88091C61635
:109FD00083FF32C883E50E947A30882309F42CC8B5
:109FE0000E94861CAB01BC014093C2165093C3165D
:109FF0006093C4167093C51688EB94E10E9432CC2E
:10A000001BC88FEB95E00E94A239ADCB8091C6169C
:10A0100082FF27C0C090C216D090C316E090C4162D
:10A02000F090C51688ED95E00E94A2394AE0C7017C
:10A03000B6010E944DC78FE20E948A396091BE1618
:10A040007091BF168091C0169091C1164AE00E948F
:10A050004DC78DE00E948A398AE00E948A390C94AB
:10A060001C488AEE95E00E94A2390C941C4880910D
:10A070004103909142030E9449CF0C941C48809167
:10A08000C6168E7F8093C6160C941C488091C61607
:10A0900083FD02C00C941C480E9418CC8091C61607
:10A0A00083FD02C00C941C4840914103509142032F
:10A0B000BE01645E7F4F80E00E9457B78C0100971D
:10A0C00011F40C941C486C8D7D8D19821C8222E049
:10A0D000AC01CE0101960E94CC6D811119C0F12C0A
:10A0E000CE0101960E94C66DB801FF2031F186E1D4
:10A0F00096E00E9429408AE00E948A391092C21696
:10A100001092C3161092C4161092C5160C941C48D7
:10A11000CE0101960E94C6CC882309F361E0CE01EE
:10A1200001960E94726C0097D1F225EEDC012C930F
:10A130001C820E9467C8F82ED3CF8EEF95E00E9454
:10A1400029408BEF95E00E94A2390C941C48209185
:10A150004103309142039091C61692609093C616C7
:10A16000C9010E9449CF0C941C480E945A907B015F
:10A170008C0120E831E541E050E00E9464E8C9012B
:10A180006DE671E00E94BAE84B015C01C801B701BD
:10A1900020E13EE040E050E00E9464E8CA01B901DD
:10A1A00028E130E040E050E00E9464E8762E672E1F
:10A1B000C62ED72E8CE3282E312C412C512CC801D1
:10A1C000B701A20191010E9464E8F62EE72ECA01B0
:10A1D000B901A20191010E9464E8CB018E010F5FD9
:10A1E0001F4F8114910431F1EF92FF927F936F938F
:10A1F0006F927F92BF92AF929F928F928CE496E083
:10A200009F938F931F930F930E94B3E10FB6F8941F
:10A21000DEBF0FBECDBFC8010E9479B80E94673A69
:10A22000B80180E696E00E9429408AE00E948A39BF
:10A230000C941C48A114B10489F0EF92FF927F9313
:10A240006F936F927F92BF92AF928CE396E09F9351
:10A250008F931F930F930E94B3E1D8CFCD2879F04D
:10A26000EF92FF927F936F936F927F9280E396E0DD
:10A270009F938F931F930F930E94B3E1C7CF892BB6
:10A2800069F0EF92FF927F936F9388E296E09F933D
:10A290008F931F930F930E94B3E1B8CFEF92FF9279
:10A2A00084E296E09F938F931F930F930E94B3E1F4
:10A2B0000F900F900F900F900F900F90ACCF80E504
:10A2C0000E94451C882311F40C941C480E945630AF
:10A2D000853608F084E68093CA030C941C4880916C
:10A2E0000006813011F00C941C4882E08093000637
:10A2F0000E94A2C16093DD037093DE038093DF03AD
:10A300009093E0030C941C480E94CB900C941C4842
:10A310000E9480440C941C480E946B3A182F87FDC1
:10A320000AC08DE696E00E94A239812F0E945371E7
:10A330008AE00E948A39C55BDF4F0FB6F894DEBF12
:10A340000FBECDBFDF91CF911F910F91FF90EF9086
:10A35000DF90CF90BF90AF909F908F907F906F9045
:10A360005F904F903F902F90089580E50E9460BBD2
:10A3700081110C941C4881E40E94451C60913706B1
:10A38000062F10E0811102C00FEF10E089E40E9457
:10A390007A30882311F40C94165C0E94563090E0B9
:10A3A0001816190614F481E090E026E0289FF001C9
:10A3B000299FF00D1124E255FA4F048115810F3FBA
:10A3C000110519F010F00FEF10E0009337060C9410
:10A3D0001C488EE40E947A30882311F40C941C48A7
:10A3E0000E94861C6093D60B7093D70B8093D80B7A
:10A3F0009093D90B0C941C4883E50E94451C88233C
:10A4000029F083E50E9460BB8093FB0A0E94673AB3
:10A410008EE796E00E94A2398091FB0A882351F1D1
:10A4200010E000E020E08091FB0A90E0B0E0A0E0C6
:10A43000002E04C0B695A795979587950A94D2F7F4
:10A4400080FF12C0FF24F394F20E222319F08CE255
:10A450000E948A39F801EE0FFF1FEC58F94F8591E1
:10A4600094910E94A2392F2D0F5F1F4F05301105C7
:10A47000D1F679C980E796E0C6CD8091FB0A83FFCB
:10A4800002C00C941C4889E40E947A30882311F49D
:10A490000C94225C0E94563090E01816190614F4B1
:10A4A00081E090E026E0289FF001299FF00D112423
:10A4B000E255FA4F828193818C38910514F08CE833
:10A4C00090E09093AC058093AB050E948A620C9457
:10A4D0001C488091FB0A83FF02C00C941C4889E44D
:10A4E0000E947A30882311F40C942D5C0E9456301F
:10A4F00090E01816190614F481E090E026E0289FF9
:10A50000F001299FF00D1124E255FA4F82819381C9
:10A510001CAA8C38910514F08CE890E09093AC055F
:10A520008093AB050E948A622091AB053091AC0507
:10A530008091A9059091AA05821793070CF03BC161
:10A5400088E996E060E00E94971F81E080935201C5
:10A550001DAA1EAA1FAA18AE1BAE1CAE1DAE1EAEB3
:10A5600021961FAE21979CE322969FAF2297ACE1E4
:10A570002496AFAF2497B6E42896BFAF2897312C26
:10A58000212CE0E8ECA7FFEBF8AB18A621E02FAFF9
:10A59000812C912C54010091AB051091AC05B801B0
:10A5A000012E000C880B990B0E9423E26B017C01A9
:10A5B000232D322D4CA558A90E941CE2882389F036
:10A5C0008091A9059091AA053CA93111F7C041E0FD
:10A5D00048A7081719070CF018A63C2C2D2CECA640
:10A5E000F8AA0E94A2C16B017C01DC01CB012BAD5A
:10A5F0003CAD4DAD5EAD821B930BA40BB50BB7FD0F
:10A600002FC0D701C60188519C4FAF4FBF4F8BAFB2
:10A610009CAFADAFBEAF80E00E94537185E896E07D
:10A620000E94A23981149104A104B10409F4DBC091
:10A63000C501B40168577C4E8F4F9F4F6C197D093F
:10A640008E099F0928EE33E040E050E00E9464E864
:10A65000CA01B9014AE00E94FA3B8AE00E948A39A5
:10A660000E9433400E94A2C16093E8057093E905FF
:10A670008093EA059093EB056091A9057091AA0576
:10A68000072E000C880B990B0E9423E269AF7AAF6A
:10A690008C019B01AC01632D722D8CA598A90E94A1
:10A6A00012E92B013C0120E030E0A9010E9496EA6A
:10A6B00087FF04C077FA709477F87094811491043E
:10A6C000A104B10409F093C020E030E040E85FE36A
:10A6D000C301B2010E941CE287FF10C09FADA2E837
:10A6E0008A2EA6E09A2EA12CB12C911103C0812CA8
:10A6F000912C54018C0C9D1CAE1CBF1CA8A5AA2338
:10A7000009F442C02DA93EA94FA958AD2115310524
:10A710004105510541F0D701C601821B930BA40BE3
:10A72000B50BB7FD31C029AD3AADA80121966FAD8B
:10A73000219722967FAD229724968FAD2497289655
:10A740009FAD28970E9412E920E030E040E85FE3E7
:10A750000E941CE287FD35C0D701C601805A954191
:10A76000AF4FBF4F8DAB9EABAFABB8AF99AD21969E
:10A770009FAF2197AAAD2296AFAF229724960FAF35
:10A78000249728961FAF2897809152018823C9F0FB
:10A7900081149104A104B10461F0B8E8CB1AB3E1CB
:10A7A000DB0AE108F108C818D908EA08FB08F7FE37
:10A7B00008C01FAEF0CE89E896E0C4CE081719078E
:10A7C00064F480915201882311F40C941C48109277
:10A7D00052010E94D7BA0C941C483C2C2D2CECA69C
:10A7E000F8AA18A6FECE8FE30E948A3936CF20E061
:10A7F00030E040E450E4C301B2010E9496EA18162A
:10A800000CF07CCF4601570179CF0E9400720E9464
:10A81000CE770E94CB901092370668EE73E080E00E
:10A8200090E00E94C83360E087EA96E00E94971F9C
:10A830000C941C48809140038F7D8061809340037D
:10A840000C941C48809140038F7E8062809340036B
:10A850000C941C4883E50E947A308823F1F00E9412
:10A86000A2C16093E8057093E9058093EA0590938F
:10A87000EB050E949A1C20E030E04AE754E40E9475
:10A8800082E20E940FEA60930B0170930C018093A7
:10A890000D0190930E010C941C488BE092E00E94F5
:10A8A000211C882339F10E94BE7788E50E94451C4F
:10A8B000882331F05E9A809194058E7F8093940571
:10A8C00089E50E94451C882331F05E9A80919405A9
:10A8D0008D7F809394058AE50E94451C882311F49E
:10A8E0000C941C48159A809194058B7F8093940555
:10A8F0000C941C480E94CE770C941C480E946B3A22
:10A9000087FF02C00C941C488BE092E00E94211C3F
:10A91000882309F48BC0EAE6CE2EE1E0DE2EFCEFC0
:10A92000EF2EFAE0FF2E10E0F60181916F010E94F8
:10A930007A30882309F465C0133009F06DC00E9495
:10A940009A1C4B015C0120E030E040EA51E40E9497
:10A950001CE287FF4EC0A501940160911C0B709111
:10A960001D0B80911E0B90911F0B0E9496E92B01ED
:10A970003C01AC019B0160911B0670911C0680910B
:10A980001D0690911E060E9482E260931B06709342
:10A990001C0680931D0690931E06A30192016091F0
:10A9A0002C0B70912D0B80912E0B90912F0B0E94F0
:10A9B00082E260932C0B70932D0B80932E0B90935F
:10A9C0002F0B60912B0670912C0680912D06909193
:10A9D0002E060E9421E2A30192010E9482E20E94BF
:10A9E0000FEA60932B0670932C0680932D069093AC
:10A9F0002E0680921C0B90921D0BA0921E0BB09203
:10AA00001F0B1F5FB4E0EB0EF11C143009F08CCF6C
:10AA10000E949A770C941C480E949A1CD701549665
:10AA20006D937D938D939C935797EBCF81E00E941C
:10AA30009CBA0C941C480E9437BA80E295E10E94AF
:10AA4000DA730C941C488091410390914203009763
:10AA500041F0FC012081222321F00E9479B80C945E
:10AA60001C480E94D7BA0C941C48009141031091D5
:10AA7000420394E0F12C40E0915009F1D8018C910F
:10AA8000282F2B7F2134A1F411962C912133B9F476
:10AA9000813419F1853409F441E098012E5F3F4F6C
:10AAA00089012F5F3F4FD8018C918032C9F3E4CFE9
:10AAB000803529F4F801818180538A3070F3411187
:10AAC0000E94673AFF2021F08CEB97E00E94A239A8
:10AAD000C8010E9491390C941C48FF24F394DDCFE7
:10AAE0000E94168F0C941C4881E0809392058093FD
:10AAF00091050E94318F0C941C481092920510927F
:10AB000091050E94318F0C941C4890E080E00C94D9
:10AB1000D84C0E94633A8FEB97E00E94A2390C94C4
:10AB20001C488AEA90E00C94EF4C8CE291E00C9483
:10AB3000EF4C85E090E00C940D4D8CE890E00C9487
:10AB40000D4D90E080E00C942D4D8FEF90E00C9433
:10AB50002D4D80E00C94724D0E946B3A87FF02C02D
:10AB60000C941C480AE611E06CEFE62E6AE0F62E23
:10AB70007EE6C72E71E0D72ED8018D918D010E94FF
:10AB8000451C882359F00E949A1C0E940FEAF70185
:10AB900060837183828393830E944C77F4E0EF0E8D
:10ABA000F11CC016D10641F70C941C480E946B3A68
:10ABB00087FF02C00C941C485AE6E52E51E0F52EA2
:10ABC00010E000E0D7018D917D010E94451C882393
:10ABD00049F00E949A1CF801E450F54F64A375A354
:10ABE00086A397A30C5F1F4F0031110559F70C94F2
:10ABF0001C4883E50E947A30882391F00E949A1CB9
:10AC00006093300B7093310B8093320B9093330B26
:10AC10006093380B7093390B80933A0B90933B0BF6
:10AC200080E50E947A30882351F00E949A1C60933C
:10AC3000300B7093310B8093320B9093330B82E582
:10AC40000E947A30882351F00E949A1C6093340B42
:10AC50007093350B8093360B9093370B84E50E94ED
:10AC60007A30882311F40C941C480E949A1C60933B
:10AC7000380B7093390B80933A0B90933B0B0C94E9
:10AC80001C4888E092E00E94211C882311F40C9457
:10AC90001C4882E40E94451C882351F00E94761CC7
:10ACA00060930C0B70930D0B80930E0B90930F0B16
:10ACB00083E50E94451C882351F00E949A1C6093F2
:10ACC0003C0B70933D0B80933E0B90933F0B84E5C0
:10ACD0000E94451C882351F00E949A1C6093400BEF
:10ACE0007093410B8093420B9093430B88E50E9435
:10ACF000451C882351F00E949A1C60930F067093A4
:10AD00001006809311069093120689E50E94451C57
:10AD1000882351F00E949A1C6093130670931406C6
:10AD200080931506909316068AE50E94451C882399
:10AD3000B1F00E949A1C60931706709318068093D6
:10AD4000190690931A062DEC3CEC4CEC5DE30E9446
:10AD50001CE2181624F084EF97E00E94A23985E4E3
:10AD60000E94451C882311F40C941C480E949A1CD4
:10AD700060931B0670931C0680931D0690931E061D
:10AD80000C941C4840900106509002066090030607
:10AD9000709004062091290130912A0140912B01E5
:10ADA00050912C01C301B2010E9413E968A779A751
:10ADB0008AA79BA78090050690900606A09007069C
:10ADC000B090080620912D0130912E0140912F0165
:10ADD00050913001C501B4010E9413E96CA77DA711
:10ADE0008EA79FA7C0900906D0900A06E0900B0698
:10ADF000F0900C06209131013091320140913301E5
:10AE000050913401C701B6010E9413E968AB79ABD8
:10AE10008AAB9BAB209135013091360140913701CF
:10AE200050913801C301B2010E9413E92B013C018A
:10AE30002091390130913A0140913B0150913C0100
:10AE4000C501B4010E9413E94B015C0120913D0151
:10AE500030913E0140913F0150914001C701B60140
:10AE60000E9413E96B017C010E94673A8FE398E02E
:10AE70000E94A23983E50E94451C882321F00E948C
:10AE80006A308093270180912701882309F43FC00D
:10AE900089EB98E00E94A23987E398E00E94A239EA
:10AEA00048A559A56AA57BA588E897E10E94483A7C
:10AEB0004CA55DA56EA57FA588E597E20E94483A5E
:10AEC00048A959A96AA97BA985E597E20E94483A51
:10AED00085E398E00E94A2398DE298E00E94A239B1
:10AEE000B301A20188E897E10E94483AB501A401A4
:10AEF00088E597E20E94483AB701A60185E597E206
:10AF00000E94483A8AE00E948A390C941C4885EBDA
:10AF100098E0C0CF82E40E94451C882341F08091D4
:10AF20001F01909120019093100180930F0182E501
:10AF30000E94451C882341F080910F0190911001DF
:10AF40009093200180931F0183E50E947A3088232B
:10AF500031F00E94961C9093200180931F01E09194
:10AF60004303F09144038081882311F40C941C481E
:10AF700060911F01709120018FE498E00E94593A7E
:10AF800085E20E948A398AE00E948A390C941C4822
:10AF90000E94673A85E40E948A3980E3800F0E940C
:10AFA0008A39F701EB5DFE4F6081718183E598E09E
:10AFB0000E94593A85E20E948A398AE00E948A39C1
:10AFC0000C941C488AE50E947A30882331F10E9453
:10AFD0009A1C20E030E040E050EC0E941CE287FD2B
:10AFE0003AC00E949A1C20E030E040E050E40E9409
:10AFF00096EA1816ACF10E949A1C2091180B309119
:10B00000190B40911A0B50911B0B0E9482E20E9477
:10B0100008EACB010E94DBC105C083E50E947A30BB
:10B020008111D5CF80E192E00E94211C81111DC0C9
:10B030000E94673A40916B0450916C0460916D04DA
:10B0400070916E048BE598E00E94483A8AE00E9475
:10B050008A390C941C4860E070E080E090ECCDCF21
:10B0600060E070E080E090E4C8CF82E50E94451C7B
:10B070008111DECF0C941C4885E40E9460BB8111D5
:10B0800074C080E50E94451C882351F00E949A1CE0
:10B090006093AA147093AB148093AC149093AD1486
:10B0A00089E40E94451C882381F00E949A1C2CEAA6
:10B0B00035EC47E25EE30E9482E26093AE14709347
:10B0C000AF148093B0149093B11484E40E94451C93
:10B0D000882381F00E949A1C2CEA35EC47E25EE35B
:10B0E0000E9496E96093B2147093B3148093B414E1
:10B0F0009093B5140E94673A4091AA145091AB14F2
:10B100006091AC147091AD1480E798E00E94483AC9
:10B110002CEA35EC47E25EE36091AE147091AF1417
:10B120008091B0149091B1140E9496E9AB01BC01DA
:10B130008CE698E00E94483A2CEA35EC47E25EE360
:10B140006091B2147091B3148091B4149091B514BD
:10B150000E9482E2AB01BC0188E698E00E94483A76
:10B160008AE00E948A390C941C480E94633A84E762
:10B1700098E00E94A2390C941C4883E50E94451C6B
:10B18000182F882369F00E94961C9C0190935D0102
:10B1900080935C0191E0232B09F090E090934806A6
:10B1A00080E50E94451C882361F020915C0130916C
:10B1B0005D01232B11F00E946A30809348060C94A5
:10B1C0001C4811110C941C480E94673A82EA98E0CE
:10B1D0000E94A23980914806882391F08AE898E07D
:10B1E0000E94A23960915C0170915D0181E998E053
:10B1F0000E94593A8DE898E00E94A2390C941C48AC
:10B2000086E898E0EDCF0E942C3C0C941C4883E526
:10B210000E94451C182F30900104882319F00E94C9
:10B220006A30382E2091440B3091450B4091460BEB
:10B230005091470B27962CAF3DAF4EAF5FAF27978E
:10B240004090480B5090490B60904A0B70904B0B0C
:10B2500080914C0B90914D0BA0914E0BB0914F0BE8
:10B260002B968CAF9DAFAEAFBFAF2B97112329F0BC
:10B27000311003C080E00E94BA3086E50E94451C70
:10B2800021968FAF21970E94DB30882309F4B8C044
:10B2900083E40E94451C882309F49FC00E949A1CE5
:10B2A0006B017C01A7E0B4E0B9ABA8ABB9A7A8A734
:10B2B000F5E0FCA71AAE1BAE28EC2FAF02EC1CAADF
:10B2C000212C38EC3DAB42E449AF88A599A52396E3
:10B2D0009FAF8EAF239715E02396AEADBFAD2397FA
:10B2E0008D909D90AD90BD902396BFAFAEAF23974C
:10B2F0002CA9322D4DA959ADC501B4010E941CE203
:10B3000087FF04C08CAA292CADAAB9AE2AAD3BADEB
:10B310004FAD502FC501B4010E9496EA181624F4CF
:10B320008AAE9BAEAFAE0B2D1150B1F6BCA5B1509D
:10B33000BCA7E8A5F9A57496F9A7E8A7B111C5CFF0
:10B340002AAD3BAD4FAD502F6CA9722D8DA999AD93
:10B350000E9413E920E030E040E05FE30E9482E2D7
:10B36000A70196010E9413E96B017C012DEB37E3E5
:10B3700046E855EB0E9496EA87FD0AC02DEB37E3BD
:10B3800046E855E3C701B6010E941CE218162CF5E9
:10B3900080E00E94BA3015E0A8A8B9A805E0D50160
:10B3A0006D917D918D919D915D014D01B4E08B1A60
:10B3B0009108A70196010E9412E9F401608371834C
:10B3C00082839383015059F7115028A939A92C5E23
:10B3D0003F4F39AB28AB1111DFCF21964FAD2197ED
:10B3E000442351F00E94DB30882331F089EE98E04D
:10B3F0000E94A2390E94C939832D0E94BA300DC023
:10B40000311005C021963FAD21973323A9F30E9447
:10B41000673A8FEF98E00E94A239332051F0809173
:10B420000104811106C00E94633A8AEC98E00E94F0
:10B43000A2390E94673A8CEB98E00E94A239809171
:10B440000104882309F43EC089EB98E00E94A239E8
:10B450008AE00E948A392091440B3091450B40913B
:10B46000460B5091470B27966CAD7DAD8EAD9FADD1
:10B4700027970E941CE281110C9496472091480B5B
:10B480003091490B40914A0B50914B0BC301B201D3
:10B490000E941CE281110C94964720914C0B309134
:10B4A0004D0B40914E0B50914F0B2B966CAD7DADDB
:10B4B0008EAD9FAD2B970E941CE281110C94964794
:10B4C0000C941C4885EB98E0C1CFC11003C00FEF6E
:10B4D0000C94A04E0E949A1C209101063091020605
:10B4E00040910306509104060E9412E920E030E0EA
:10B4F00040E252E40E9412E920E030E046E951E4E3
:10B500000E9413E92EE034E74AED5CE30E9482E2F8
:10B510000E9408EA062F653010F40C94A04ED7CF95
:10B52000F11003C01FEF0C94AF4E0E949A1C2091A3
:10B5300005063091060640910706509108060E94C4
:10B5400012E920E030E040E252E40E9412E920E0FB
:10B5500030E046E951E40E9413E92EE034E74AED79
:10B560005CE30E9482E20E9408EA162F653010F424
:10B570000C94AF4ED7CF07FD02C017FF08C00E9442
:10B58000633A8EE099E00E94A2390C941C480E9414
:10B590009A1CE02E000FFF08A12F110FBB0B20E01B
:10B5A00030E0A901BB2091F025E02E9DF0012F9DF8
:10B5B000F00D1124EA0FFB1FEE0FFF1FEE0FFF1F10
:10B5C000E95FFB4F2081318142815381E5E0EE9DAF
:10B5D0008001EF9D100D11240A0F1B1F000F111F7A
:10B5E000000F111F095F1B4F0E9413E9D8016D93D3
:10B5F0007D938D939C9313970C941C480E940BBBD6
:10B6000081110C941C489AE6C92E96E1D92EE4E4E7
:10B61000FBE0F9A7E8A79E012F5F3F4F19017901D1
:10B6200010E000E0F6016591759185919491A8A5CF
:10B63000B9A58D909D90AD90BD90B9A7A8A7A50183
:10B6400094010E9412E92B013C01F70140825182D2
:10B650006282738220E030E040EA51EC0E9496EA78
:10B6600087FD0AC020E030E040EA51E4C301B201A6
:10B670000E941CE2181684F4F801E550F94DE4919B
:10B680001E1654F4B7FAB094B7F8B094D7018D925F
:10B690009D92AD92BC921397F70181909190A190E9
:10B6A000B1907F0120E030E040EA51ECC501B401E7
:10B6B0000E9496EA87FD3FC020E030E040EA51E476
:10B6C000C501B4010E941CE21816ACF10F5F1F4FB8
:10B6D000F4E0CF0ED11C0330110509F0A3CF85E9AA
:10B6E000E82E85E0F82E10E0F10181919191A19171
:10B6F000B1911F01F70181939193A193B1937F01C0
:10B70000812F0E944B851F5F133071F70E94348E8A
:10B7100060E087E499E00E94971F63E972E084E6A5
:10B7200090E00E94BA946AEB72E084E690E00E9496
:10B73000BA940C941C480E94633A85E699E00E94F2
:10B74000A23961E087E599E00E94971F0E948D1D54
:10B7500068E270E088EC90E00E94BA940C941C4877
:10B760000E9478A60C941C480E943C8F0C941C48A4
:10B7700081E080936F040E946CA610926F0488236E
:10B7800011F40C941C480E94673A83E899E00E94E7
:10B79000A2390C941C4883FD02C00C941C480E94E2
:10B7A00018CC0C941C4881E08093A405109296124A
:10B7B00060E083E50E94953081110C941C480E9442
:10B7C000B3B80C941C480E944DD281110C941C48B3
:10B7D0000C94224F109145030E94A2C16093E8058A
:10B7E0007093E9058093EA059093EB05112311F41A
:10B7F0000C941C480E94673A84E50E948A39812F84
:10B800000E94B4C780E20E948A398EEA99E00E94C1
:10B81000A2390C941C4883E50E947A30882311F4E5
:10B820000C941C480E94961C0C94744C83E50E9456
:10B830007A30882311F40C94DF510E94861C8B010E
:10B840000C94DF5183E50E947A30882311F40C9424
:10B850001C480E94961C0C945C5283E50E947A302E
:10B860008CAB811107C082E50E947A30882311F4E5
:10B870000C941C480E94961C0C948952F1100C9454
:10B880004D4A90E1E4E4FBE0ADEEB3E001900D92AF
:10B890009A95E1F70C945B4A80E001110C942C47D7
:10B8A00080E1E4E4FBE0ADEEB3E001900D928A9517
:10B8B000E1F70C94814A4F925F926F927F928F9240
:10B8C0009F92AF92BF92CF92DF92EF92FF920F932F
:10B8D0001F93CF93DF93CDB7DEB77C014DB65EB635
:10B8E0006090F1057090F2058DB69EB66AE070E04A
:10B8F000C7010E945EE16C018C010E191F09892BA2
:10B9000021F4C7010E9469E18C01C80101962DB79D
:10B910003EB7281B390B0FB6F8943EBF0FBE2DBFA4
:10B920008DB79EB701965C01A801B7010E948AE11C
:10B93000F501E00FF11F1082C5010E94502F81E038
:10B940000E946746C114D10451F076019FEFE91AB5
:10B95000F90A0FB6F8949EBE0FBE8DBEC5CF0FB6C6
:10B96000F8949EBE0FBE8DBEC3010E94502F0FB62D
:10B97000F8945EBE0FBE4DBEDF91CF911F910F9127
:10B98000FF90EF90DF90CF90BF90AF909F908F90FF
:10B990007F906F905F904F9008954F925F926F925B
:10B9A0007F928F929F92AF92BF92CF92DF92EF924F
:10B9B000FF920F931F93CF93DF93CDB7DEB72897F6
:10B9C0000FB6F894DEBF0FBECDBF83E50E9460BB0B
:10B9D000863028F087E295E00E94A23949C0833082
:10B9E00009F46EC1E8F4813071F1823009F45AC073
:10B9F00084E195E00E94A2390E94DB308823F1F0B7
:10BA000080910104811117C085EB98E00E94A23952
:10BA10008AE00E948A390E94C9390E94348E28C067
:10BA2000843009F493C1853019F780E00E94BA3060
:10BA30000E94AA30F2CF89EB98E0E8CF86E095E04B
:10BA40000E94A239EACF0E94AA3010920A011092F5
:10BA500009018091D203811125C08EE40E94451C0A
:10BA600081111DC084EF94E09093A2058093A105FD
:10BA700028960FB6F894DEBF0FBECDBFDF91CF91F1
:10BA80001F910F91FF90EF90DF90CF90BF90AF90FC
:10BA90009F908F907F906F905F904F9008958AEF66
:10BAA00094E0E2CF8091090190910A0197FF03C0D1
:10BAB0008BEC94E091CF009709F0A8C01D821E8204
:10BAC0001F8218868DEC9CECACE4BEE389839A83DC
:10BAD000AB83BC83BE016B5F7F4FCE0101960E949A
:10BAE00054868091090190910A01893191050CF0E9
:10BAF000B3C021E0209328019C012F5F3F4F30937A
:10BB00000A012093090165E00E94ACE880FF03C0B0
:10BB100024E0291B922F24E09202F0011124E75621
:10BB2000FA4E80809180A280B38094E08902F00177
:10BB30001124EB57FA4E40805180628073808DEC67
:10BB40009CECACE4BEE38D839E83AF83B8871982FF
:10BB50001A821B821C82CE0101966C01E12CF12C11
:10BB600000EA10E4A3019201C501B4010E949C8582
:10BB700019821A821B821C82B601CE0105960E9490
:10BB800054868092440B9092450BA092460BB09243
:10BB9000470B4092480B5092490B60924A0B7092AF
:10BBA0004B0B1092D2030091090110910A0189E117
:10BBB000E82EF12C093111050CF47801B70184E667
:10BBC00094E00E94593A69E170E08FE594E00E94A8
:10BBD000593A8AE00E948A39101611060CF01DCFDE
:10BBE0001F9289E18F93FF92EF9288E494E09F93F4
:10BBF0008F9386E594E09F938F931F920E947E1F00
:10BC00000FB6F894DEBF0FBECDBF07CF815065E001
:10BC10000E94ACE880FF03C024E0291B922F25E09E
:10BC20009202F0011124E80FF11D87FDFA95EE0F45
:10BC3000FF1FEE0FFF1FE95FFB4F80914C0B9091B0
:10BC40004D0BA0914E0BB0914F0B80839183A2833B
:10BC5000B3831092280145CF80E090E0A0EAB0E4E1
:10BC600080934C0B90934D0BA0934E0BB0934F0BC6
:10BC700081E291E00E9481850E94BE778FEF9FEF65
:10BC800090930A018093090187EB94E00E94A23906
:10BC900085EA94E00E9479B863E972E084E690E076
:10BCA0000E94BA946AEB72E084E690E00E94BA9433
:10BCB0008FE994E00E945B5C81E00E94BA3071CF12
:10BCC00089E40E947A30882371F00E94961C182F14
:10BCD000853068F064E070E08CE894E00E94593AA6
:10BCE00089E894E079CE8AE40E94C339C1CE8AE41F
:10BCF0000E947A308823B9F30E94961C082F853061
:10BD000048F064E070E086E794E00E94593A83E7E7
:10BD100094E062CE8AE50E947A308823A9F00E94DE
:10BD20009A1C25E01202F0011124E00FF11D07FD1D
:10BD3000FA95EE0FFF1FEE0FFF1FE95FFB4F6083C9
:10BD400071838283938369CE8AE5CECF8AE50E9490
:10BD50007A308823C9F30E949A1C60936B04709315
:10BD60006C0480936D0490936E0457CECF93DF9351
:10BD7000C0913E0C81E6C89FE0011124C05CD34F06
:10BD80008091FB0A80FF05C00E94673ACE010E94A5
:10BD90009139CE010E94502F80E0DF91CF910C9419
:10BDA00067460F931F93CF93DF93CDB7DEB76097AE
:10BDB0000FB6F894DEBF0FBECDBF8C01DC01ED9154
:10BDC000FC910280F381E02DBE016F5F7F4F0995EA
:10BDD000882309F464C08981807CC9F56F81637010
:10BDE00070E0762F6627770F770F8885B4E08B9FFA
:10BDF000C0011124682B792B8985829586958695BB
:10BE00008370682B6F5F7F4F90E080E02A852370FE
:10BE1000220F3B8537FB332730F9232B3E813F70C0
:10BE2000230F3327331F2750310904C0660F771FB4
:10BE3000881F991F2A95D2F760960FB6F894DEBF37
:10BE40000FBECDBFDF91CF911F910F910895803428
:10BE500019F568856695669570E090E080E0CB0105
:10BE6000772766272A85622B098510E0102F002787
:10BE7000012E000C220B330B602B712B822B932B8A
:10BE80006F5F7F4F8F4F9F4F4AE0660F771F881F6E
:10BE9000991F4A95D1F7D0CF8BE0F801848360E0F9
:10BEA00070E0CB01C9CF0895FC0182810895CF9243
:10BEB000DF92EF92FF9280910604882309F457C025
:10BEC000C0900204D0900304E0900404F0900504B4
:10BED00020E030E0A901C701B6010E941CE28823DE
:10BEE00009F445C020E030E040E05FE3C701B6015F
:10BEF0000E9482E29B01AC010E9482E22BED3FE0B6
:10BF000049E450E40E9482E29B01AC0160E070E0F1
:10BF100080E89FE30E9496E96B017C01C092FD03DB
:10BF2000D092FE03E092FF03F0920004609125019D
:10BF300070912601072E000C880B990B0E9423E2BA
:10BF40002AE037ED43E25CE30E9482E2A70196011A
:10BF50000E9482E2609358017093590180935A01C4
:10BF600090935B01FF90EF90DF90CF900895C12CEC
:10BF7000D12C80E8E82E8FE3F82ED0CF2F923F927D
:10BF80004F925F926F927F928F929F92AF92BF92E9
:10BF9000CF92DF92EF92FF920F931F93CF93DF9395
:10BFA000CDB7DEB766970FB6F894DEBF0FBECDBF34
:10BFB000DC01CD90DD90ED90FC90139714962D91BF
:10BFC0003D914D915C9117972B873C874D875E87FC
:10BFD00020E030E040E252E4C701B6010E9412E9DD
:10BFE0002EE034E74AED5CE30E9482E20E9408EA18
:10BFF00064300CF428C163E0662E660F7708F30105
:10C00000EE0FFF1FEE0FFF1FE756FA4E8080918064
:10C01000A280B380F3013196FA83E98320E030E017
:10C0200040E252E46B857C858D859E850E9412E9F5
:10C030002EE034E74AED5CE30E9482E20E9408EAC7
:10C0400064300CF404C163E0062F660F110BF80195
:10C05000EE0FFF1FEE0FFF1FE756FA4E20813181D2
:10C06000428153812B833C834D835E83A8014F5FC4
:10C070005F4F5E8B4D8BA5E0A69DC001A79D900DE7
:10C080001124988B8F87FC01E00FF11FEE0FFF1F2B
:10C09000EE0FFF1FE95FFB4F208131814281538109
:10C0A0002F83388749875A87E981FA81EE0FFF1F6E
:10C0B000EE0FFF1FE756FA4EA501940160817181D2
:10C0C000828193810E9412E9698B7A8B8B8B9C8B86
:10C0D000A5019401C701B6010E9412E92B013C01A0
:10C0E00085E049815A81849F1001859F300C11247D
:10C0F000F101E00FF11FEE0FFF1FEE0FFF1FE95FD1
:10C10000FB4F2F81388549855A85608171818281F5
:10C1100093810E9412E929893A894B895C890E949E
:10C1200096E9A30192010E9482E22F813885498518
:10C130005A850E9413E96B017C01EF85F889AD896E
:10C14000BE89EA0FFB1FEE0FFF1FEE0FFF1FE95F17
:10C15000FB4F80809180A280B380FD01E20DF31D32
:10C16000EE0FFF1FEE0FFF1FE95FFB4FA5019401CC
:10C1700060817181828193810E9412E929893A89C3
:10C180004B895C890E9496E9A30192010E9482E298
:10C19000A50194010E9413E9A70196010E9412E9EA
:10C1A0004B015C01ED89FE89EE0FFF1FEE0FFF1FB3
:10C1B000E756FA4E2B813C814D815E816081718111
:10C1C000828193810E9412E99B01AC01C501B401F7
:10C1D0000E9496E94B015C012B813C814D815E817F
:10C1E0006B857C858D859E850E9412E99B01AC0143
:10C1F000C501B4010E9482E2A70196010E9413E9E1
:10C2000020916B0430916C0440916D0450916E0448
:10C210000E9413E966960FB6F894DEBF0FBECDBF3D
:10C22000DF91CF911F910F91FF90EF90DF90CF9012
:10C23000BF90AF909F908F907F906F905F904F9046
:10C240003F902F90089567FFD7CE60E0D5CE67FF6F
:10C25000FBCE60E0F9CE8F929F92AF92BF92CF92C9
:10C26000DF92EF92FF92FC01C080D180E280F380E8
:10C2700020E030E040E251E4C701B6010E9482E2D2
:10C2800020E030E040E251E40E9482E24B015C0198
:10C2900020E030E0A901C701B6010E941CE220E0C5
:10C2A00030E040EA50E487FF04C020E030E040EA9C
:10C2B00050ECC501B4010E9413E920E030E040E2F7
:10C2C00051E40E9496E90E9408EA9B018BE237FF45
:10C2D00005C022273327261B370B8DE28093D60318
:10C2E000C90168EE73E00E94CEE8CB01EAE0F0E01D
:10C2F000BF010E94CEE8805D8093D703C90164E648
:10C3000070E00E94CEE8CB01BF010E94CEE8805DC4
:10C310008093D803C901BF010E94CEE8282FCB012A
:10C32000BF010E94CEE8805D8093D9038EE28093A6
:10C33000DA03205D2093DB0386ED93E0FF90EF901E
:10C34000DF90CF90BF90AF909F908F90089524E69C
:10C35000829FC001112481589F4F6FEF70E00E94AF
:10C36000CEE8262F81E3643609F080E28093D8037B
:10C3700090E22A3040F03AE0822F632F0E94A0E83A
:10C380000E94A0E8905D9093D903822F6AE00E94FA
:10C39000A0E8905D9093DA0385E28093DB0388ED5B
:10C3A00093E008956091250170912601072E000CFD
:10C3B000880B990B0E9423E22AE037ED43E25CE30D
:10C3C0000E9482E22091FD033091FE034091FF0321
:10C3D000509100040E9482E26093580170935901C9
:10C3E00080935A0190935B0108958091E505811136
:10C3F00004C08091C0058093370608958091BB16D4
:10C400008823C1F081508093BB16EEEEF4E18823BF
:10C4100051F08150990B2BE1289FF001299FF00DDD
:10C420001124E355FA4E8BE1A3EDB4E101900D9296
:10C430008A95E1F72091BB16211105C08091C6169F
:10C4400080628093C61681E090E0A0E0B0E0211108
:10C4500003C080E090E0DC018093CE059093CF058F
:10C46000A093D005B093D1051092C70581E08093C9
:10C47000DE0583E0809353010895CF93DF93EC01B1
:10C48000CB01BA010E9423E220E030E0A9010E9422
:10C4900013E90E9408EA79836883DF91CF910895B8
:10C4A000CF93DF93EC01CB01BA010E9423E229EC88
:10C4B00038EC48EC5EE30E9496E920E030E040E092
:10C4C0005FE30E9413E90E940FEA6883DF91CF9136
:10C4D00008950E9423E229EC38EC48EC5EE30E94C8
:10C4E00096E920E030E040E05FE30E9413E90E941B
:10C4F0000FEA862F0C94A761E091E50586E0E8023B
:10C50000F0011124E255FA4F8091C00590E0958327
:10C51000848308952091AB053091AC052115310538
:10C52000E9F08091A9059091AA050296245031095D
:10C53000821793079CF49093100580930F050E9437
:10C54000A2C1605E70448D4F9F4F60931105709340
:10C550001205809313059093140508951092110508
:10C560001092120510921305109214050895CF939E
:10C57000DF93EC018D810E94E93B60E08B81DF91CC
:10C58000CF910C94ABC0DF92EF92FF920F931F9369
:10C59000CF93DF938C01C62FD22FF32EE42ED52E0E
:10C5A0000E94B7620E9421C28C2F80640E94DD3BF2
:10C5B0008D2D0E94DD3B8E2D0E94DD3B8F2D0E9434
:10C5C000DD3B8D2F0E94DD3B87E8C11101C085E96D
:10C5D0000E94DD3BCC3011F40E94E23BC0E00E949F
:10C5E000E23BF801868387FF04C0CF3F11F0CF5FA5
:10C5F000F6CFDF91CF911F910F91FF90EF90DF90D9
:10C60000089561E0FC0183810E94ABC08FEF0C9420
:10C61000DD3B0F931F93CF938C010E94B7620E9462
:10C6200021C2C82F882371F08DEF0E94DD3B0E944C
:10C6300021C2C82FC8010E9401638C2FCF911F9186
:10C640000F91089582E1F8018483F4CF8F929F9235
:10C65000AF92BF92CF92DF92EF92FF920F931F9310
:10C66000CF93DF93EC016A017B01590120E030E0B8
:10C67000A90167E30E94C362A501980167E1CE01A9
:10C680000E94C362811127C08F81833039F089E015
:10C69000CC0CDD1CEE1CFF1C8A95D1F7A70196017E
:10C6A00069E1CE010E94C36211E0882319F010E015
:10C6B00087E08C83CE010E940163812FDF91CF91AF
:10C6C0001F910F91FF90EF90DF90CF90BF90AF90B0
:10C6D0009F908F90089589E08C8310E0EBCFCF93EB
:10C6E000DF93EC016EBDFA01CA019E5F0DB407FE37
:10C6F000FDCF20812EBD0DB407FEFDCF21812EBDC3
:10C700003296E817F90791F70DB407FEFDCF8FEFCA
:10C710000E94DD3B8FEF0E94DD3B0E94E23B8E8357
:10C720008F71853049F083E18C83CE010E940163D3
:10C7300080E0DF91CF91089581E0FBCF0F931F93AD
:10C74000CF93DF93EC018B010E94B7620E9421C25C
:10C7500081110CC085E18C8310E0CE010E94016341
:10C76000812FDF91CF911F910F910895A8016CEF58
:10C77000CE010E946F63182F882361F3EECF0F93D1
:10C780001F93CF93DF93EC0189018F81833039F0C0
:10C7900089E0440F551F661F771F8A95D1F79A01CC
:10C7A000AB0168E1CE010E94C36281112AC0A801D9
:10C7B0006EEFCE010E946F63182F8823B1F00E94A4
:10C7C00021C2182F8823D1F020E030E0A9016DE0CC
:10C7D000CE010E94C362882321F086E18C8310E0A1
:10C7E00004C00E94E23B8111F8CFCE010E94016398
:10C7F000812FDF91CF911F910F91089587E18C8355
:10C80000F4CF86E0EBCF1F93CF93DF93EC010E9430
:10C81000B76220E030E0A9016CE0CE010E94C36263
:10C8200011E0882319F010E083E08C83CE010E9490
:10C830000163812FDF91CF911F9108951F93CF93B3
:10C84000DF93EC018F81833039F089E0440F551F6D
:10C85000661F771F8A95D1F79A01AB0162E1CE017D
:10C860000E94C36211E0882319F010E085E08C83F8
:10C87000CE010E940163812FDF91CF911F91089516
:10C880008F929F92AF92BF92EF92FF920F931F935E
:10C89000CF93DF938C01EB017A010E94A2C14B017F
:10C8A0005C012CE2820E21E0921EA11CB11C0E94B0
:10C8B000E23BF80186838F3F69F40E94A2C16819A8
:10C8C00079098A099B0997FDF2CF81E1F8018483F8
:10C8D000C0E021C08E3F71F5F1E0EF1AF1088FEF53
:10C8E0008EBDFE012FEF0DB407FEFDCF8EB58193F7
:10C8F0002EBDCF018C1B9D0B8E159F05A0F30DB493
:10C9000007FEFDCF8EB5CE0DDF1D88830E94E23B72
:10C910000E94E23BC1E0C8010E9401638C2FDF91BD
:10C92000CF911F910F91FF90EF90BF90AF909F908C
:10C930008F9008958FE0CACF0F931F93CF93DF930B
:10C94000EC018B010E94B76240E052E0B801CE01D9
:10C95000DF91CF911F910F910C9440640F931F931F
:10C96000CF93DF93EC0189018F81833039F089E027
:10C97000440F551F661F771F8A95D1F79A01AB01A7
:10C9800061E1CE010E94C36281110AC040E052E021
:10C99000B801CE01DF91CF911F910F910C944064AB
:10C9A00084E08C83CE010E94016380E0DF91CF910F
:10C9B0001F910F9108958F929F92AF92BF92CF9245
:10C9C000DF92EF92FF920F931F93CF93DF93EC01CF
:10C9D000162F1F821C824B830E94A2C16B017C0117
:10C9E00020EDC20E27E0D21EE11CF11CA89561E0EB
:10C9F0008B810E94ABC08B810E945AB8249A2C9ADA
:10CA0000279A2698259A81E00E94E93B85E08D834C
:10CA10000E94E93B0AE08FEF0E94DD3B0150D9F70D
:10CA2000A89520E030E0A90160E0CE010E94C36239
:10CA30008E83813081F00E94A2C16C197D098E091C
:10CA40009F0997FDEECF81E08C83CE010E940163A8
:10CA50001A8280E06AC0A8952AEA31E040E050E0FE
:10CA600068E0CE010E94C362853041F581E08F838A
:10CA7000A8958F81812C912C5401823029F4812C2E
:10CA8000912CA12C80E4B82E20E030E0A90167E3CE
:10CA9000CE010E94C362A501940169E2CE010E9409
:10CAA000C3628E838823F1F00E94A2C16C197D09B4
:10CAB0008E099F0997FDE8CF8AE0C6CF04E00E9467
:10CAC000E23B8E830150D9F78A3A11F482E0CFCF4E
:10CAD0000E94A2C16C197D098E099F0997FDBCCFE8
:10CAE00082E0B2CF8F818230C1F420E030E0A90132
:10CAF0006AE3CE010E94C362882311F088E0A4CFCC
:10CB00000E94E23B807C803C11F483E08F830E9492
:10CB1000E23B0E94E23B0E94E23BCE010E940163A5
:10CB200081E08A83173070F41D83DF91CF911F91CC
:10CB30000F91FF90EF90DF90CF90BF90AF909F90BC
:10CB40008F90089588E18C8384CF0F931F93CF93A8
:10CB5000DF93EC018B0120E030E0A90169E00E9445
:10CB6000C36281110AC040E150E0B801CE01DF91FB
:10CB7000CF911F910F910C94406480E18C83CE0182
:10CB80000E94016380E0DF91CF911F910F91089582
:10CB9000CF93C82FCB010E94A23981E096E10E9479
:10CBA000A23982EF95E1CC2311F087EF95E10E9445
:10CBB000A2398AE0CF910C948A390C94AEC10C94BE
:10CBC000AEC140916F0421E042276CE070E00C940C
:10CBD00001BA40916F0421E0422764E070E00C94B8
:10CBE00001BA40916F0421E0422761E070E00C94AB
:10CBF00001BA40916F0421E0422762E070E00C949A
:10CC000001BA40916F0421E0422761E070E00C948A
:10CC100001BA40916F0421E0422768E070E00C9473
:10CC200001BA40916F0421E042276CE070E00C945F
:10CC300001BA41E061E070E00C9401BA40916F04E8
:10CC400021E042270C9401BA62E070E00C943AC1F2
:10CC50006CE070E00C943AC164E070E00C943AC16E
:10CC600061E070E00C943AC161E070E00C943AC16C
:10CC70006CE070E00C943AC10F931F93CF93811135
:10CC800013C0C42F8B010E94673A8FEE96E10E9479
:10CC9000A239C8010E94A239CC2331F08AE0CF9199
:10CCA0001F910F910C948A39CF911F910F91089584
:10CCB000CF93DF9380911E1590911F15891B80954E
:10CCC0008F7019F40E943340F5CF80911E158F5F4D
:10CCD0008F70A0911E159BE4A99FD0011124FD0126
:10CCE000E55BF94FEF0119929A95E9F798E0908387
:10CCF000A05AB94F90E1E0E2F5E101900D929A95CA
:10CD0000E1F720911E1590911F15291303C094E699
:10CD100090931B1580931E15DF91CF910C940331D6
:10CD200020E040E070E060E088E597E60E94D21CD9
:10CD300081E08093C6051092EF051092EE050895EC
:10CD400020E040E070E060E08EE699E60C94D21CB2
:10CD500080914806811114C080915C0190915D0121
:10CD600001972091A5143091A6142817390744F48F
:10CD700020E040E070E060E083E799E60C94D21C8C
:10CD80000C94A06621E02093C605FC01808191816E
:10CD9000A281B38180931B0190931C01A0931D017C
:10CDA000B0931E0120E040E070E060E08091BE059D
:10CDB0009091BF050C94D21CCF93DF9300D000D08C
:10CDC000CDB7DEB78DEC9CECACECBCE389839A83E9
:10CDD000AB83BC83CE0101960E94C2660F900F9078
:10CDE0000F900F90DF91CF910895CF93DF9300D0F4
:10CDF00000D0CDB7DEB78DEC9CECACECBDE3898305
:10CE00009A83AB83BC83CE0101960E94C2660F90C9
:10CE10000F900F900F90DF91CF910895CF93DF93F4
:10CE200000D000D0CDB7DEB780E090E0A0E8BFE34F
:10CE300089839A83AB83BC83CE0101960E94C2662C
:10CE40000F900F900F900F90DF91CF910895CF9397
:10CE5000DF9300D000D0CDB7DEB780E090E0A0E255
:10CE6000B1E489839A83AB83BC83CE0101960E948F
:10CE7000C2660F900F900F900F90DF91CF910895A1
:10CE800081E08093C6051092940510927E0420E004
:10CE900040E070E060E089E09CE60E94D21C8CE4F7
:10CEA00095E19093A2058093A10508950C94A61D89
:10CEB0008F929F92AF92BF92CF92DF92EF92FF92AA
:10CEC000CF938091C4051092C405882369F0109215
:10CED000C605CF91FF90EF90DF90CF90BF90AF90BD
:10CEE0009F908F900C94A61D4091CE055091CF0538
:10CEF0006091D0057091D10541155105610571050D
:10CF000099F01092CE051092CF051092D005109294
:10CF1000D10581E0809353012AE0249FC001259F21
:10CF2000900D11240E94DBC180915301882309F4E4
:10CF3000AEC06091EE057091EF05072E000C880BD6
:10CF4000990B0E9423E220914006309141064091C6
:10CF50004206509143060E9482E26B017C0120E070
:10CF600030E040E251E40E9482E220E030E04AE713
:10CF700054E40E9482E24B015C0120E030E0A90110
:10CF8000C701B6010E941CE220E030E040EA50E414
:10CF900087FF04C020E030E040EA50ECC501B40156
:10CFA0000E9413E920E030E040E251E40E9496E95B
:10CFB0000E9408EA6B017C018BE2F7FE09C0F09445
:10CFC000E094D094C094C11CD11CE11CF11C8DE2F2
:10CFD0008093D503C701B60120E137E240E050E07D
:10CFE0000E94E2E88AE0882E912CA12CB12CCA0183
:10CFF000B901A50194010E94E2E8605D6093D60347
:10D00000C701B60128EE33E040E050E00E94E2E8BC
:10D01000CA01B901A50194010E94E2E8605D609334
:10D02000D7038EE28093D803C701B60124E630E02F
:10D0300040E050E00E94E2E8CA01B901A501940174
:10D040000E94E2E8605D6093D903C701B601A501C3
:10D0500094010E94E2E8C62FCA01B901A50194011A
:10D060000E94E2E8605D6093DA03C05DC093DB0379
:10D0700065ED73E08EEA95E1CF91FF90EF90DF9040
:10D08000CF90BF90AF909F908F900C94AC23CF9196
:10D09000FF90EF90DF90CF90BF90AF909F908F90D8
:10D0A00008956FEF8091C0050C9461C04F925F921C
:10D0B0006F927F928F929F92AF92BF92CF92DF92A8
:10D0C000EF92FF920F931F93CF93DF930091C005D0
:10D0D0000E94B5BDC091C70510E0000F111F035895
:10D0E0001A4E95E0592E5C0E23E6E22E25E1F22E33
:10D0F000D3E0DC1B31E5C32E38E6D32E45E5A42E64
:10D1000045E1B42E82E0782E7C1A5AE8852E55E14E
:10D11000952E81E0682E6C1A4C2E4194C11137C0B7
:10D120008091C9058823B1F080915301882359F07B
:10D1300081E09091C905911180E024E041E755E13B
:10D14000642D0E9489BCCF5F5C12E8CF84E080939D
:10D15000C8050CC08091C4051092C405882321F332
:10D160000E94A61D8091DE058823F1F2DF91CF9108
:10D170001F910F91FF90EF90DF90CF90BF90AF90F5
:10D180009F908F907F906F905F904F900895C130E7
:10D1900059F5F801859194919093E7058093E60500
:10D1A0008091C905813081F080915301882359F223
:10D1B0001F929F928F926F9281E09091C90591305A
:10D1C00009F474C080E072C08091C4051092C40557
:10D1D000882351F38091C005682F0E9461C080911F
:10D1E000DE05882309F3C2CFC23009F042C0F8013E
:10D1F000859194919093E7058093E6058091C90508
:10D200008230D1F080915301882309F49CCFDF92C2
:10D21000CF92BF92AF927F9281E09091C9059230F8
:10D2200009F080E08F930E94C41C0F900F900F9024
:10D230000F900F900F9087CF8091C4051092C40576
:10D24000882301F30E9451688091DE058823D1F282
:10D250008DCF8091C4051092C4058823C1F06091E0
:10D26000C0058FEF0E9461C08091DE05882379F0B0
:10D270007DCFC33009F067CFF801859194919093E9
:10D28000E7058093E6058091C905833011F380910D
:10D290005301882309F457CF1F92FF92EF92DF9337
:10D2A00081E09091C905933009F08CCF8F930E9453
:10D2B000C41C0F900F900F900F900F9044CF6EEE04
:10D2C0007BE682E00C948ED463EF7BE681E00C94E5
:10D2D0008ED468EF7BE680E00C948ED465EA79E624
:10D2E00083E00C948ED4EF92FF920F931F938AEFFA
:10D2F000E82E84E1F82E0CEF14E126E537E640EA4B
:10D3000056E66CE075E181E195E10E94C0C41F9191
:10D310000F91FF90EF900895EF92FF920F931F935C
:10D320008CE3E82E84E1F82E0FEA14E126E537E6D7
:10D330004EEF5FE16EE374E183E494E10E94C0C4C8
:10D340001F910F91FF90EF900895CF93DF9300D03E
:10D3500000D0CDB7DEB78091C4051092C4058823F4
:10D3600059F01092C6050E94A61D0F900F900F90C5
:10D370000F90DF91CF9108956091CE057091CF0508
:10D380008091D0059091D1056115710581059105B8
:10D3900061F10E9423E220911B0130911C01409118
:10D3A0001D0150911E010E9482E22091500B30918C
:10D3B000510B4091520B5091530B0E9413E9609313
:10D3C000500B7093510B8093520B9093530B83E04F
:10D3D0000E94632081E0809353011092CE05109249
:10D3E000CF051092D0051092D1058091530188236A
:10D3F00009F4BBCF2091BA053091BB054091BC0523
:10D400005091BD056091500B7091510B8091520B62
:10D410009091530B0E9412E969837A838B839C83DA
:10D42000CE0101960E942B61BC018CEC96E20E9419
:10D43000AC239BCF2F923F924F925F926F927F923D
:10D440008F929F92AF92BF92CF92DF92EF92FF9214
:10D450001F93CF93DF93CDB7DEB72C970FB6F89419
:10D46000DEBF0FBECDBF1C01162F8091C4051092E8
:10D47000C4058823E1F01092C6050E94A61D2C96D3
:10D480000FB6F894DEBF0FBECDBFDF91CF911F91D5
:10D49000FF90EF90DF90CF90BF90AF909F908F90D4
:10D4A0007F906F905F904F903F902F900895809164
:10D4B000CE059091CF05A091D005B091D1058D8377
:10D4C0009E83AF83B887892B8A2B8B2B09F460C08E
:10D4D00080912701882309F4BDC080912801811122
:10D4E000B9C0613009F494C0623009F4A2C08090E0
:10D4F000290190902A01A0902B01B0902C01C0909E
:10D500003501D0903601E0903701F0903801612E5E
:10D51000712C6D817E818F8198850E9423E22091FC
:10D520001B0130911C0140911D0150911E010E9470
:10D5300082E2D301AA0FBB1FAA0FBB1FBC87AB8718
:10D54000AC5BB44FBA87A9872D913D914D915C9109
:10D550000E9413E92B013C018D819E81AF81B8852A
:10D56000B7FF8FC0A5019401C301B2010E941CE264
:10D5700087FD7FC0EB85FC85EC5BF44F40825182D8
:10D5800062827382812F0E94632081E08093530125
:10D590001092CE051092CF051092D0051092D105B1
:10D5A00080915301882309F46ACFF4E01F9FC001E2
:10D5B0001124FC01EC5BF44F8F5F994FDC012D913E
:10D5C0003D914D915C9160817181828193810E9436
:10D5D00013E96B017C01C982DA82EB82FC822DECBB
:10D5E0003CEC4CEC5DE360911B0170911C0180915F
:10D5F0001D0190911E010E9496EA87FD52C0CE0146
:10D6000001960E942B61BC01C1010E94AC2337CF5F
:10D6100080902D0190902E01A0902F01B0903001AC
:10D62000C0903901D0903A01E0903B01F0903C016C
:10D630006ECF8090310190903201A0903301B09074
:10D640003401C0903D01D0903E01E0903F01F09048
:10D6500040015DCF812C30E5932E33ECA32E37ECC7
:10D66000B32EC12C40E5D42E43ECE42E47E4F42E37
:10D670004ECFA985BA858D929D92AD92BC9213979B
:10D6800081CFA7019601C301B2010E9496EA181644
:10D690000CF070CFE985FA85C082D182E282F382F4
:10D6A00071CF20E030E040E251E4C701B6010E94B2
:10D6B00082E220E030E04AE754E40E9482E24B013B
:10D6C0005C0120E030E0A901C701B6010E941CE224
:10D6D00020E030E040EA50E487FF04C020E030E082
:10D6E00040EA50ECC501B4010E9413E920E030E0AB
:10D6F00040E251E40E9496E90E9408EA6B017C0135
:10D70000F7FC62C020EA36E841E050E00E94E2E81F
:10D71000CA01B9012AE030E040E050E00E94E2E8AE
:10D72000605D6093D503C701B60120E137E240E0B8
:10D7300050E00E94E2E88AE0882E912CA12CB12CC6
:10D74000CA01B901A50194010E94E2E8605D6093FD
:10D75000D603C701B60128EE33E040E050E00E9456
:10D76000E2E8CA01B901A50194010E94E2E8605D06
:10D770006093D7038EE28093D803C701B60124E6F5
:10D7800030E040E050E00E94E2E8CA01B901A501A2
:10D7900094010E94E2E8605D6093D903C701B6017D
:10D7A000A50194010E94E2E8162FCA01B901A50162
:10D7B00094010E94E2E8605D6093DA03105D1093CB
:10D7C000DB0385ED93E01FCFF094E094D094C094F8
:10D7D000C11CD11CE11CF11C6DE2A3CF62E085ED00
:10D7E00096E20C941A6A61E08CED96E20C941A6A47
:10D7F00060E083EE96E20C941A6A6DE372E683EBC6
:10D8000092E90C94EC2460E572E689E692E60C94C9
:10D81000EC2480915301882331F041E062E773E109
:10D8200082E00E942CBC80917E048770873041F496
:10D8300020E040E070E060E08FE890EA0C94D21CB9
:10D8400008950F931F93CF93DF93CDB7DEB72A9739
:10D850000FB6F894DEBF0FBECDBF80915301882371
:10D86000F1F01F9289E18F938091D30390E00196AC
:10D870009F938F938FE493E19F938F938E010F5F1C
:10D880001F4F1F930F930E94B3E1B80184E493E10B
:10D890000E94AC230FB6F894DEBF0FBECDBF84E06C
:10D8A000809353018091D203811108C020E040E0B1
:10D8B00070E060E08BE294E20E94D21C2A960FB6E0
:10D8C000F894DEBF0FBECDBFDF91CF911F910F91B6
:10D8D0000895CF93DF93EC010E94E3CB1B82DF918D
:10D8E000CF910895CF93DF93EC01462F41706C8563
:10D8F0007D858E859F850E94B0C8882351F08889D8
:10D9000020E2829FC001112489569D4EDF91CF9164
:10D91000089590E080E0FACFCF93DF93EB01FC0114
:10D920002381211104C080E0DF91CF91089522501E
:10D93000223028F48FE28883198281E0F5CF60E0FD
:10D940000E94726C009779F3DC0160E080E09EE257
:10D950002D91203299F0883031F49E01260F311D2F
:10D96000F90190836F5F9E01260F311DAD0141507B
:10D970005109FA014081F90140836F5F8F5F8B305D
:10D9800039F7FE01E60FF11D1082D7CF3F924F927B
:10D990005F926F927F928F929F92AF92BF92CF923F
:10D9A000DF92EF92FF920F931F93CF93DF93CDB748
:10D9B000DEB72C970FB6F894DEBF0FBECDBF5C016B
:10D9C000DC0159968D909C90F40181859285A38508
:10D9D000B4859C01AD012F5F3F4F4F4F5F4F2987AB
:10D9E0003A874B875C87D50114964D905D906D907A
:10D9F0007C901797411451046104710409F459C0D3
:10DA0000BFEF4B1A5B0A6B0A7B0A312C7301620170
:10DA10001D821E821F821886F40181859285A3854E
:10DA2000B4852D813E814F815885281739074A07D3
:10DA30005B0708F056C089859A85AB85BC858C1537
:10DA40009D05AE05BF0550F482E0C82ED12CE12C17
:10DA5000F12C92E0492E512C612C712C9E012F5FEC
:10DA60003F4FB701A601C4010E94EACA8823C9F149
:10DA700089819A81AB81BC81892B8A2B8B2B01F107
:10DA8000260137019FEF491A590A690A790A2D813F
:10DA90003E814F8158852F5F3F4F4F4F5F4F2D8302
:10DAA0003E834F8358873FEFC31AD30AE30AF30A32
:10DAB000B3CF408051806280738033243394A6CFEB
:10DAC000C414D504E604F70411F70FEF1FEF2FEF8E
:10DAD0003FE0B701A601C4010E9458CA782E811107
:10DAE0001AC0712C872D2C960FB6F894DEBF0FBE8E
:10DAF000CDBFDF91CF911F910F91FF90EF90DF90FD
:10DB0000CF90BF90AF909F908F907F906F905F90DD
:10DB10004F903F900895F50144815581668177814A
:10DB2000411551056105710539F097018601C40160
:10DB30000E9458CA8823A9F2D5011496CD92DD928D
:10DB4000ED92FC921797332051F0D701C601019650
:10DB5000A11DB11DF40180839183A283B383F501DC
:10DB600085899689A789B08D892B8A2B8B2B09F003
:10DB7000B9CFC58AD68AE78AF08E81818068818391
:10DB8000B1CF40E050E0BA010C9432CCFC012381CB
:10DB900021110C94696C08952F923F924F925F92DD
:10DBA0006F927F928F929F92AF92BF92CF92DF92AD
:10DBB000EF92FF920F931F93CF93DF93CDB7DEB712
:10DBC000C354D1090FB6F894DEBF0FBECDBF4C01D0
:10DBD0005B016A01222E19821C821C8E1F8E611528
:10DBE000710521F510E0CE014C960E94C66DCE0164
:10DBF00001960E94C66D812FCD5BDF4F0FB6F89462
:10DC0000DEBF0FBECDBFDF91CF911F910F91FF906F
:10DC1000EF90DF90CF90BF90AF909F908F907F90CC
:10DC20006F905F904F903F902F900895FC018381FB
:10DC30008111D8CFFA0180818F32A1F18B01CE0101
:10DC400001967C013C0180E2382E2E019CE1490EB8
:10DC5000511C2396EFAE23972496FFAE249722966D
:10DC60003FAE229721963FAE21973FAE3EAE3DAEEE
:10DC70003CAE3BAE3AAE39AE38AE3FAA960190E02C
:10DC800047E0D9018D91882309F447C08F3209F408
:10DC900044C08E3209F54A3009F4A4CF98E04AE036
:10DCA0009D01EFCFFB01838182508B01823060F0B8
:10DCB000618D728DCE014C960E94A2D18E01045EC0
:10DCC0001F4F882309F48ECFC6016C010196F6011F
:10DCD00020812F32D1F3B3CFECECF2E22491222356
:10DCE00021F031968213FACF7DCF491708F47ACF0D
:10DCF000813208F477CF8F3709F474CF3FE9380FBA
:10DD00003A3108F420EEE7E3F0E0EC0FFD1FE90FF5
:10DD1000F11D820F80839F5FC3CF8FA9803209F4EA
:10DD200061CF6901F90180812F5F3F4F8F32C9F3C5
:10DD3000882301F121E0AE01495C5F4FB801C701C2
:10DD40000E94C0D2882309F44DCF0A151B0519F093
:10DD5000C8010E94696C942D852D6E147F0431F0EA
:10DD600023969FAD239724968FAD24978701E92EA4
:10DD7000F82E75CF222DAE01495C5F4FB801C4016A
:10DD80000E94C0D2182F2FCF2F923F924F925F92B6
:10DD90006F927F928F929F92AF92BF92CF92DF92BB
:10DDA000EF92FF920F931F93CF93DF93CDB7DEB720
:10DDB000ED970FB6F894DEBF0FBECDBF8091CA05B8
:10DDC000882369F18091C61600E010E083FF23C02C
:10DDD00083ED94E10E94C16D8BE1E3EDF4E1DE019E
:10DDE000919601900D928A95E1F710E000E0BE0156
:10DDF0006F5F7F4FCE0181960E9453CE18163CF480
:10DE0000CE0101960E9436C8080F111DF0CFCE0139
:10DE100081960E94C66D00937304109374040E944F
:10DE2000B5BD1091C7051CAF85E0810F8DAF312EB8
:10DE300031948EEFC82E81E6D82E98EEA92E94E16B
:10DE4000B92E81E0782E711A2CEE822E24E1922ECA
:10DE5000111113C08091C905882391F1809153015C
:10DE6000882359F081E09091C905911180E024E068
:10DE700045EF54E1632D0E9489BC8091C61685FF51
:10DE800055C01130D9F48091C9058130F1F18091EC
:10DE90005301882309F45BC11F929F928F927F9256
:10DEA00081E09091C905913009F080E08F930E9444
:10DEB000C41C0F900F900F900F900F9082E066C0DF
:10DEC0008091C4051092C405882341F20E94A61DCA
:10DED0008091DE05882311F2ED960FB6F894DEBF2F
:10DEE0000FBECDBFDF91CF911F910F91FF90EF90AB
:10DEF000DF90CF90BF90AF909F908F907F906F906A
:10DF00005F904F903F902F9008958091C40510929C
:10DF1000C405882309F4BBCF1092C7050E94F2D133
:10DF20008091DE05882309F4B2CFD6CF83FF2DC0C0
:10DF3000113021F68091C9058130D1F080915301D3
:10DF4000882309F404C1DF92CF92BF92AF927F92EF
:10DF500081E09091C905913009F080E08F930E9493
:10DF6000C41C0F900F900F900F900F900F90A6CFA2
:10DF70008091C4051092C405882301F30E94FE61BC
:10DF80008091DE058823D1F2A7CF81E090915301E3
:10DF9000992309F4DDC0582E082FF12CE12C412ED5
:10DFA0009CAD491A802F2091730430917404E216BD
:10DFB000F30608F0CDC00113A5C083ED94E10E94E3
:10DFC000C16D202E25188BE1E3EDF4E1DE01919681
:10DFD00001900D928A95E1F7612CBE016F5F7F4F32
:10DFE000CE0181960E9453CE18167CF4CE01019684
:10DFF0000E9436C8882389F326106BC0BE016F5F6C
:10E000007F4F83EF95E00E9451C8CE0181960E9418
:10E01000C66D8091C6169091C90584FF78C0911392
:10E0200066C08091C4051092C405882309F45FC0BE
:10E0300019821C828091D6146EEE74E1882311F04F
:10E0400063ED74E121E043EF55E0CE0101960E94BB
:10E05000CC6D882309F43FC08BE1FE013196A3ED1E
:10E06000B4E101900D928A95E1F78091C6168F7DFB
:10E070008093C616A091BB16AA3080F481E08A0F67
:10E080008093BB168BE18A9FD0011124A355BA4E11
:10E09000E3EDF4E101900D928A95E1F7CE0101964E
:10E0A0000E94C66D1092C70582E090E0A0E0B0E04B
:10E0B0008093CE059093CF05A093D005B093D10562
:10E0C00081E08093DE051092D40383E080935301B6
:10E0D00003CF639482CF0E94673A63EF75E082EDCD
:10E0E00094E10E9429408AE00E948A39D7CF80912A
:10E0F0005301882339F081E0911380E041E0642DE1
:10E100000E94CABC8FEFE81AF80A0F5F4BCF911735
:10E1100059F0809153018823A9F381E09091C905BA
:10E12000911380E040E0EBCF8091C4051092C405CC
:10E13000882379F383EF95E00E94D8C70E948D1D54
:10E140000E94D7BA8091DE05882319F3C5CE82E0FC
:10E150001F5F9DAD91137CCE8093C805BDCE8F927D
:10E160009F92AF92BF92CF92DF92EF92FF92CF93A6
:10E170006B017C01B42E20E030E0A9010E941CE27A
:10E1800087FF07C08DE20E948A39F7FAF094F7F80A
:10E19000F094C0E060E070E080E09FE3CB1541F0D8
:10E1A0002DEC3CEC4CEC5DE30E9482E2CF5FF6CFBD
:10E1B000A70196010E9413E96B017C010E940FEAFE
:10E1C0004B015C014AE00E944DC7CC2379F1C501A7
:10E1D000B4010E9421E29B01AC01C701B6010E947B
:10E1E00012E96B017C018EE20E948A39C150F0F085
:10E1F00020E030E040E251E4C701B6010E9482E233
:10E200006B017C010E940FEA4B015C014AE00E9415
:10E210004DC7C501B4010E9421E29B01AC01C701B9
:10E22000B6010E9412E96B017C01E0CFCF91FF9013
:10E23000EF90DF90CF90BF90AF909F908F90089518
:10E24000EF92FF920F931F93CF937C018B01C2E457
:10E250004F3F09F0C4E580E20E948A398C2F0E946A
:10E260008A398AE30E948A39F7016081718182814B
:10E27000938142E00E94AF7080EC92E20E94A2394A
:10E28000F801608171818281938142E00E94AF70C8
:10E2900062E070E080E090E0CF911F910F91FF90DD
:10E2A000EF900C9407C11F93CF93DF93CDB7DEB7E8
:10E2B00028970FB6F894DEBF0FBECDBF182F609120
:10E2C000A7147091A814072E000C880B990B0E94BC
:10E2D00023E26D837E838F8398876091A51470916C
:10E2E000A614072E000C880B990B0E9423E2698369
:10E2F0007A838B839C834AEFBE016B5F7F4FCE0195
:10E3000001960E9420716091AB057091AC05072EBB
:10E31000000C880B990B0E9423E26D837E838F8310
:10E3200098876091A9057091AA05072E000C880BAB
:10E33000990B0E9423E269837A838B839C834FEF3E
:10E34000BE016B5F7F4FCE0101960E9420716091EC
:10E35000AD051F3F39F085E11802F0011124EF559A
:10E36000FB4E608570E088EC92E20E94593A609121
:10E37000AD0570E083EC92E20E94593A28960FB600
:10E38000F894DEBF0FBECDBFDF91CF911F910895EE
:10E390000F930FB70F9300916E000B7F00936E00E9
:10E3A00078940F930BB70F930CB70F921F922F9384
:10E3B0003F934F935F936F937F938F939F93AF930D
:10E3C000BF93EF93FF9311240E94857AFF91EF9101
:10E3D000BF91AF919F918F917F916F915F914F917D
:10E3E0003F912F911F900F900CBF0F910BBF0F917A
:10E3F0000460F89400936E000F910FBF0F91189571
:10E40000CF93DF93C1EAD4E11F821E820E94AEC186
:10E4100018865D98C5EAD5E01F821E820E948A6236
:10E4200018865C98DF91CF910895109237060E946C
:10E4300000720C948D1D4F925F926F927F928F921B
:10E440009F92AF92BF92EF92FF920F931F93CF9341
:10E45000DF93B0E2A0E06A2F70E0AB014B0F511DDB
:10E4600055954795411117C0E4EEF1E285919491DD
:10E47000282F822FDF91CF911F910F91FF90EF9066
:10E48000BF90AF909F908F907F906F905F904F90D4
:10E490000895B42FE2CFA41711F0B41303C0E0E63F
:10E4A000F2E2E4CF9A0121503109220F331F220FEB
:10E4B000331FF901EE51FE4DE590F490F901EA5158
:10E4C000FE4D059114918E159F051CF3A42F08177E
:10E4D00019070CF4C0CFBC01F901EC51FE4DC591F8
:10E4E000D491F901E851FE4DA590B4906E197F09C1
:10E4F000072E000C880B990B0E9423E22B013C0194
:10E50000B5016C1B7D0B072E000C880B990B0E942C
:10E5100023E29B01AC01C301B2010E9482E24B01E4
:10E520005C01B8016E197F09072E000C880B990B4E
:10E530000E9423E29B01AC01C501B4010E9496E94F
:10E540004B015C01BE01DD0F880B990B0E9423E299
:10E550009B01AC01C501B4010E9413E90E9408EAC5
:10E56000262F972F86CFCF93DF93C1EAD4E18A81FC
:10E570009B810E94B8B69D838C83C5EAD5E08A81D1
:10E580009B810E941B729D838C83A89510927204BC
:10E59000DF91CF910895EF92FF920F931F93CF9346
:10E5A000DF93C82F7B018A018091A4058130A1F4FB
:10E5B0000E94633AC7010E94A23988E991E20E9451
:10E5C000A239C7FD33C08C2F0C2E000C990B0E9472
:10E5D00050B78AE00E948A390E940072A895809103
:10E5E000F504811132C081E08093F50480E88093C6
:10E5F000A4050E940072D5E1D150149AE1F069E1BE
:10E6000070E080E090E00E9407C1A895149868E24D
:10E6100070E080E090E00E9407C1A89568E270E099
:10E6200080E090E00E9407C1A895E6CF84E991E2DE
:10E630000E94A239CECF6DE871E2CF3F11F061E9BF
:10E6400071E240E0C8010E94903ADF91CF911F91A2
:10E650000F91FF90EF9008954F925F926F927F928B
:10E660008F929F92AF92BF92CF92DF92EF92FF92E2
:10E670000F931F93CF93DF93EC016B014A01B22EEE
:10E68000FA014080518062807380A30192016D8104
:10E690007E818F8198850E941CE28823A1F04D82A3
:10E6A0005E826F827886AA24A39420E030E0A901DC
:10E6B000F40160817181828193810E9496EA18162B
:10E6C0000CF0A12CAC828C818230A1F0833009F453
:10E6D0005AC08130C9F52D813E814F815885F601A0
:10E6E00060817181828193810E941CE287FD2CC030
:10E6F00082E08C83B701FF0C880B990B0E9423E208
:10E700009B01AC016D817E818F8198850E9412E909
:10E710009B01AC01F60160817181828193810E942D
:10E7200096EA87FD22C00E94A2C16B017C0198017C
:10E73000A8EEB3E00E9491E8C60ED71EE81EF91EAF
:10E74000C882D982EA82FB82DF91CF911F910F911B
:10E75000FF90EF90DF90CF90BF90AF909F908F9001
:10E760007F906F905F904F9008950E94A2C10881A2
:10E7700019812A813B81601B710B820B930B97FDE2
:10E78000E3CF83E08C8342E652E262E772E28B2DB4
:10E79000DF91CF911F910F91FF90EF90DF90CF907D
:10E7A000BF90AF909F908F907F906F905F904F90B1
:10E7B0000C94CB72CF93DF93EC01488159816A812D
:10E7C0007B8183E891E20E941B3C4C815D816E81DC
:10E7D0007F818AE697E20E941B3C488559856A85BD
:10E7E0007B8586E697E20E941B3C8AE0DF91CF9111
:10E7F0000C948A39BC012091D6043091D704409101
:10E80000D6045091D7042417350731F481E0261738
:10E81000370709F080E008959A01F1CF0F930FB701
:10E820000F9300916E000F930B7F00936E00009189
:10E830006F000D7F00936F000F930BB70F930CB712
:10E840000F921F922F933F934F935F936F937F93FA
:10E850008F939F93AF93BF93EF93FF9311240E94E5
:10E860001A7CFF91EF91BF91AF919F918F917F9112
:10E870006F915F914F913F912F911F900F900CBF1F
:10E880000F910BBF0F910260F89400936F000F91EE
:10E8900000936E000F910FBF0F91189500000000BC
:10E8A000000000008091930580FF27C0459A8FEFFC
:10E8B00080938C0480919305869580FF21C0479AB0
:10E8C0008FEF80938D04809193058695869580FFC8
:10E8D0001AC02A988FEF80938E04809193058695B5
:10E8E0008695869580FF12C0289A8FEF80938F04BB
:10E8F00000000000000000000895459881E0D8CF96
:10E90000479881E0DECF2A9A81E0E5CF289881E020
:10E91000EDCFCF92DF92EF92FF920F931F93CF93A1
:10E92000DF93CDB7DEB7C658D1090FB6F894DEBF76
:10E930000FBECDBFC358DF4F188219821A821B82C7
:10E94000CD57D0408091140290911502A0911602EB
:10E95000B0911702CF57DF4F88839983AA83BB8377
:10E96000C158D04084E690E090930E0680930D0647
:10E970001092B7141092B61410928B0464E070E0F9
:10E98000CE018F579F4F0E943AC180910D06909102
:10E990000E06029690930E0680930D061092B71401
:10E9A0001092B61481E0CA57DF4F8883C658D04012
:10E9B000CE018A579F4F0E94346668E470E08CEF66
:10E9C0009AE00E943AC160E170E08FE096E00E9418
:10E9D0003AC18AE097EDA3EABCE3C358DF4F8883CE
:10E9E0009983AA83BB83CD57D040CE0183589F4FD4
:10E9F0000E942C6685E995E00E9438667E018DE6CE
:10EA0000E80EF11C8FEFD7018C93C7010E9434668A
:10EA100019821A821B821C828E010F5F1F4FC80150
:10EA20000E942C6619821A821B821C82C8010E94D5
:10EA30002C6685E08983F70180838BE694E00E9451
:10EA40002C66C8010E943466C7010E94346664E6E1
:10EA500070E087E094E00E943AC18CE0D8011D92FA
:10EA60008A95E9F7C8010E943866C358DF4F1882BB
:10EA700019821A821B82CD57D0403AE0D32EDA9405
:10EA8000DD2031F0CE0183589F4F0E942C66F7CFD6
:10EA900088E0F701982F11929A95E9F7D8011D9215
:10EAA0008A95E9F783E0CB57DF4F8883C558D0407C
:10EAB000EA968FAFEA97CE018B579F4F0E9434663C
:10EAC000CE0187589F4F0E94346668E070E0C8010D
:10EAD0000E943AC168E070E0C7010E943AC1C35881
:10EAE000DF4F188219821A821B82CD57D0402AE04C
:10EAF000C22ED12CB1E0CB1AD10831F0CE0183580F
:10EB00009F4F0E942C66F6CF19828FEFF70180830A
:10EB1000C8010E943066C7010E94346680E1D82E89
:10EB2000D801ED2D1D92EA95E9F760E170E0C8018A
:10EB30000E943AC11982C8010E9430666CE070E000
:10EB40008EEA95E00E943AC1198A1A8A1B8A1C8AA9
:10EB500080E090E0A0E8BFE38D879E87AF87B88B09
:10EB60008091AA149091AB14A091AC14B091AD1403
:10EB700089839A83AB83BC832CEA35EC47E25EE35E
:10EB80006091AE147091AF148091B0149091B11453
:10EB90000E9496E96D837E838F8398872CEA35ECFB
:10EBA00047E25EE36091B2147091B3148091B414A3
:10EBB0009091B5140E9482E269877A878B879C873F
:10EBC00064E170E0C8010E943AC184E190E09A8358
:10EBD0008983C8010E9424668CE0E6E9F1E0D8014F
:10EBE00001900D928A95E1F7C8010E9428668CE099
:10EBF000E6E9F1E0D80101900D928A95E1F7C801AC
:10EC00000E9428661982C8010E9434668FE790E04E
:10EC10009A838983C8010E94246685E0E2EAF1E0D4
:10EC2000D80101900D928A95E1F765E070E0C80186
:10EC30000E943AC11982C8010E94306680E2E7EA68
:10EC4000F1E0D80101900D928A95E1F760E270E061
:10EC5000C8010E943AC1D7011C92C7010E943066C8
:10EC600086E094E00E94306682E094E00E942C6688
:10EC7000C358DF4F188219821A821B82CD57D040A9
:10EC8000CE0183589F4F0E942C6680E2F8011192BA
:10EC90008A95E9F760E270E0C8010E943AC1FE017E
:10ECA000F99688E0DF011D928A95E9F744E650E085
:10ECB00060E070E049835A836B837C834D835E837D
:10ECC0006F83788783E090E0A0E0B0E089879A873F
:10ECD000AB87BC874D875E876F87788B498B5A8B54
:10ECE0006B8B7C8B8D8B9E8BAF8BB88F898F9A8F24
:10ECF000AB8FBC8F8D8F9E8FAF8FB8A38EE190E0CE
:10ED0000A0E0B0E089A39AA3ABA3BCA38DA39EA36C
:10ED1000AFA3B8A789A79AA7ABA7BCA78DA79EA7A3
:10ED2000AFA7B8AB89AB9AABABABBCAB8DAB9EAB73
:10ED3000AFABB8AF60E470E0C8010E943AC1F8011F
:10ED40008D2D11928A95E9F760E170E0C8010E946B
:10ED50003AC1D8011D92DA94E9F760E170E0C80188
:10ED60000E943AC1C358DF4F188219821A821B824F
:10ED7000CD57D040CE0183589F4F0E942C669CE017
:10ED8000D92EF8018D2D11928A95E9F76CE070E08B
:10ED9000C8010E943AC18CE6D8011D928A95E9F714
:10EDA0006CE670E0C8010E943AC18FE794E00E94CF
:10EDB0002866F70110821182128213821482158252
:10EDC0001682178268E070E0C7010E943AC1F7011D
:10EDD0001192DA94E9F7CB57DF4F1882C558D0402B
:10EDE00080E090E0A0E4B0E4ED968CAF9DAFAEAFD4
:10EDF000BFAFED97C7010E943866CE018B579F4F7A
:10EE00000E943466CE0187589F4F0E942C668091E5
:10EE10008B04811124C000910D0610910E06809183
:10EE2000B6149091B714D7018D939C9384E690E02B
:10EE300090930E0680930D0664E070E083ED91E000
:10EE40000E943AC1C7010E94246691E00D3413402C
:10EE500009F490E080918B04892B80938B0480913E
:10EE60008B04811105C060E08BEC96E10E94971F36
:10EE700090918B0481E08927CA57DF4F0FB6F89431
:10EE8000DEBF0FBECDBFDF91CF911F910F91FF90DD
:10EE9000EF90DF90CF900895AF92BF92CF92DF9224
:10EEA000EF92FF920F931F93CF93DF93CCEFDAE0B3
:10EEB0000FE116E08CE0A82E8BE0B82EC12CD12CEF
:10EEC0007601C39469917991899199910E9421E287
:10EED000288939894A895B890E9482E20E940FEA67
:10EEE000F80161937193819391938F01C616D706B0
:10EEF000E806F90610F46B017C01AC16BD0611F7AB
:10EF00006FEF7FEFCB01A70196010E9464E8209389
:10EF10002F06309330064093310650933206DF912E
:10EF2000CF911F910F91FF90EF90DF90CF90BF9006
:10EF3000AF9008950F931F93CF93DF9300E11BE0F1
:10EF4000C8E3D6E0F80121913191419151918F01AF
:10EF500060E070E080E89FE30E9496E9699379930E
:10EF600089939993F6E0C834DF0761F70E94BBB933
:10EF7000DF91CF911F910F910C944C7790911E15BA
:10EF800080911F15981306C08091490690914A06FA
:10EF9000892B19F00E943340F1CF089590911E15EE
:10EFA00080911F15981308C08091490690914A06D8
:10EFB000892B11F40C94EC330E943340EFCFCF93A4
:10EFC000DF9320910104222379F0EC010E94BE5FBF
:10EFD0009B01AC01688579858A859B850E9412E931
:10EFE000688779878A879B87DF91CF910895CF9330
:10EFF000DF9320910104222379F0EC010E94BE5F8F
:10F000009B01AC01688579858A859B850E9413E9FF
:10F01000688779878A879B87DF91CF9108954F9280
:10F020005F926F927F928F929F92AF92BF92CF9298
:10F03000DF92EF92FF920F931F93CF93DF93CDB7A1
:10F04000DEB76A970FB6F894DEBF0FBECDBF9A8FBA
:10F05000898F5B018A01DC01D6966D917D918D913E
:10F060009C91D9970E9421E26B017C01F5012081DE
:10F070003181428153810E9482E20E947FE92B010B
:10F080003C01D8012D913D914D915C91C701B60194
:10F090000E9482E20E947FE94B015C01C301B20140
:10F0A0000E940FEA698B7A8B8B8B9C8B683771057A
:10F0B0008105910540F428E730E040E050E0298BDD
:10F0C0003A8B4B8B5C8BC501B4010E940FEA6D87B4
:10F0D0007E878F87988B683771058105910540F48D
:10F0E00088E790E0A0E0B0E08D879E87AF87B88B7F
:10F0F000E98DFA8DEE5BFF4F208131814281538192
:10F1000029833A834B835C83CA01B9010E9423E2BD
:10F110002B013C0169897A898B899C890E9421E2B3
:10F1200069877A878B879C8720E030E0A901C3013B
:10F13000B2010E941CE2882309F43BC1A701960199
:10F14000C701B6010E9482E24B015C0129853A8524
:10F150004B855C85CA01B9010E9482E29B01AC012A
:10F16000C501B4010E9412E94B015C01A3019201A7
:10F17000C301B2010E9413E99B01AC01C501B401B6
:10F180000E9496E90E947FE90E940FEA6D837E83C8
:10F190008F83988769817A818B819C8190958095F6
:10F1A000709561957F4F8F4F9F4F0E9423E24B01D7
:10F1B0005C016D857E858F8598890E9421E2698337
:10F1C0007A838B839C8320E030E0A901C501B401E0
:10F1D0000E941CE2882309F4F0C029813A814B8106
:10F1E0005C81CA01B9010E9482E26D8B7E8B8F8B9C
:10F1F000988FA7019601C701B6010E9482E29B0188
:10F20000AC016D897E898F89988D0E9412E96B010E
:10F210007C01A5019401C501B4010E9413E99B0181
:10F22000AC01C701B6010E9496E90E943EEAA98D91
:10F23000BA8D95968D909D90AD90BC9098977501E4
:10F2400064012D813E814F815885C21AD30AE40A98
:10F25000F50A0E940FEAC61AD70AE80AF90AF7FE69
:10F260006EC020E030E0A901C301B2010E941CE29F
:10F27000882309F4A6C0C501B4010E9421E26B01F4
:10F280007C01A3019201C301B2010E9413E99B0119
:10F29000AC01C701B6010E9482E26B017C012985A5
:10F2A0003A854B855C85CA01B9010E9482E29B01C7
:10F2B000AC01C701B6010E9412E96B017C012981F2
:10F2C0003A814B815C81CA01B9010E9482E29B01B3
:10F2D000AC01C701B6010E9413E96B017C0120E07B
:10F2E00030E040E850E4C301B2010E9482E29B0199
:10F2F000AC01C701B6010E9496E90E947FE96B014B
:10F300007C0120E030E0A9010E9496EA18161CF06A
:10F31000C12CD12C7601C701B6010E940FEA6D8382
:10F320007E838F83988786169706A806B90620F4F1
:10F330008D829E82AF82B886C12CD12C76018D81C0
:10F340009E81AF81B885E98DFA8D81A792A7A3A789
:10F35000B4A7C80ED91EEA1EFB1EC5A6D6A6E7A6F0
:10F36000F0AA29893A894B895C8922AF33AF44AF2F
:10F3700055AFFE962D853E854F8558892083318374
:10F38000428353836A960FB6F894DEBF0FBECDBF9B
:10F39000DF91CF911F910F91FF90EF90DF90CF9071
:10F3A000BF90AF909F908F907F906F905F904F90A5
:10F3B000089560E070E0CB01E5CE60E070E0CB0145
:10F3C00034CF60E070E0CB0198CF90916F0081E086
:10F3D00091FD02C080E0089590916F009D7F909311
:10F3E0006F000895CF93C82F0E94E57994E0C99FDC
:10F3F00090011124F901E752FB4F2B513B4FD901EA
:10F400004D915D916D917C914083518362837383B3
:10F4100091E09093D804882319F0CF910C94033194
:10F42000CF910895CF92DF92EF92FF9280917D0469
:10F43000329B60C0816080937D0480917D04339B0A
:10F440005BC0826080937D0480917D04349B56C0B4
:10F45000846080937D04C090C904C0FE10C0809178
:10F46000930580FF0CC080917D0480FF08C08091CF
:10F47000A30581608093A30580E00E94F279D12CDE
:10F48000F12CE12CD701C601B695A79597958795E4
:10F4900080FF11C080919305869580FF0CC08091FC
:10F4A0007D0481FF08C08091A30582608093A3053D
:10F4B00081E00E94F27982E0F694E794D794C794B1
:10F4C0008A95D1F7C0FE1CC08091930586958695DC
:10F4D00080FF16C080917D0482FF12C08091A30539
:10F4E00084608093A30582E0FF90EF90DF90CF903F
:10F4F0000C94F2798E7F9FCF8D7FA4CF8B7FA9CF85
:10F50000FF90EF90DF90CF9008950F931F93CF93CC
:10F51000DF93809147018F3708F447C08F57909150
:10F52000A91490931805992309F43DC05D9A909110
:10F53000AD0590931705992309F441C05C9A8F5F3C
:10F54000809347018091160591E0892780931605E5
:10F5500081110E94122080914601C1E0C80F8530C0
:10F560000CF0C0E0823009F4D3C05CF5882309F4C4
:10F570003EC0813009F4C1C0C0934601809192051C
:10F5800081110E94127A8091490690914A06009753
:10F5900029F0019790934A0680934906DF91CF9115
:10F5A0001F910F9108955D98C2CF9091180589170A
:10F5B00008F05D9890911705891708F4C0CF5C9802
:10F5C000BECF843009F4BBC00CF4B5C08530A1F6C1
:10F5D00090911505911102C0809315058091150534
:10F5E000815080931505882339F2C5E0C5CF8091FD
:10F5F00045018F5F80311CF480934501BDCF10928F
:10F60000450180917204811113C08091A1149091E1
:10F61000A2149093A4148093A3148091A5059091B3
:10F62000A6059093A8058093A70581E080937204B6
:10F630001092A2141092A1141092A6051092A50582
:10F640000091A3141091A4148091A7149091A81470
:10F65000D1E0181619062CF08091A914811101C06F
:10F66000D0E080914C0190914D01081719073CF4AE
:10F6700042E852E26FE872E280E00E94CB72DD2342
:10F6800071F080914A0190914B01801791073CF4F1
:10F6900041EA52E26EEA72E280E00E94CB7200918F
:10F6A000AB051091AC052091A7053091A80580917C
:10F6B0008F0590919005281739073CF442E852E2F3
:10F6C0006FE872E28FEF0E94CB72101611060CF0F9
:10F6D00053CF2091A7053091A805809148019091C2
:10F6E0004901821793070CF047CF41EA52E26EEAD4
:10F6F00072E28FEF0E94CB723FCF10927B0087E4C3
:10F7000080937C0080917A00806480937A0034CF6B
:10F7100080917A0086FD26C0209178003091790092
:10F720008091A1149091A214820F931F9093A21420
:10F730008093A11421CF10927B0086E4E1CF8091C9
:10F740007A0086FD11C02091780030917900809177
:10F75000A5059091A605820F931F9093A60580930F
:10F76000A5050ACFC2E008CFC4E006CF0E94E57924
:10F770001092330610923406109235061092360617
:10F7800081110C94033108950F931F9380911E15DE
:10F7900090911F15891B8F7009F449C090911B151A
:10F7A000992361F0833040F48FEF890F29F0809323
:10F7B0001B1590E080E038C010921B1580911F153A
:10F7C0002BE4829FC0011124855B994FFC012081AD
:10F7D00020FDEFCF409133065091340660913506FD
:10F7E00070913606E95BFF4F0081118122813381E0
:10F7F000401B510B620B730B40933306509334063E
:10F80000609335067093360620911F152F5F2F7079
:10F8100020931C1530911F1520911D15321304C023
:10F8200020911C1520931D151F910F9108950E9482
:10F83000B67BBFCF2F923F924F925F926F927F9293
:10F840008F929F92AF92BF92CF92DF92EF92FF92F0
:10F850000F931F93CF93DF9300D000D0CDB7DEB7C7
:10F860008FEF9FEF90938900809388000AE00983CF
:10F87000312C212C78948091D2049091D304A091C2
:10F88000D404B091D504892B8A2B8B2B09F0C4C1E9
:10F890008091D8048823E1F08091D6049091D70418
:10F8A0001092D804892B09F4B7C11092D704109292
:10F8B000D6041092C90490911E1580911F159817B7
:10F8C00009F4AAC180911F158F5F8F7080931F1557
:10F8D0008091D6049091D704892B09F49DC1409161
:10F8E000CE045091CF046091D0047091D1048091E6
:10F8F000CA049091CB04A091CC04B091CD040091A6
:10F90000BC0410E030E020E0841B950BA60BB70B85
:10F91000081719072A073B0710F4D901C8018A8381
:10F92000840F951FA61FB71F8093CE049093CF041A
:10F93000A093D004B093D104E1E0C0909404D0909F
:10F940009504E0909604F09097048091A40490911F
:10F95000A504A091A604B091A704C80ED91EEA1E62
:10F96000FB1EC092A404D092A504E092A604F092DB
:10F97000A704F7FC33C040918C04042E000C550BF7
:10F98000660B770B8091E5049091E604A091E70463
:10F99000B091E804840F951FA61FB71F8093E5045C
:10F9A0009093E604A093E704B093E8048091900458
:10F9B00090919104A0919204B0919304A7019601B3
:10F9C000281B390B4A0B5B0BDA01C9018093A40495
:10F9D0009093A504A093A604B093A7040091980463
:10F9E0001091990420919A0430919B048091A8046D
:10F9F0009091A904A091AA04B091AB04080F191F1B
:10FA00002A1F3B1F0093A8041093A9042093AA0463
:10FA10003093AB0437FD33C080918D04082E000C69
:10FA2000990BAA0BBB0B4091E9045091EA04609139
:10FA3000EB047091EC04840F951FA61FB71F8093F1
:10FA4000E9049093EA04A093EB04B093EC04809152
:10FA5000900490919104A0919204B0919304B90103
:10FA6000A801481B590B6A0B7B0BDB01CA01809371
:10FA7000A8049093A904A093AA04B093AB04409166
:10FA80009C0450919D0460919E0470919F0480910C
:10FA9000AC049091AD04A091AE04B091AF04480FB6
:10FAA000591F6A1F7B1F4093AC045093AD046093B1
:10FAB000AE047093AF0477FD33C080918E04082E9E
:10FAC000000C990BAA0BBB0B8090ED049090EE04F8
:10FAD000A090EF04B090F004880D991DAA1DBB1DE5
:10FAE0008093ED049093EE04A093EF04B093F004A0
:10FAF0008091900490919104A0919204B09193040C
:10FB00002A013B01481A590A6A0A7B0AD301C20139
:10FB10008093AC049093AD04A093AE04B093AF0473
:10FB20008090A0049090A104A090A204B090A3049F
:10FB30008091B0049091B104A091B204B091B3044B
:10FB4000880D991DAA1DBB1D8093B0049093B1042C
:10FB5000A093B204B093B304B7FD33C040908F04B8
:10FB6000042C000C5508660877088090F1049090EA
:10FB7000F204A090F304B090F404840C951CA61C2D
:10FB8000B71C8092F1049092F204A092F304B09218
:10FB9000F4048090900490909104A0909204B0900E
:10FBA00093042C013D01481859086A087B08530149
:10FBB00042018092B0049092B104A092B204B0923B
:10FBC000B304E11104C0E0918400F0918500F7FED8
:10FBD0005F9A37FF469A77FF2B9AB7FF299AE091F1
:10FBE0008400F0918500E0918400F0918500F7FE9B
:10FBF0005F9837FF469877FF2B98B7FF29985A8070
:10FC0000552021F080918400909185000A81015057
:10FC10000A83E0E0011191CE80905401909055014B
:10FC2000A0905601B090570181149104A104B10431
:10FC300009F047C08091EC059091ED05009709F41B
:10FC40002FC023B1247015980000000000000000B0
:10FC5000181619060CF0D7C02A9A00000000000000
:10FC600000002B9A34E03A950000E9F72B98000049
:10FC7000000000000000222309F4C7C02A9A0000F7
:10FC8000000000000000181619060CF0C0C080919A
:10FC9000EC059091ED0501979093ED058093EC05AF
:10FCA0000E94B133882309F4B8C080ED97E0A0E04A
:10FCB000B0E08093540190935501A0935601B09306
:10FCC00057018091D2049091D304A091D404B091B3
:10FCD000D504892B8A2B8B2B09F053C4E091D604D1
:10FCE000F091D704309709F427C58091CE04909104
:10FCF000CF04A091D004B091D1044091CA04509196
:10FD0000CB046091CC047091CD0484179507A607AD
:10FD1000B70708F486C01092D7041092D604109248
:10FD2000C90490911E1580911F15981709F404C5F8
:10FD300080911F158F5F8F7080931F1580EDC82EE7
:10FD400087E0D82EE12CF12C8091D6049091D70435
:10FD5000892B09F00EC40E94C47B9093D704809332
:10FD6000D604892B09F405C44090D6045090D704DA
:10FD70005C824B82D2018C9183FFB3C2F201858DEC
:10FD8000968DA78DB0A1418D528D638D748D05899F
:10FD900016892789308D0093E5041093E60420939B
:10FDA000E7043093E8044093E9045093EA04609335
:10FDB000EB047093EC048093ED049093EE04A09315
:10FDC000EF04B093F00481A192A1A3A1B4A1809308
:10FDD000F1049093F204A093F304B093F40410920E
:10FDE000D7041092D6041092C90490911E158091E8
:10FDF0001F15981709F4AFCF80911F158F5F8F7073
:10FE000080931F15A8CF2A9828CF2A9838CF8091A1
:10FE1000EC059091ED0501963FCF8FEF9FEFDC0150
:10FE200048CF4091C5045091C6046091C7047091B9
:10FE3000C804481759076A077B0708F4DEC0809199
:10FE4000C1049091C204A091C304B091C40441A91B
:10FE500052A963A974A91127859F412C969F9001EF
:10FE6000A69F300DA59F200D311D869F400C211DA2
:10FE7000311F959F400C211D311FA49F400C211D57
:10FE8000311F949F410C211F311F4694211F311FA8
:10FE9000789F200D311D799F300D112442AD53AD57
:10FEA00064AD75AD420F531F611D711D4093BD04BC
:10FEB0005093BE046093BF047093C00406A917A9B1
:10FEC00020AD31AD041715072607370740F400931E
:10FED000BD041093BE042093BF043093C00440902F
:10FEE000BD045090BE046090BF047090C00423E62F
:10FEF00031E201E00A83F9014591559165917491D0
:10FF0000441555056605770570F476946794579403
:10FF100047941A81110F1A832C5F3F4F4FE751E22C
:10FF20004217530741F75A815093BC0460E24616CA
:10FF300051046104710428F410E2412E512C612C0B
:10FF4000712C70E2471A5108610871084114E8E009
:10FF50005E066104710408F42EC0F4E05F9E900117
:10FF600011242D59324EF901329645915491042DA8
:10FF7000EE27059FB001049F610D7E1F06946E1F42
:10FF80007E1F1124AB0170E060E0F901C590D490B0
:10FF9000F12CE12CC41AD50AE60AF70A8C0D9D1D36
:10FFA000AE1DBF1D8093C1049093C204A093C304EF
:10FFB000B093C404C9CEB301A20176956795579555
:10FFC00047959A012C7F2D59364EF901C590D49052
:10FFD000F901329645915491142D1770149F900198
:10FFE000159F300D1124F3E036952795FA95E1F72A
:10FFF000C21AD30AF12CE12CD1CF4091B804509110
:020000021000EC
:10000000B9046091BA047091BB04481759076A0794
:100010007B0708F0D4C08091B4049091B504A091FE
:10002000B604B091B70441A952A963A974A92227C3
:10003000859F312D969F8001A69F100DA59F000DD5
:10004000111D869F300D011D121F959F300D011D42
:10005000121FA49F300D011D121F949F310D021F0E
:10006000121F3695021F121F789F000D111D799FD8
:10007000100D112430E020E04091BD045091BE04E9
:100080006091BF047091C004FE96408051806280F0
:100090007380041715072607370758F4401B510BC8
:1000A000620B730B441655066606770610F42A0198
:1000B0003B0123E631E241E04A83F9014591559144
:1000C00065917491441555056605770570F476942D
:1000D0006794579447945A81550F5A832C5F3F4F2A
:1000E0006FE771E26217730741F77A817093BC047E
:1000F000E0E24E1651046104710428F400E2402E3F
:10010000512C612C712CF0E24F1A510861087108D2
:10011000411408E050066104710408F42EC014E094
:10012000519E900111242D59324EF901329645917C
:100130005491F42DEE27F59FB001F49F610D7E1FC1
:1001400006946E1F7E1F1124AB0170E060E0F90180
:10015000C590D490F12CE12CC41AD50AE60AF70A0E
:100160008C0D9D1DAE1DBF1D8093B4049093B504EE
:10017000A093B604B093B704E7CDB301A20176957E
:100180006795579547959A012C7F2D59364EF90161
:10019000C590D490F901329645915491042D077081
:1001A000049F9001059F300D112413E0369527958B
:1001B0001A95E1F7C21AD30AF12CE12CD1CF809124
:1001C000410190914201A0914301B0914401B7FFD8
:1001D0005DC0C6A8D7A8E0ACF1AC83E691E221E00F
:1001E000FC0145915591659174914C155D056E0525
:1001F0007F0558F4F694E794D794C794220F049699
:100200004FE751E24817590759F72093BC0450E2D1
:10021000C516D104E104F10428F470E2C72ED12CF4
:10022000E12CF12C60E2C61AD108E108F108C114F2
:1002300078E0D706E104F10408F431C0A4E0DA9EC6
:10024000C00111248D59924EFC01329625913491B2
:10025000BC2D6627B39FA001B29F410D561F069487
:10026000461F561F112470E060E0FC0185919491B7
:10027000B0E0A0E0841B950BA60BB70B8093410167
:1002800090934201A0934301B0934401C090410177
:10029000D0904201E0904301F090440155CDD70148
:1002A000C601B695A795979587958C7F8D59964EE3
:1002B000FC0125913491FC01329645915491EC2D2D
:1002C000E770E49FC001E59F900D112463E09695CF
:1002D00087956A95E1F7281B390BC901B0E0A0E0CA
:1002E000CDCFAB81BC8155960D911D912D913C9147
:1002F000589781E0011511052105310509F480E0C9
:10030000EB81FC81C18CD28CE38CF48CC114D104C0
:10031000E104F10409F08260AB81BC815D964D91EE
:100320005D916D917C919097411551056105710525
:1003300009F084608093C9041092B4041092B5044B
:100340001092B6041092B7041092C1041092C20425
:100350001092C3041092C404EB81FC8185A196A184
:10036000A7A1B0A58093CA049093CB04A093CC041A
:10037000B093CD04442455243201481A590A6A0A1C
:100380007B0A4092A4045092A5046092A604709245
:10039000A7044092A8045092A9046092AA04709203
:1003A000AB044092AC045092AD046092AE047092E3
:1003B000AF044092B0045092B1046092B2047092C3
:1003C000B30441A052A063A074A0440C551C661C49
:1003D000771C000F111F221F331F009394041093EA
:1003E00095042093960430939704CC0CDD1CEE1CEE
:1003F000FF1CC0929804D0929904E0929A04F09263
:100400009B04440F551F661F771F40939C04509315
:100410009D0460939E0470939F044092A0045092A8
:10042000A1046092A2047092A304880F991FAA1FCE
:10043000BB1F8093900490939104A0939204B09377
:1004400093041092CE041092CF041092D004109214
:10045000D10481A592A5A3A5B4A58093C5049093CA
:10046000C604A093C704B093C80485A596A5A7A504
:10047000B0A98093B8049093B904A093BA04B09340
:10048000BB0485A990919305891721F0809393056A
:100490000E944E748091920581110E94127A442428
:1004A0004A94542C32014092410150924201609290
:1004B000430170924401AB81BC81DA964D915D910C
:1004C0006D917C91DD974093BD045093BE04609381
:1004D000BF047093C00483E691E2A1E0FC010591A2
:1004E000159125913491041715072607370758F4FD
:1004F0007695679557954795AA0F0496EFE7F1E231
:10050000E817F90759F7A093BC044032510561057B
:10051000710520F440E250E060E070E04052510983
:10052000610971094115F8E05F076105710508F47B
:10053000DAC004E0509FC00111248D59924EFC0195
:10054000329625913491AA27439FF001429FE10DF5
:10055000FA1F0694EA1FFA1F1124AF0170E060E051
:10056000FC01C590D490F12CE12CC41AD50AE60AFE
:10057000F70AC092D204D092D304E092D404F0924D
:10058000D50489288A288B28C9F48091D2049091B7
:10059000D304A091D404B091D5048A3F9105A1055C
:1005A000B10560F42AEF30E040E050E02093D2043F
:1005B0003093D3044093D4045093D5044091540114
:1005C0005091550160915601709157010091D204EC
:1005D0001091D3042091D4043091D5044F3F8FEF74
:1005E00058076807780799F0D901C801B695A7950B
:1005F00097958795481759076A077B0740F48093BA
:10060000540190935501A0935601B0935701409126
:1006100054015091550160915601709157014F3F1F
:100620009FEF59076105710508F07DC04B835A8320
:10063000F62FE72F8B819A81AF2FBE2F081719074E
:100640002A073B0710F4D901C801081B190B2A0B14
:100650003B0B0093D2041093D3042093D404309323
:10066000D5044F3FEFEF5E076E077E0761F0481B32
:10067000590B6A0B7B0B40935401509355016093C7
:10068000560170935701F8942091840030918500B1
:10069000205F3F4F098101500983002309F44AC0BC
:1006A000280E391E2216330610F40C943A7C309230
:1006B00089002092880078940F900F900F900F90EF
:1006C000DF91CF911F910F91FF90EF90DF90CF902E
:1006D000BF90AF909F908F907F906F905F904F9062
:1006E0003F902F900895DB01CA01B695A795979585
:1006F00087958C7F8D59964EFC01C590D490FC0156
:100700003296259134914770429FC001439F900DCE
:100710001124A3E096958795AA95E1F7C81AD90AFE
:10072000F12CE12C26CFAFEFAB83BFEFBA83F0E023
:10073000E0E080CF1901BBCF80EDC82E87E0D82E36
:10074000E12CF12C08CBFC012081318142815381C5
:1007500060911C0B70911D0B80911E0B90911F0BD3
:100760000E9482E20E949BEA60932C1570932D15E3
:1007700080932E1590932F1590911E1580911F1523
:1007800098130C9458660E94BE770E94E5794091B8
:100790002C1550912D1560912E1570912F154093A9
:1007A000F1045093F2046093F3047093F404811104
:1007B0000C94033108954F925F926F927F928F92C3
:1007C0009F92AF92BF92CF92DF92EF92FF920F93E0
:1007D0001F93CF93DF93EC018B015A01F901209114
:1007E0001C0B30911D0B40911E0B50911F0B608113
:1007F0007181828193810E9482E20E949BEA6B0157
:100800007C012091180B3091190B40911A0B5091DB
:100810001B0BF50160817181828193810E9482E2CC
:100820000E949BEA4B015C012091140B3091150B47
:100830004091160B5091170BF801608171818281F4
:1008400093810E9482E20E949BEA2B013C0120914D
:10085000100B3091110B4091120B5091130B6881CA
:1008600079818A819B810E9482E20E949BEA609347
:100870002015709321158093221590932315409293
:100880002415509225156092261570922715809296
:10089000281590922915A0922A15B0922B15C09276
:1008A0002C15D0922D15E0922E15F0922F159091C7
:1008B0001E1580911F15981791F0DF91CF911F9110
:1008C0000F91FF90EF90DF90CF90BF90AF909F90EF
:1008D0008F907F906F905F904F900C9458660E941D
:1008E000BE770E94E57940912815509129156091B5
:1008F0002A1570912B150091241510912515209122
:10090000261530912715C0902015D0902115E09024
:100910002215F0902315C092E504D092E604E092EF
:10092000E704F092E8040093E9041093EA042093AA
:10093000EB043093EC044093ED045093EE04609389
:10094000EF047093F00440912C1550912D15609197
:100950002E1570912F154093F1045093F20460937B
:10096000F3047093F404882391F0DF91CF911F91E9
:100970000F91FF90EF90DF90CF90BF90AF909F903E
:100980008F907F906F905F904F900C940331DF9128
:10099000CF911F910F91FF90EF90DF90CF90BF907C
:1009A000AF909F908F907F906F905F904F90089541
:1009B000CF92DF92EF92FF92CF93DF93C82F0E94E6
:1009C000E57994E0C99FE0011124FE01EB51FB4F52
:1009D000C080D180E280F38081110E940331C85C25
:1009E000D94FC701B6010E9423E2288139814A818B
:1009F0005B810E9482E2DF91CF91FF90EF90DF90C8
:100A0000CF900895CF92DF92EF92FF92CF93DF9332
:100A1000C82F0E94E57994E0C99FE0011124FE01EE
:100A2000E752FB4FC080D180E280F38081110E94A9
:100A30000331C85CD94FC701B6010E9423E2288167
:100A400039814A815B810E9482E2DF91CF91FF90E0
:100A5000EF90DF90CF900895CF930E94E579C82F53
:100A600080911F1580931E1580931D1580931C1572
:100A700084E680931B150E94B67B80ED93E09093F3
:100A80004A0680934906C1110E94033181E0809398
:100A9000D804CF910895CF93DF9324E0829FC001C3
:100AA0001124EC01CF5FD94FFC01EB56FA4F8F5167
:100AB0009C4FDC012D913D914D915C916081718144
:100AC000828193810E9413E9688379838A839B835F
:100AD000DF91CF91089580FF04C090917E0490FD36
:100AE0008E7F81FF05C090917E04969590FD8D7F4D
:100AF00082FF06C090917E049695969590FD8B7F1F
:100B00000895CF92DF92EF92FF920F931F93C12C23
:100B1000D12C76018C0120E53BE04CE45BE068E4FD
:100B20007BE084E49BE00E9459B91F910F91FF90F4
:100B3000EF90DF90CF9008954F925F926F927F92E7
:100B40008F929F92AF92BF92CF92DF92EF92FF92DD
:100B50000F931F93CF93DF93CDB7DEB72C970FB6CC
:100B6000F894DEBF0FBECDBF2B013C0129873A8729
:100B70004B875C8747015801F601E080F1800281D4
:100B8000138120E030E0A901B701C8010E941CE2F6
:100B9000882309F484C05E2D4F2D302F212F852FFF
:100BA000942FA32FB22F89839A83AB83BC8320E039
:100BB00030E0A901B701C8010E941CE2811104C004
:100BC000E12CF12C08E413E4C701D8018D839E8346
:100BD000AF83B887A501940160914C0B70914D0BC8
:100BE00080914E0B90914F0B0E941CE287FF0CC02E
:100BF00080924C0B90924D0BA0924E0BB0924F0BEB
:100C0000CE0101960E9481854092440B5092450B83
:100C10006092460B7092470B89859A85AB85BC859F
:100C20008093480B9093490BA0934A0BB0934B0BC6
:100C3000CE0105960E948185A501940160914C0B1F
:100C400070914D0B80914E0B90914F0B0E9496EA44
:100C5000181664F480924C0B90924D0BA0924E0BA0
:100C6000B0924F0BCE0101960E9481850E94BE7703
:100C70002C960FB6F894DEBF0FBECDBFDF91CF919B
:100C80001F910F91FF90EF90DF90CF90BF90AF90AA
:100C90009F908F907F906F905F904F90089550E05D
:100CA00040E030E820E47BCFCF92DF92EF92FF92DA
:100CB0000F931F936B01FC01E080F180028113818F
:100CC000E4E4FBE0248135814681578160817181B4
:100CD000828193810E949C851F910F91FF90EF90DC
:100CE000DF90CF9008950C94BBB92F923F924F9212
:100CF0005F926F927F928F929F92AF92BF92CF92AC
:100D0000DF92EF92FF920F931F93CF93DF93CDB7B4
:100D1000DEB76C970FB6F894DEBF0FBECDBF8091E3
:100D20007104811150C18091700481113CC1809186
:100D30007204811119C06C960FB6F894DEBF0FBE15
:100D4000CDBFDF91CF911F910F91FF90EF90DF907A
:100D5000CF90BF90AF909F908F907F906F905F905B
:100D60004F903F902F9008950E94B3720E94A2C1AD
:100D70004B015C010091A5141091A61480915001C3
:100D800090915101801791070CF448C26091A7140B
:100D90007091A814072E000C880B990B0E9423E277
:100DA0006D837E838F839887B801110F880B990B11
:100DB0000E9423E269837A838B839C832AE0E22E5C
:100DC000F12C0CE310E020E0AE014B5F5F4FBE0161
:100DD0006F5F7F4F89E095E10E942C730091A5140D
:100DE0001091A61480914E0190914F0180179107A8
:100DF0000CF4F0C060E06093A91480919D14909170
:100E00009E14A0919F14B091A0140097A105B10564
:100E100039F1A5019401281B390B4A0B5B0BDA0150
:100E2000C901B7FD1DC080919B1490919C140817B7
:100E300019070CF413C28091A7149091A81400977D
:100E400039F00E5F1F4F0497081719070CF41CC2E6
:100E500010929D1410929E1410929F141092A01440
:100E60008091A9059091AA05873991050CF0E2C1FE
:100E70008091110590911205A0911305B091140570
:100E80000097A105B10561F1A5019401281B390B5B
:100E90004A0B5B0BDA01C901B7FD22C08091A9059D
:100EA0009091AA0520910F053091100582179307A4
:100EB0000CF4CCC12091AB053091AC052115310566
:100EC00039F0029624503109821793070CF4EFC1D0
:100ED000109211051092120510921305109214052C
:100EE00080910B0590910C05A0910D05B0910E0518
:100EF000A5019401281B390B4A0B5B0BDA01C901D0
:100F0000B7FD19CF38E8830E33E1931EA11CB11C45
:100F100080920B0590920C05A0920D05B0920E05E3
:100F20006091AB057091AC05072E000C880B990BF6
:100F30000E9423E26D837E838F8398876091A90549
:100F40007091AA05072E000C880B990B0E9423E2D2
:100F500069837A838B839C8382E0E82EF12C02E301
:100F600010E02FEFAE014B5F5F4FBE016F5F7F4F11
:100F700082E195E10E942C738091A9059091AA05C8
:100F80009C01255031092239310508F05BC12091BF
:100F9000AB053091AC05821793070CF467C180E074
:100FA0008093AD05C8CE109270040E942C850E94DB
:100FB000BE770E94F4B80E947386809172048823E1
:100FC00009F4B9CED1CE41E070E060E084ED91E269
:100FD0000E94903A80915001909151010817190791
:100FE0000CF008CFE090A714F090A814B801012EDF
:100FF000000C880B990B0E9423E21B012C01E114C9
:10100000F10409F43CC1B701601B710B072E000C01
:10101000880B990B0E9423E26B017C0120E030E0F9
:1010200040E251EC0E941CE287FD29C120E030E043
:1010300040E251E4C701B6010E9496EA18160CF48A
:1010400049C180910A05811149C120910205309161
:101050000305409104055091050529873A874B8780
:101060005C878091060590910705A0910805B091D5
:1010700009058D879E87AF87B88BA201910160918A
:10108000F6047091F7048091F8049091F9040E949D
:1010900012E92091B2143091B3144091B4145091DC
:1010A000B5140E9482E229853A854B855C850E94B1
:1010B00012E920ED3CEC4CE45DE30E9482E22985DC
:1010C0003A854B855C850E9413E9698B7A8B8B8B03
:1010D0009C8B6093020570930305809304059093A5
:1010E00005052091AE143091AF144091B014509189
:1010F000B1142D8B3E8B4F8B588F2D853E854F85A0
:101100005889C701B6010E9413E9762E672E898798
:101110009D8720E030E0A9010E941CE287FDE9C024
:101120002D893E894F89588D60E070E08FE793E408
:101130000E9496E9698F7A8F8B8F9C8F272D362D91
:1011400049855D850E941CE287FF06C0798C6A8C08
:101150003B8D39874C8D4D87872D962DA985BD8573
:101160008093060590930705A0930805B0930905A1
:101170002091AA143091AB144091AC145091AD144D
:10118000C701B6010E9482E26B017C01C092FA04A1
:10119000D092FB04E092FC04F092FD04272D362D42
:1011A00049855D856D897E898F89988D0E9482E24F
:1011B0009B01AC012093FE043093FF044093000593
:1011C00050930105C701B6010E9413E929893A89A4
:1011D0004B895C890E9413E920E030E0A9010E945C
:1011E00013E96B017C0120E030E0A9010E941CE2C0
:1011F00087FD48C020E030E04FE753E4C701B60167
:101200000E9496EA1816A4F56FE72092F604309231
:10121000F7044092F8045092F904EDCD42E852E20E
:101220006FE872E280E00E94CB720091A5141091E9
:10123000A614ACCD42E852E26FE872E28FEF0E9452
:10124000CB7216CE1092AD055C9875CD46EB51E28F
:1012500065EC71E28FEF0E94CB7242CE46EB51E219
:1012600065EC71E280E00E94CB72FACD8FE798CEF8
:10127000C701B6010E9408EA75956795C6CF81E05F
:1012800080930A0560E0C1CF10939C1400939B14D7
:101290000E94A2C1605B7C438F4F9F4F60939D145F
:1012A00070939E1480939F149093A014D9CD909323
:1012B000100580930F050E94A2C1605E70448D4F9F
:1012C0009F4F6093110570931205809313059093BF
:1012D000140506CE81E080930A0596CF10920A0588
:1012E0001D861E861F86188A19861A861B861C86EE
:1012F000C4CE712C612C19861D862ECF2F923F9261
:101300004F925F926F927F928F929F92AF92BF9215
:10131000CF92DF92EF92FF920F931F93CF93DF93C1
:10132000CDB7DEB7A6970FB6F894DEBF0FBECDBF20
:1013300080912701882309F4CDC080917E04C82EB6
:10134000D12CF12CE12C80FF3CC0809029019090A1
:101350002A01A0902B01B0902C012091ED03309137
:10136000EE034091EF035091F003C501B4010E94D8
:1013700096EA181644F48092ED039092EE03A09240
:10138000EF03B092F0038090350190903601A09069
:101390003701B09038012091ED033091EE03409178
:1013A000EF035091F003C501B4010E941CE287FFD6
:1013B00008C08092ED039092EE03A092EF03B092EA
:1013C000F003D701C601B695A7959795879580FF3D
:1013D0003CC080902D0190902E01A0902F01B090E4
:1013E00030012091F1033091F2034091F3035091C9
:1013F000F403C501B4010E9496EA181644F48092E1
:10140000F1039092F203A092F303B092F403809060
:10141000390190903A01A0903B01B0903C0120919D
:10142000F1033091F2034091F3035091F403C501AD
:10143000B4010E941CE287FF08C08092F1039092E1
:10144000F203A092F303B092F40392E0F694E794CF
:10145000D794C7949A95D1F7C0FE3CC0C090310193
:10146000D0903201E0903301F09034012091F503E7
:101470003091F6034091F7035091F803C701B6018C
:101480000E9496EA181644F4C092F503D092F6032F
:10149000E092F703F092F803C0903D01D0903E0136
:1014A000E0903F01F09040012091F5033091F60368
:1014B0004091F7035091F803C701B6010E941CE266
:1014C00087FF08C0C092F503D092F603E092F703BD
:1014D000F092F8038091FB0A83FD7EC02091500BAF
:1014E0003091510B4091520B5091530B6091F90385
:1014F0007091FA038091FB039091FC030E941CE21F
:10150000882309F469C010914806111161C08091C7
:101510005C0190915D0101972091A5143091A61472
:10152000281739073CF40E94673A8FE496E10E943D
:10153000A23911E02091500B3091510B4091520B88
:101540005091530B6091F9037091FA038091FB0362
:101550009091FC030E9412E96B017C0120E030E0D5
:10156000A9010E9496EA87FF04C0F7FAF094F7F801
:10157000F094209158013091590140915A015091B5
:101580005B01C701B6010E9482E220E030E84BE334
:1015900054E40E9496EA1816ECF40E94673A80E33D
:1015A00096E10E94A2398091F9039091FA03A091EB
:1015B000FB03B091FC038093500B9093510BA093CD
:1015C000520BB093530B89EF93E00E94A38304C0A6
:1015D00010E0B0CF1111E7CF2AE037ED43E25CE332
:1015E0006091210170912201809123019091240149
:1015F0000E9482E26B017C0160911F0170912001C9
:10160000072E000C880B990B0E9423E29B01AC0172
:10161000C701B6010E9482E2698B7A8B8B8B9C8B0F
:1016200080910104882309F46CC02091440B30910F
:10163000450B4091460B5091470B6091ED03709123
:10164000EE038091EF039091F0030E9412E96D8BFD
:101650007E8B8F8B988F2091480B3091490B409156
:101660004A0B50914B0B6091F1037091F203809102
:10167000F3039091F4030E9412E9698F7A8F8B8FA4
:101680009C8F20914C0B30914D0B40914E0B509103
:101690004F0B6091F5037091F6038091F7039091E1
:1016A000F8030E9412E96D8F7E8F8F8F98A320918F
:1016B000500B3091510B4091520B5091530B609154
:1016C000F9037091FA038091FB039091FC030E944F
:1016D00012E96B017C0120E030E0A9016D897E896F
:1016E0008F89988D0E941CE281110FC020E030E0AC
:1016F000A901698D7A8D8B8D9C8D0E941CE28111D0
:1017000004C0C12CD12C76012CC12D893E894F8972
:10171000588DCA01B9010E9482E24B015C01298DFA
:101720003A8D4B8D5C8DCA01B9010E9482E29B010A
:10173000AC01C501B4010E9413E94B015C012D8D80
:101740003E8D4F8D58A1CA01B9010E9482E29B01D2
:10175000AC01C501B4010E9413E94B015C01A70172
:101760009601C701B6010E9482E29B01AC01C5014E
:10177000B4010E9413E90E94D4EA4B015C012DEBF5
:1017800037E346E855E30E941CE287FF0FC020E0E4
:1017900030E0A901C701B6010E9496EA460157014F
:1017A00087FF04C0B7FAB094B7F8B0942DEB37E3D5
:1017B00046E855E3C501B4010E941CE287FDDEC086
:1017C00020E030E040EA51E4C501B4010E9496E90E
:1017D0000E940FEA1B01672B19F422242394312C59
:1017E000B10190E080E00E9421E29B01AC0160E049
:1017F00070E080E89FE30E9496E92B013C01AC0178
:101800009B01C501B4010E9482E24B015C01A3016E
:1018100092016D897E898F89988D0E9482E26D8BFD
:101820007E8B8F8B988FA3019201698D7A8D8B8D22
:101830009C8D0E9482E2698F7A8F8B8F9C8FA3018F
:1018400092016D8D7E8D8F8D98A10E9482E26D8FA9
:101850007E8F8F8F98A3A3019201C701B6010E94CA
:1018600082E269A37AA38BA39CA380E1E4E4FBE07A
:101870008E010F5F1F4FD80101900D928A95E1F7FD
:101880000E94A2C12B013C0128EC420E511C611C9C
:10189000711C0DA31EA381E0281A310809F45FC052
:1018A0000E94A2C18B019C01041915092609370960
:1018B00037FD86C02B013C0128EC420E511C611CF7
:1018C000711C0E9433402D893E894F89588D698152
:1018D0007A818B819C810E9413E969837A838B834F
:1018E0009C83298D3A8D4B8D5C8D6D817E818F819E
:1018F00098850E9413E96D837E838F8398872D8D51
:101900003E8D4F8D58A169857A858B859C850E9477
:1019100013E969877A878B879C8729A13AA14BA114
:101920005CA16D857E858F8598890E9413E96D87FE
:101930007E878F87988B750164018E010F5E1F4F24
:101940009E01235F3F4FAE01475F5F4FBE016B5F5C
:101950007F4F8DA19EA10E9459B981119CCF750125
:1019600064018E010F5E1F4F29EF33E045EF53E016
:1019700061EF73E08DEE93E00E9459B980E1EDEEE6
:10198000F3E0A4E4BBE001900D928A95E1F7A696FE
:101990000FB6F894DEBF0FBECDBFDF91CF911F9180
:1019A0000F91FF90EF90DF90CF90BF90AF909F90FE
:1019B0008F907F906F905F904F903F902F90089501
:1019C0000E94758680CF2F923F924F925F926F92C6
:1019D0007F928F929F92AF92BF92CF92DF92EF92BF
:1019E000FF920F931F93CF93DF93CDB7DEB761972D
:1019F0000FB6F894DEBF0FBECDBF898BE82EF12C59
:101A0000F701E550F94D6491062E000C770B880B19
:101A1000990B0E9423E24B015C011701220C331C3D
:101A2000220C331CF101E955F94E25913591459170
:101A30005491C501B4010E9482E22B013C01F101E5
:101A4000E556F94E659175918591949120E030E0CD
:101A500040EC5FE30E9482E2A50194010E9482E2D1
:101A6000AB01BC0100E010E0980189890E9467BBCE
:101A700020E030E0A901C301B2010E941CE28823EA
:101A800009F441C0B301A201705800E010E09801D0
:101A900089890E9467BBA3019201C301B2010E9420
:101AA00013E92B013C01F701E856F94E149111118D
:101AB00007C00E94673A86E796E10E94A2391AE0C1
:101AC0008989823008F0CBC060E070E88BE395E450
:101AD00020E030E040E752E40E9496E96B017C018F
:101AE000612F70E090E080E00E9421E29B01AC0158
:101AF000C701B6010E9496E98B019C01B301A201C6
:101B000089890E9467BB81E090E0A0E0B0E009888D
:101B100004C0880F991FAA1FBB1F0A94D2F72091F7
:101B20009405282B2093940520917E04822B80938A
:101B30007E04F101E659F94E85919591A591B491F4
:101B400081010C5B144FF80180839183A283B383DE
:101B5000F101EF51FC4F10821182128213828989A8
:101B60000E944B850E947386F801C080D180E2807C
:101B7000F380F101E351FC4FC082D182E282F38213
:101B80008CE0E7ECF1E0DE01119601900D928A9570
:101B9000E1F7E1E0F0E0EC0FFD1FE20DF31D408006
:101BA00051806280738020E030E0A901C301B2015E
:101BB0000E941CE28823D1F120E030E0A901C3019A
:101BC000B2010E9496EA87FF04C077FA709477F812
:101BD000709481010C5B144FA3019201C501B40103
:101BE0000E9482E29B01AC01C701B6010E9412E98A
:101BF000F8016083718382839383F98960E070E8E0
:101C00008BE395E4F23020F060E070E080E793E44D
